:020000040800F2
:10000000F8FF012029830908C5830908F96E05084E
:10001000C5830908C5830908C583090800000000D5
:10002000000000000000000000000000C583090877
:10003000C583090800000000C5830908315604087B
:10004000C5830908C5830908C5830908C58309084C
:10005000C5830908C5830908E9270408112804088D
:100060003928040861280408892804084903000085
:100070005D03000071030000850300009903000088
:10008000AD030000C1030000C5830908C58309084A
:10009000C5830908C5830908C5830908B128040870
:1000A000C5830908C93B0408C5830908B93B04088E
:1000B000D93B0408E93B0408F93B0408B91A0408D1
:1000C000AD1A0408ED1A0408E11A0408C5830908EA
:1000D000C5830908413C0000913D0000FD3E000041
:1000E000F1280408C583090800000000B53C040895
:1000F0008D3C0408C53C04087D3C0408D503000081
:10010000C5830908C5830908093C0408C583090893
:100110006D400000DD410000193C040899C3080847
:10012000E9030000FD0300001104000025040000A5
:1001300039040000C5830908C5830908C583090877
:1001400000000000000000000000000000000000AF
:100150004D04000061040000750400004D430000E0
:10016000211B0408151B0408C5830908C583090859
:10017000C5830908C5830908C58309080000000074
:10018000C5830908C5830908BD4400002D46000049
:10019000C5830908C5830908C5830908C5830908FB
:1001A000C5830908C5830908C5830908C5830908EB
:1001B000C5830908C5830908C5830908551B0408B8
:1001C000491B0408C5830908C5830908C5830908B4
:1001D000C5830908D9B90808C5830908C583090872
:1001E000C5830908C5830908C5830908C5830908AB
:1001F000C5830908C5830908C5830908C58309089B
:10020000C5830908C5830908C5830908C58309088A
:10021000D53C0408E53C0408F53C0408C5830908FE
:10022000C5830908C5830908C583090800000000C3
:10023000C5830908C583090800000000C5830908B3
:10024000C5830908C5830908C5830908C58309084A
:10025000C5830908C5830908C5830908C58309083A
:10026000C5830908C5830908C5830908C58309082A
:10027000C5830908C58309089D47000000000000E8
:10028000C583090800000000C583090800000000BC
:0802900000000000C58309080D
:020000040804EE
:10000000114A037A0168D35C10B4CC58CA1824F0A2
:100010000104CC501368DB07FCD4037D1F2B09D9E6
:10002000203B20225DF8044B02FA03F343F018034F
:10003000CB60704720225DF8044B02FA03F343F0D3
:1000400018038B60704700BFD4230A084368426DD1
:1000500030B49A61EFF31182502383F31288416820
:10006000D2B2856C0B68046D23EA050323430B6051
:1000700082F31188436981681A68096822F00102D5
:10008000D0E908541A60826A1D605C615A60D0E948
:100090000B429C60DA600023B0F86C2030BCCA626E
:1000A00003777047002A4FEA014C034630B508BF7A
:1000B000E64600F1C00514BF8E468C460024196840
:1000C0000C3353F8042C43F8084C41EA0C0142EA83
:1000D0000E02AB4243F80C1C43F8042CEFD1D0F8CD
:1000E000C03043EA0E03C0E93144C0F8C03030BD2F
:1000F00010B40C4C6368002B11DD002004F1080CD7
:100100000146DCF8AC3003F1C00259600C33934275
:10011000FBD1013063680CF5867C8342F1DC5DF82D
:10012000044B704704000020F0B5404C04EB401332
:1001300093F8543403B9F0BD3D4B42011D7893F858
:1001400001C065450CD00CEB4C0E03EBCE0E9EF8B7
:1001500004604FEA4C0E771E012F5AD9032E52D05D
:100160002244A2F83814EFF31181902383F312880C
:1001700092F83A34C9B2B2F8380443EA4003002096
:100180009BB282F83A0481F311881909207881EA38
:1001900013215940D8B1C9431B01D2F8505401244E
:1001A000D2F83C049BB201F00F01D5F8AC2084409A
:1001B0000B4302F1C000590013F4004F8BB202D17F
:1001C0005168214351600C329042F4D1F0BDD2F815
:1001D0003C041B01D2F8502401F00F0110309BB2F7
:1001E0000124D2F8AC200B43844002F1C000590036
:1001F00013F4004F8BB202D15168214351600C328D
:100200009042F4D1F0BD0CF1010606F00306AE42B7
:10021000A6D0E64403EBCE030344597C00299FD0CB
:10022000A318012083F83A049AE700BF04000020D5
:10023000601B0024704700BF024B03EB401393F890
:100240005504704704000020D0E90920131A5842D1
:100250005841704790F8573830B53BB990F8551869
:10026000012490F85638DAB2914200D830BD04FA31
:1002700003F2B0F85E5801332A43A0F85E28F2E793
:100280000379024613F0010006D0D2E90731D268A3
:100290005B1A013A03EA0200704710B5037904467D
:1002A00013F001030ED0FFF7EBFF034650B1226AB3
:1002B0006369E1689B5C0132B2FBF1F0DBB201FBE8
:1002C00010222262184610BD03799B070AD5436AA3
:1002D0008269D154436A02690133B3FBF2F102FB34
:1002E00011334362704770470171704703790146CB
:1002F00013F0020007D00B69D1E90921013B521A22
:100300001A40D2B2981A70472DE9F04F4C484FF07E
:10031000010A4C494FF002094B4B4FF004080827E3
:100320001026202540244FF0800EDFF820C130F841
:10033000022F12F0010F03D01960083323F804AC28
:1003400012F0020F03D01960083323F8049C12F056
:10035000040F03D01960083323F8048C12F0080F3F
:1003600003D01960083323F8047C12F0100F03D077
:100370001960083323F8046C12F0200F03D01960C1
:10038000083323F8045C12F0400F03D019600833DF
:1003900023F8044C12F0800F03D01960083323F8BF
:1003A00004EC12F4807F05D04FF4807B1960083391
:1003B00023F804BC12F4007F05D04FF4007B1960D1
:1003C000083323F804BC12F4806F05D04FF4806B1F
:1003D0001960083323F804BC12F4006F05D04FF401
:1003E000006B1960083323F804BC12F4805F05D059
:1003F0004FF4805B1960083323F804BC12F4005FEB
:1004000005D04FF4005B1960083323F804BC12F4E4
:10041000804F05D04FF4804B1960083323F804BC9B
:10042000D20B05D04FF400421960083323F8042C96
:1004300001F5806161457FF47AAFBDE8F08F00BFC0
:1004400026A1090800000258C41B002400240258F9
:1004500010B584464FEA810E102312F4004F4FEA84
:10046000420214BF0E240724013B92B2CCF8004094
:10047000F444F2D100EB81128C010351122042F8B6
:10048000213010BD10B584464FEA810E0424130BB1
:10049000013C4FEA021203EB430392B203F118034B
:1004A000CCF80030F444F2D100EB01130A0184507F
:1004B000062043F8214010BD704700BF704700BFC1
:1004C00000EB4000024B03EBC00393F84905704773
:1004D00004000020064B93F8F825824206D900EB71
:1004E000400003EBC003D3F84C0570470020704771
:1004F000040000201D4B93F8FC25AAB3D3F838154F
:1005000009B100200860012A2ED0D3F8501509B196
:1005100000200860022A27D0D3F8681509B100200E
:100520000860032A20D0D3F8801509B100200860A4
:10053000042A19D0D3F8981509B100200860052ABB
:1005400012D0D3F8B01509B100200860062A0BD0EC
:10055000D3F8C81509B100200860072A04D0D3F8E1
:10056000E0350BB100221A60704700BF0400002084
:100570001D4B93F8FC25AAB3D3F8381509B1002018
:100580000860012A2ED0D3F8501509B10020086068
:10059000022A27D0D3F8681509B100200860032A81
:1005A00020D0D3F8801509B100200860042A19D0A2
:1005B000D3F8981509B100200860052A12D0D3F8A5
:1005C000B01509B100200860062A0BD0D3F8C81571
:1005D00009B100200860072A04D0D3F8E0350BB138
:1005E00000221A60704700BF04000020C44B1B7833
:1005F000002B40F04F81C34B93F8FC25002A00F0FC
:10060000498193F8481530B500294ED1D3F83815F3
:100610000020012A086047D993F86015002966D1A7
:10062000D3F850150020022A08603DD993F87815B8
:10063000002940F0CB80D3F868150020032A086019
:1006400032D993F89015002940F0E280D3F8801554
:100650000020042A086027D993F8A815002940F043
:10066000F880D3F898150020052A08601CD993F863
:10067000C015002940F00F81D3F8B0150020062ADC
:10068000086011D993F8D815002959D1D3F8C815A5
:100690000020072A086007D993F8F025002A73D1B3
:1006A000D3F8E03500221A6030BDD3F83C25910A1A
:1006B000A1F58011522940F20F814FF0FE0CEFF3AB
:1006C0001181502080F312888F4C4FF02C0E556A08
:1006D000C9B250690EFB0C4C013540F00100CCF85A
:1006E0000C55506181F3118893F8FC258EE7D3F8FF
:1006F0005425910AA1F58011522940F2F2804FF061
:10070000FE0CEFF31181502080F312884FF02C0E75
:10071000556A7D4CC9B2506901350EFB0C4440F05E
:100720000100C4F80C55506181F3118893F8FC2541
:100730000020D3F85015022A08603FF677AFB3E7E0
:10074000D3F8CC25910AA1F58011522900F2EA8054
:100750006E48014491F814C0EFF31181502080F3EA
:1007600012884FF02C0E556A674CC9B2506901359A
:100770000EFB0C4440F00100C4F80C55506181F3AD
:10078000118893F8FC2581E7D3F8E425910AA1F5B7
:100790008011522900F2C9805C48014491F814C0CC
:1007A000EFF31181502080F312884FF02C0E556A20
:1007B000554CC9B2506901350EFB0C4440F00100A4
:1007C000C4F80C55506181F3118869E7D3F86C25A2
:1007D000910AA1F58011522940F288804FF0FE0E57
:1007E000EFF31181502080F312884FF02C0C556AE2
:1007F000454CC9B2506901350CFB0E4440F0010074
:10080000C4F80C55506181F3118893F8FC2512E768
:10081000D3F88425910AA1F5801152296BD94FF0A4
:10082000FE0CEFF31181502080F312884FF02C0E54
:10083000556A354CC9B2506901350EFB0C4440F085
:100840000100C4F80C55506181F3118893F8FC2520
:10085000FCE6D3F89C25910AA1F58011522957D9BD
:100860004FF0FE0CEFF31181502080F312884FF00F
:100870002C0E556A244CC9B2506901350EFB0C444C
:1008800040F00100C4F80C55506181F3118893F8D1
:10089000FC25E6E67047D3F8B425910AA1F580114E
:1008A00052293AD94FF0FE0CEFF31181502080F31A
:1008B00012884FF02C0E556A134CC9B2506901359D
:1008C0000EFB0C4440F00100C4F80C55506181F35C
:1008D000118893F8FC25CFE60C48014491F814C028
:1008E000EDE60A48014491F814C00AE707480144BC
:1008F00091F814E074E70548014491F814C090E7BA
:100900000000002404000020601B002428A1090826
:100910000748014491F814C0A4E70548014491F840
:1009200014C0C1E74FF0FE0C16E74FF0FE0C37E79E
:1009300028A1090800EE100AB8EE400A704700BF6F
:10094000BCEEC00A10EE103A98B2704707280AD8D9
:100950004FF4B472054B02FB0033B3F80006B0FA53
:1009600080F0400970470020704700BF040000205D
:10097000072807D8044B4FF4B471012201FB003360
:1009800083F80226704700BF04000020072808D81B
:10099000044B03EB401393F8542412B1012283F863
:1009A0003A24704704000020072808D8054B03EBC1
:1009B0004013B3F83804B0FA80F0400970470020C3
:1009C000704700BF04000020054B93F8F8258242D1
:1009D00004D903EB4013D3F8440470470020704758
:1009E00004000020436A02461B681B6A5B689B7810
:1009F00013F0010008BF5077704700BFC2628161E9
:100A0000704700BF0346012200205A77704700BF9D
:100A1000826908B50346006BD96A02449A6101B144
:100A20008847002008BD00BF704700BF04307047F2
:100A30000C4B93F87C27D3F8781702440144D2B2C8
:100A4000C3F8781783F87C2793F87C27120605D51E
:100A500093F87C2782F0800283F87C27024B0122E6
:100A60005A707047601B0024000000242DE9F84FE5
:100A7000164FD7F88057ED0A23D00026DFF850A094
:100A800007F28479B0467419D7F884174FF0100331
:100A9000524648BF0134D1F828B04846C7F8B0875D
:100AA0006410E102D8470F280BDD094B03F1100158
:100AB00053F8042B013207D18B42F9D12546B542B8
:100AC000E1DCE802BDE8F88F661CF8E7601B002453
:100AD00060E30024194BD3F8B817D3F8BC278A1A5F
:100AE000322A05DCD3F8D0278A1A002A11DC704795
:100AF000D3F8C01749B193F8CC27888802F00102D7
:100B00000968120100FA02F28A610022C3F8D027B4
:100B10007047D3F8C0276AB110683231928810B498
:100B20004469C3F8D01722425DF8044B18BF120481
:100B3000826170473231C3F8D0177047601B0024C0
:100B4000074AD2F8C0374BB192F8CC279988186879
:100B500002F001031B0101FA03F3836100207047D7
:100B6000601B0024044B4FF4007C0020D3F8E037D6
:100B7000A2F800C00B607047601B00240020704783
:100B80000120704701207047002070472DE9F04197
:100B90004FF425728EB00021734858F04DFF734B0F
:100BA000734D4FF00008D3F8F02040F27D27A5F1F7
:100BB000680605F6F41442F00102C3F8F020D3F8F9
:100BC000F02002F001020092009AD3F8E82042F0EF
:100BD0000102C3F8E820D3F8E82002F001020192F4
:100BE000019AD3F8E82042F00202C3F8E820D3F8D3
:100BF000E82002F002020292029AD3F8E82042F0C2
:100C00000402C3F8E820D3F8E82002F004020392BB
:100C1000039AD3F8E82042F00802C3F8E820D3F89A
:100C2000E82002F008020492049AD3F8E82042F087
:100C30001002C3F8E820D3F8E82002F01002059271
:100C4000059AD3F8E82042F02002C3F8E820D3F850
:100C5000E82002F020020692069AD3F8F02042F033
:100C60000202C3F8F020D3F8F02002F0020207924B
:100C7000079AD3F8E82042F04002C3F8E820D3F8FE
:100C8000E82002F040020892089AD3F8E82042F0E7
:100C90008002C3F8E820D3F8E82002F0800209922D
:100CA000099AD3F8E82042F48072C3F8E820D3F818
:100CB000E82002F480720A920A9AD3F8F02042F4F3
:100CC0008032C3F8F020D3F8F02002F480320B9287
:100CD0000B9AD3F8F02042F40032C3F8F020D3F896
:100CE000F02002F400320C920C9AD3F8F02042F477
:100CF0008022C3F8F020D3F8F03003F480230D9362
:100D00000D9B55F82810002354F83320914226D02B
:100D100001330E2BF8D1002008F1070850F056FBE4
:100D2000B845EED14FF0000840F27D2755F8281065
:100D3000002354F8332091420CD001330E2BF8D10C
:100D4000002008F1070850F041FBB845EED10EB085
:100D5000BDE8F08106EBC303B3F8600AF1E706EBE8
:100D6000C303B3F8600AD7E74420002400440258C4
:100D700090A1090810B5044658F028F9014620460C
:100D800089B2BDE81040FFF7CFB900BF38B50B4DB1
:100D900000EB400005F5A763C40003EBC003254446
:100DA00093ED027AD3ED037AE7EE007AB0EE670AAC
:100DB00058F00CF9D5F83835186038BD040000201B
:100DC00002692DE9F843C36812EA030828D00546F2
:100DD0000E464FF00047B8FA88F327FA03F21B3BA0
:100DE000D24308EA02082A61042B16D8DFE803F090
:100DF0003B30251A0300B36A002B3FD003F1FF39C3
:100E000000231FFA89F9B362746A34B1236820465B
:100E1000494698476468002CF8D1B8F1000FDAD140
:100E2000BDE8F88370680028F7D0696B036889B261
:100E30009847B8F1000FCED1F2E7B0680028ECD0A7
:100E4000A96B036889B29847B8F1000FC3D1E7E7EF
:100E5000F0680028E1D0E96B036889B29847B8F1DF
:100E6000000FB8D1DCE730690028D6D0296C0368C0
:100E700089B29847B8F1000FADD1D1E7EB6A1FFAFC
:100E800083F9C1E72DE9F043144C83B0DFF85090AB
:100E9000DFF8508004F5906602E00834B44219D0BF
:100EA00094F90650002DF8D12768083407EB0803A1
:100EB0009B0A09EB4303B3F8CC0A50F087FA34F8E5
:100EC000041C01232A463846CDE9005553F034FA74
:100ED000B442E5D103B0BDE8F08300BFC41B0024D9
:100EE00028A109080000FEA78069B43047F060BE61
:100EF000F8B5A0F507642379DB0725D5657994F863
:100F0000543805F001073D46FBB1D4F848341A685F
:100F1000D36A5B08536294F8583823B1B4F8623846
:100F20000133A4F8623885F00101606C4EF062FE76
:100F3000012384F85738002384F8553884F856384C
:100F4000A4F85E3884F85438F8BD94F85768012E38
:100F500003D194F8553884F856382046FFF77AF9CB
:100F60004EB9012385EA030184F85738606CBDE867
:100F7000F8404EF03FBE0023394684F85738F5E775
:100F800038B549F0A1FA0D490D4CD1F8FC20A4FB6D
:100F900000400C4D42F080720B4B800CC1F8FC20DD
:100FA0004FF060420949C5F86008C2F8B01F00223E
:100FB0005A601A6842F001021A6038BD00ED00E084
:100FC00083DE1B43601B0024001000E055CEACC53F
:100FD00019484FF6FF0C194A84B0C168184B01EA52
:100FE0000C010A43C260D3F8D020D3F8DC2042F0D1
:100FF0000052C3F8DC20D3F8DC2002F0005201924A
:10100000019AD3F8DC2042F08042C3F8DC20D3F808
:10101000DC2002F080420292029AD3F8DC2042F0F7
:101020000042C3F8DC20D3F8DC3003F00043039324
:10103000039B04B0A4E700BF00ED00E00005FA0543
:101040000044025870B505460A26084C013E00D1FE
:1010500070BD94F9000019F0F5FD031E04DB617802
:10106000EA185172A278EA540434EFE706AC090892
:1010700010B590F828300446012B03D0002301203E
:10108000637710BD406A03681A7B42B954F002FED0
:1010900000F00103C243637702F00100F1E71B6A2D
:1010A000002BF3D0002010BD38B5114D044694F844
:1010B0002830012B05D00023637700230120236211
:1010C00038BD606A03681A7B72B954F0E3FD00F022
:1010D00001036377C307F0D5D5F8B837226A9B1AA6
:1010E000002BE4DB002038BD1B6A002BEDD0F3E7BA
:1010F000601B002410B5FF22044690F82810406AB7
:1011000056F054FB0E4B2046D3F8B8370233236217
:10111000FFF7CAFF94F82830012B00D010BD002241
:10112000A021606A56F0F8FA94F82830012BF5D126
:10113000606A1822B021BDE8104056F0EDBA00BF39
:10114000601B002438B504460D46FFF7ADFF0622AC
:1011500094F82810606A56F029FB012294F8283090
:101160006277934205D0074BD3F8B8370F33236229
:1011700038BDE288D821606AB5FBF2F256F0F2FA87
:10118000F1E700BF601B00242DE9F843838853B3C7
:1011900004460025DFF85480012707E0D8F8B83767
:1011A0000135A2880F33AA4223621CD92046268A21
:1011B000B4F80690FFF778FF062294F82810606ACA
:1011C00056F0F4FA94F828306777012BE6D109FB42
:1011D00006F6E288D821606A05FB06F6B6FBF2F255
:1011E00056F0C0FADAE7BDE8F88300BF601B0024C0
:1011F00070B5104D95F8643803B970BDC3880446C6
:10120000D5F86868B6FBF3F60B4B5E60FFF74CFF52
:1012100094F82830012B07D0D5F8B83700220233D4
:1012200085F86428236270BD32461021606A56F04A
:1012300099FAF1E7601B0024000000242DE9F04F2B
:10124000584F0C461D46C18897F8643899B0064639
:101250009046B4FBF1F903BBDFF854A1DAF804308F
:101260004B452FD101FB194496F82830091BA942A0
:1012700034BF8DB2ADB2012B4ED0D7F8B83730465F
:1012800002333362FFF710FF80B396F82830012B4A
:1012900036D0284619B0BDE8F08FD7F86828DFF8B7
:1012A00010A1B2FBF1FBCAF804B0FFF7FDFE96F8FF
:1012B0002830012B69D0D7F8B837023333620023C6
:1012C00087F864383046FFF7EFFE78B14FF0FF3310
:1012D000CAF8043096F82830012B5CD0D7F8B8371C
:1012E000304602333362FFF7DFFE18B9002019B031
:1012F000BDE8F08FF188CAF80490B4FBF1F9B1E7CA
:10130000706A54F0C7FCC0F30113023B012BC0D834
:101310003046FFF7EFFEBCE78DF81C3000228DF859
:10132000443004A98DF858301F4B8DF80E40240A24
:101330001B688DF80D40ADF808301B0C746A8DF8F1
:101340000A3003232046CDF83C808DF80C300693FC
:10135000164B1095089303AB8DF80F2009930423C7
:101360000A920B9302AB8DF83020049301AB1792D5
:101370000593CDE90D22CDE91222CDE9142241F0E9
:101380008FFD206854F082FC77E75A461021706A7E
:1013900056F0E8F98FE74A461321706A56F0E2F9F1
:1013A0009CE700BF601B002400230A08E50904082D
:1013B000000000242DE9F04FD0F8249083B03F4F77
:1013C0000446D9F800000E46904654F05FFC97F8AA
:1013D0006438002B40D0D7F86C58E288DFF8E8B0CA
:1013E000DFF8E8A0B5FBF2F302FB13538BF82230D1
:1013F0001B0A8BF8213033685146314E4846C6F8F7
:10140000A83006F1A802D8F80030C6F8B0300023A2
:10141000C6F8B83043F09CF9D8F800200123E188E1
:10142000154487F86438B5FBF1F301FB1353C7F893
:101430006C581BB3234BC6F8B830637F0BB90AF165
:10144000140A51464846226341F02AFDE36A6BB311
:10145000206B03B0BDE8F08FA569E288DFF868B0C3
:10146000DFF86CA0C7F86858B5FBF2F302FB135322
:101470008BF842301B0A8BF84130BCE7D7F868285C
:1014800048460193B2FBF1F2726052BA06F1A8012C
:10149000ABF8622006F1D00243F05AF9019BD8F86C
:1014A000002087F86438C7F86858C6E7636A186888
:1014B00054F0ECFB206B03B0BDE8F08F601B002400
:1014C00000000024110A040860E30024080000243E
:1014D0005800002433B910B51C46C36A204698470B
:1014E000204610BD66E700BF10B582B00C460192E1
:1014F00001A9049A8461C2626A460093FFF75AFF09
:1015000002B010BD2DE9F843DDF820800F461646E5
:101510000021202204461D4658F08EFAB8F1000F33
:101520000CD0D8F80030B8F80A20E3811B0C2382D5
:10153000D8F804306282E3821B0C2383384656F0CD
:101540000BFAF30619D4431EB8B107EB000C01E007
:10155000013B12D31CF801EDBEF12E0FF8D1C01AD9
:1015600003F10109421EB944032AA8BF0322082B34
:10157000A8BF082390461A4606E008280246B94646
:101580004FF00008A8BF08224FF02033394620460C
:101590002360636058F0F2F9164B04F108004246EC
:1015A00049462381837058F0E9F9611EE21D11F864
:1015B00001CFACF16103ACF1200C192B98BF81F87D
:1015C00000C09142F3D104F10A0011F8013FA3F1E8
:1015D0006102203B192A98BF0B708142F5D1182374
:1015E00065832D0CE6722373099BA582E361BDE838
:1015F000F88300BF202020002DE9F04FDFF8589439
:1016000085B0D9F8B807C9F8BC07002B60D00C46E4
:10161000154601F5FE7603EB020B1FE0002D64D0AA
:10162000D9F8EC37AB4200F0C780D9F8E837AB42C5
:1016300000F0F980D9F8F037D9F8F417AB424BD85D
:101640008D42C0F07481691A20464DF089FC013545
:1016500004F5007406F500765D4539D0D9F8F82711
:10166000AA42DBD8AA1AD9F80878D308396B02F055
:10167000070802338B4202D3BA6B93420BD9394627
:10168000184603934DF03CFC039B0746002800F0EE
:101690006E81C9F808083A79002A40F01F81D7F80E
:1016A00028A0BAF1000F00F05B813A6B01352046AB
:1016B0004FF400719B1AFA6804F5007406F5007681
:1016C00008EBC3083B4602EB4822D0475D45C5D135
:1016D000002005B0BDE8F08F8D42B4D24FF4007207
:1016E0000021204658F0A8F9B1E74FF400722946CE
:1016F000204658F0A1F98023CB4A84F8BE310C2350
:1017000084F8C231D9F8E817D9F8E0379142C4F823
:10171000C611C4F8CA3100F30F81C44A013BC44F5B
:1017200082FB0102C81787FB01C70A44C0EB6212A3
:10173000C0EB2730BF4F87FB02C7C2EB821C84F887
:10174000C1018010A1EB0C01174420F03F000131D2
:101750000843D117C1EBE71184F8C0010A4484F8AB
:10176000BF21B14A934200F3F380B04AB04882FBF4
:101770000312D91780FB03701A44C1EB6212C1EB4C
:101780002031AC4880FB0270C2EB821784F8C5118F
:101790008910DB1B104421F03F0101331943D3179B
:1017A000C3EBE01384F8C4111A4484F8C3214AF649
:1017B0005523A4F8FE314AE74FF0FF3300274FF4DA
:1017C000F072201D84F8EC31394684F8ED3184F84C
:1017D000EE3184F8EF315223237063706123A370DC
:1017E00084F8E7314123E37084F8E631722384F80A
:1017F000E43184F8E531D9F80038C4F8E83158F01C
:101800001BF95523C4F8F07184F8FE316FF05503CD
:10181000C4F8F471C4F8F87184F8FC7184F8FD71AF
:1018200084F8FF3113E74FF400720021204658F08E
:1018300003F9814B022203CB45F6EB03227422739A
:1018400023809023A273A370F82384F82C2008220D
:10185000C4F803006273C4F807106375D9F8E81779
:10186000D9F8E0375B1AD9F8F0172362D9F8F437C2
:101870005B1A4AF6552163620023E372E3736377D0
:10188000A377E37784F82D3084F82E3084F82F3056
:1018900084F83130694BA3613E232377012384F818
:1018A0003030802384F84030654BC4F84230654BBB
:1018B00084F84620A4F8FE11634A03CBC4F84B1009
:1018C0001988C4F847009B78A4F84F1084F8513069
:1018D00003CAC4F85200C4F85610B8E64FF40072B8
:1018E0000021204658F0A8F83B6CB8F1000F45D114
:1018F00004F1200A002B00F081803B6B1122534938
:101900002046CDE90088FFF7FDFD3B6C1A6C002AEC
:1019100000F081801B6B504611224D49CDE90088B3
:10192000FFF7F0FD04F1400A4FF4E07871E0E91AA6
:1019300020464DF015FB8AE6FF22013B84F8C121C9
:101940004FF6FF72A4F8BF21374A93427FF70DAFDD
:10195000FF2384F8C5314FF6FF73A4F8C33126E79F
:1019600051464FF40072204658F066F86FE6231F88
:10197000384A43F8042F9E42FBD168E6002B7F6C67
:1019800014BF02230123C3EB0813002F3FF45FAE03
:10199000013BBF6C002B01DD002FF9D1A2464FF4B3
:1019A0000078002F3FF453AE0AEB080303959A46E4
:1019B0000BE00025A8F12008CDE900E5FFF7A2FD26
:1019C000BF6CCFB1B8F11F0F16D93D7907F11C0ECE
:1019D000112239683B6BAAEB0800002DE9D17A7916
:1019E000A8F120083D6942F02102CDE900E5FFF7AA
:1019F00089FDBF6C002FE5D1039D28E6CDE9008865
:101A000043464FF4F0780822D9F8E4172046FFF750
:101A100079FD7F6CC5E75046434611220C49CDE95C
:101A20000088FFF76FFD7DE7FF03FB00832008823E
:101A300097554541818080800C230A083F00FF00B4
:101A400029940E0D18230A0824230A0804230A08DF
:101A500008230A08DEADBEEF601B002430B40D4C35
:101A6000BFF34F8F0C4BC3F85C42BFF34F8FBFF3F4
:101A70006F8F0A4B0A4D03F13000DA792AB1597998
:101A800034F8112092B225F811200C338342F4D19E
:101A900030BC704700E7002400ED00E0D0230024B4
:101AA00020E6002400207047704700BF014848F03E
:101AB000C7B900BF3C240024084810B4D0F8DC3873
:101AC000D0F8104999691A682CB1234600F6DC0059
:101AD0005DF8044B18475DF8044B7047601B002409
:101AE000014848F0ADB900BFA0240024084810B454
:101AF000D0F84039D0F8744999691A682CB1234656
:101B000000F514605DF8044B18475DF8044B70470E
:101B1000601B0024014848F093B900BF042500244D
:101B2000084810B4D0F8A439D0F8D84999691A688F
:101B30002CB1234600F6A4105DF8044B18475DF85D
:101B4000044B7047601B0024014848F079B900BF7E
:101B500068250024084810B4D0F8083AD0F83C4A68
:101B600099691A682CB1234600F608205DF8044BE9
:101B700018475DF8044B7047601B0024B0F1FF3F2D
:101B800000F0628203282DE9F04F054683B000F390
:101B90002B816420BE4C05FB00F004EB000CDCF84C
:101BA000DC080CF6DC0B002800F01E81FF2A4FEA4F
:101BB00041077ED09CF81D19202940F00F819CF828
:101BC0001C19012900F00A810121D4F8548A8CF8EB
:101BD0001C1906E0D4F8541AA1EB0801192900F2E7
:101BE0000781816911F40049F4D14FF0640A0C991E
:101BF000CDF8008058460AFB054ACAF80019222190
:101C0000CAF810998AF81D1940218AF81E19394618
:101C1000CAF82099AAF806390A234FF007FA0028D3
:101C200040F00281BAF806399BB2FF2B40F2E58101
:101C3000DAF8DC18FF239748AAF804394B68964A6B
:101C400003403B431A434A604FF0640909FB0549CE
:101C500006E0D4F8543AA3EB08030A2B00F23C81C7
:101C60008A6912F00402F4D04A6AD9F800391A706D
:101C7000B9F80639D9F80029013B01329BB2C9F8FD
:101C80000029A9F80639B9F80439B9F80629013B41
:101C900092B29BB2A9F8043912B1002B00F0548122
:101CA000B9F806399BB2002B00F0B981D9F8DC18DD
:101CB000D6E79CF81D29202A40F090809CF81C292A
:101CC000012A00F08B8001228CF81C29D4F854CA18
:101CD00006E0D4F8542AA2EB0C02192A00F28880FC
:101CE000826912F40042F4D164214FF0220E0C9E5E
:101CF00001FB054181F81DE94FF0100EC1F80069A4
:101D000081F81EE9C1F82029A1F80639B1F8063991
:101D1000C1F810299BB2FF2B7BD8B1F80639426875
:101D20009BB2A1F80439DBB25A4947EA03430A409F
:101D300013435A4A1A4342604FF0640808FB0548AF
:101D4000B8F806399BB2002B00F03B81D8F8DC18BC
:101D50000BE08B6913F0200340F0CE80D4F8542AB6
:101D6000A2EB0C020A2A00F2E1808B695B076ED4B9
:101D70008B69DB06EDD58B6913F0200309D1D4F80C
:101D8000542AA2EB0C020A2A51D88B6913F02003C3
:101D9000F5D020231022CA61CB618B699E0701D543
:101DA00000238B628B69D80703D48B6943F001034E
:101DB0008B614A6864233A4E002003FB054332409E
:101DC00020264A60D3F8202983F81C0942F0040237
:101DD000C3F8202983F81D6983F81E09B4F8583A1E
:101DE00001339BB2A4F8583A002003B0BDE8F08F4D
:101DF00064232020002103FB0543D3F8202983F826
:101E00001C190243C3F8202983F81D0983F81E1901
:101E1000E4E743681F4A13401F4A3B431A43FF232A
:101E2000A1F80439426087E78AF81C99D6E7642252
:101E3000202002FB0542D2F8201982F81C39014308
:101E4000C2F8201982F81D0982F81E39C6E74A6ACD
:101E5000D8F800391A70B8F80639D8F80029013BCB
:101E600001329BB2C8F80029A8F80639B8F804393D
:101E7000B8F80629013B92B29BB2A8F80439002AAF
:101E80003FF45EAF002B7FF45BAFD8F8DC180FE0B7
:101E9000601B0024009800FC0024FF8100240082C5
:101EA00000E800FED4F8543AA3EB0C030A2B13D835
:101EB0008A6912F08002F5D0B8F806399BB2FF2B80
:101EC0005FD94B68614A1340614A3B431A43FF2381
:101ED000A8F804394A6033E76423202003FB054354
:101EE000D3F8201983F81C290143C3F8201983F87B
:101EF0001D0983F81E2971E78B695A0703D5B8F8C5
:101F00000439002BA3D12020524AC8614B681340EA
:101F100000224B60642303FB0543C3F8202983F8A8
:101F20001C2983F81D0983F81E2957E76422202005
:101F300002FB0542D2F8201982F81C390143C2F88D
:101F4000201982F81D0949E7D9F8DC1805E0D4F812
:101F5000543AA3EB08030A2BBED88A6912F0800218
:101F6000F5D0B9F806399BB2FF2B1AD94B68374A1E
:101F70001340374A3B431A43FF23A9F804394A6008
:101F80008EE6B8F8063931489BB24A68A8F8043999
:101F9000DBB2024047EA0343134343F000734B6054
:101FA000CEE6B9F8063929489BB24A68A9F804393F
:101FB000DBB2024047EA0343134343F000734B6034
:101FC0006EE6614658464FF069F8034600287FF4F4
:101FD00005AFD8F8DC2820201E4ED0615168314072
:101FE000516088F81D0988F81E39642200230120F9
:101FF00002FB054484F81C39F7E6BAF80639DAF82A
:10200000DC189BB214484A68AAF80439DBB20240D3
:1020100047EA03431343114A1A434A6014E6414610
:1020200058464FF03BF8034600287FF4D7AED9F866
:10203000DC282020074ED06151683140516089F87A
:102040001D0989F81E39D0E700207047009C00FC6C
:102050000000FF0100E800FE009800FC0024008260
:102060002DE9F0410468D4E90435A8611A7D1F68A0
:102070001F2A49D9203A20212E6801FA02F242F0A3
:102080001802FA602A7D1F2A48D9203A202101FA35
:1020900002F242F01802F2606A680021586801609A
:1020A00038461160116841F01001116093F8088002
:1020B000A269414651F0ACF92D7AE26930462946D1
:1020C00051F0A6F9226A63689468184A12F8080069
:1020D000515D5A686FF30F0222435A603A5842F03A
:1020E00001023A50725842F0010272509A6842F46A
:1020F00040429A601A6842F001021A601A6842F47B
:1021000000721A60BDE8F08120212E6801FA02F207
:1021100042F01802BA602A7D1F2AB6D8202101FA9F
:1021200002F242F01802B260B6E700BFD4230A08F8
:10213000D3B20F2B22D8124B00B503F17E0E02E072
:102140000333734517D093F800C08445F8D193F852
:1021500001C08C45F4D102EB42020A48997800EBA9
:10216000820300F59070C3F8281100EB820083F819
:1021700020115DF804FB00205DF804FB002070478F
:102180002CAC09080000002410B40C4C002304F609
:102190005C2C01E0152B0CD003EB430201331CF83F
:1021A00002108142F6D1144494F95E0A5DF8044BA2
:1021B00070474FF0FF305DF8044B7047601B002400
:1021C00030B5134D002305F6843C02E001331A2B91
:1021D0001BD05CF833408442F8D10CEBC30EDC001A
:1021E0009EF804E08E45F1D102EB4202094B2544F2
:1021F00003EB820103F5907395F8894B03EB8200A2
:10220000C1F8284181F8204130BD002030BD00BF19
:1022100028A1090800000024F0B1002310B50446ED
:102220000E4894F804E000F65C2C01E0152B11D068
:1022300003EB430201331CF802107145F6D18318F9
:102240006179206893F95E2AD3B20F2B02D8BDE8DA
:102250001040B5E7002010BD00207047601B00242F
:1022600001380E4B0E4A00EBC000D2F8D81003EB39
:10227000800310B4D3F8E03183B00A4CA34214BFFA
:10228000022301231943C2F8D810D2F8D8201340F2
:102290000193019B03B05DF8044B704700000024DC
:1022A00000440258000002400138F8B500EBC000BD
:1022B000124C1D46124B04EB800417460E46D4F810
:1022C000E001984214BFA120A0204FF07FF8B4F99C
:1022D000F601B909C4F8F061C4F8F8514EF014FBE6
:1022E000B4F9F631002B07DB03F01F0001225B0974
:1022F0000449824041F82320F8BD00BF00000024BB
:102300000000024000E100E02DE9F04F002385B01D
:10231000DFF800A34FF001090193B94B0AF1F00B6C
:10232000B84FA3F590780BE0019B09F101090AF180
:10233000280A0BF1050B0133062B019300F0F18005
:102340009AF80030022BEFD19BF90320511C00F0CA
:10235000EB80D2B2944602EB4204A94B9DF80410E4
:1023600003EB84040F2A5ED8A74802E00330B8428A
:1023700059D00378002BF9D145788D42F6D1857874
:10238000D8F8E4616068A560B042257000F044812F
:10239000D8F80862B04200F05E81D8F82C62B042F2
:1023A00000F06281D8F85062B04200F06281D8F843
:1023B0007462B04200F06C81D8F89862B04200F0CC
:1023C0008081D8F8BC62B04200F07681D8F8E06233
:1023D000B04200F08081D8F80463B04200F076810A
:1023E000D8F82833984200F08C81D8F84C339842C2
:1023F00000F08181D8F87033984200F0A581D8F8B8
:102400009433984200F09A81D8F8B833984200F09B
:10241000A781D8F8DC33984200F0A881D8F80034BE
:10242000984200F0978101320C34D2B2624599D9BA
:10243000002303939BF90420531C79D0D2B2964613
:1024400002EB42046E4B9DF8041003EB84040F2A48
:102450005DD86D4802E00330B84258D00378012BB4
:10246000F9D145788D42F6D18578D8F8E461606875
:10247000A560B04225705FD0D8F80862B04200F085
:10248000EF80D8F82C62B04200F0F880D8F85062A3
:10249000B04200F0F880D8F87462B04200F0FD80DD
:1024A000D8F89862B04200F00281D8F8BC62B0421D
:1024B00000F0F880D8F8E062B04200F01781D8F858
:1024C0000463B04200F00C81D8F82863B04200F0F9
:1024D0002481D8F84C33984200F01981D8F8703331
:1024E000984200F02581D8F89433984200F01A8180
:1024F000D8F8B833984200F04B81D8F8DC339842D2
:1025000000F04081D8F80034984200F03581013263
:102510000C34D2B296459AD200220023CAE9042391
:1025200002E705B0BDE8F08F4FF00F0C002212E774
:102530004FF00F0E002283E700231E46029306EBA6
:10254000C600013608EB800090F9FCC1BCF1000F19
:10255000DDD1624680F8E831AC462C4B1546029A34
:10256000C0F8ECC1134480F8FD91CAF8143013236D
:1025700080F8FC313046FFF773FE039B002BCBD075
:10258000DAF814402046FDF73BFDDAF81000FDF7BD
:1025900037FDDAF81830C168DAF8042059624021B2
:1025A0005D60996002F120019D631960C3E90355E4
:1025B000C3E90555C3E90755C3E90A55C3E90C55F5
:1025C000A4B1DAF81C303032E1681D625962C3E907
:1025D00000254FF48032C3E90255C3E90455C3E92D
:1025E0000655C3E90B55C3E90D559A6200233046E1
:1025F00007491A46FFF758FE01238AF80C3093E684
:1026000020010024AAAC09082CAC0908E001002430
:1026100045060000002600241846029300EBC00E79
:10262000013008EB8E0E9EF9FC61002E7FF4FBAEAC
:10263000029A8EF8E831594BCEF8EC5113448EF8DB
:10264000FD91CAF8103014238EF8FC31FFF708FE14
:1026500001230393EEE62420012302901846DDE7D0
:1026600024201E4602906AE7482002230290184662
:10267000D4E76C20032302901846CFE702234820BA
:102680001E4602905BE703236C201E46029056E72D
:102690009020042302901846C0E7042390201E4691
:1026A00002904CE70623D8201E46029047E70523F8
:1026B000B4201E46029042E7D82006230290184616
:1026C000ACE7B420052302901846A7E74FF49070BA
:1026D00002900820A2E7FC200723029018469DE7FD
:1026E0004FF4907308260293002328E70723FC2069
:1026F0001E46029023E74FF4B470022302900A2092
:102700008CE74FF4A27309200293012386E74FF46C
:10271000B47002230A26029011E74FF4A270092632
:1027200002900CE74FF4D8730C260293042306E7BB
:102730004FF4C6730B260293032300E74FF4D873BC
:102740000C200293042369E74FF4C6730B20029315
:10275000032363E74FF407730F20029307235DE71A
:102760004FF4EA730D200293052357E74FF4FC73EF
:102770000E200293062351E74FF407730F260293AE
:102780000723DCE64FF4FC730E2602930623D6E6FD
:102790004FF4EA730D2602930523D0E6E0010024EE
:1027A000800AA0F58010522807D8054B03441B7DF2
:1027B0000D2B02D8034AD05670470020704700BF47
:1027C00028A10908C4230A0860B182884FF0B041EB
:1027D0004FF00043B2FA82F2D1F88000D3400343B5
:1027E000C1F88030704700BF4FF0B042D2F880305F
:1027F000D2F888100B4003F00103C2F8883023B1EF
:10280000024BD3F8B00B036818477047601B0024D5
:102810004FF0B042D2F88030D2F888100B4003F06D
:102820000203C2F8883023B1024BD3F8B40B03681B
:1028300018477047601B00244FF0B042D2F8803038
:10284000D2F888100B4003F00403C2F8883023B19B
:10285000024BD3F8B80B036818477047601B00247D
:102860004FF0B042D2F88030D2F888100B4003F01D
:102870000803C2F8883023B1024BD3F8BC0B0368BD
:1028800018477047601B00244FF0B042D2F88030E8
:10289000D2F888100B4003F01003C2F8883023B13F
:1028A000024BD3F8C00B036818477047601B002425
:1028B000F8B54FF0B043D3F88050D3F888201540D6
:1028C00005F47875C3F888507DB1084F0126B5FA34
:1028D00085F4C4F11F0407EB840306FA04F4D3F86B
:1028E000B00B03689847A543F1D1F8BD601B0024E5
:1028F000F8B54FF0B043D3F88050D3F88820154096
:1029000005F47C45C3F888507DB1084F0126B5FA1F
:1029100085F4C4F11F0407EB840306FA04F4D3F82A
:10292000B00B03689847A543F1D1F8BD601B0024A4
:1029300030B1036882881B691A4214BF012000204D
:10294000704700BF10B1036882889A61704700BF6A
:1029500018B1838802681B049361704770B50D46F7
:1029600082B00446164640B101680C4B0C4A0B4439
:102970009B0A02EB4303B3F8CC0A4EF027FDC5F3E4
:102980008101C5F3411305F01302CDE90016A188BA
:10299000206851F0D1FC02B070BD00BF0000FEA75E
:1029A00028A1090800B1D9E770472DE9F84FC44FB5
:1029B0006423044603FB0073D3F8C468002E00F0C0
:1029C0006981D3F8CC88B8F1000F04D098F90630AB
:1029D000002B40F05F81642303FB0473D3F8D058CD
:1029E00025B195F90630002B40F05481631CDBB211
:1029F000B8F1000F04D0152288F8073088F80620B7
:102A000015B11622EB71AA714FF0640A308D4EF0A9
:102A1000DDFC29460AFB04FA404654F087F840469C
:102A200007EB0A09DFF8BC8299F8D63899F8D42860
:102A3000002B0CBF4FF01E0B4FF03E0B5946FFF71B
:102A4000B1FF28469F4D594699F8D5285544FFF7C0
:102A5000A9FF4C220021284656F0EEFFD9F8C438D1
:102A6000994A5B689342C9F8DC38DFF87C9240F001
:102A7000138147F04BFDD9F82030C3F302134344D0
:102A800093F8543C03F01F039FED907A9FED905A0A
:102A9000B0EE084AD8406423F7EE003A4FF0000C3D
:102AA00007EE900A03FB047340F21458F8EE677ABD
:102AB000B3F8D8A8C7EE275A07EE90AA9FED857AFB
:102AC000F8EEE77AC7EE274ADFED837AB0EE007AB8
:102AD000E5EE877AA5EE875A25EE844A37EE856AB9
:102AE00074EEE72ABAF5C87F0CF1010ED5BF4FF49A
:102AF000967278226423322307EE90EAD8BF4FF40F
:102B000016791344A2F13202F8EEE76AC8BF4FF417
:102B1000827907EE903AD4BF41464FF4FA7166EEDF
:102B2000A56AB8EEE77AC7EE267A07EE102A01EB1F
:102B30000902B8EEC77A37EE447A77EEE37AFCEE14
:102B4000E77A17EE903AC7EE267AFCEEE77A17EEB0
:102B5000900A07EE909AB8EEE73A07EE902AF8EE60
:102B6000E77A23EE243A83EE277A37EE453A32EEBF
:102B7000C77AC3EE267A77EEE37AFCEEE77A17EEB1
:102B8000901AC7EE267A77EEE37AFCEEE77A17EE34
:102B9000902A02F1020909EB010BB0EE467A07EE2A
:102BA00090BAF8EE677AA6EEA77AF4EEC74AF1EE8D
:102BB00010FA7DDC43EA00095FFA89F9B9F10F0FD9
:102BC00078D841EA02091FFA89F9B9F1FF0F71D8E3
:102BD0001B05000403F07F6392B200F47F000343FF
:102BE0003E4843EA0C7300EA01210B43134364227D
:102BF000284602FB04740027C4F8E0380123C4F817
:102C0000E478C4F8E838C4F8EC78C4F8F078C4F88C
:102C1000F878C4F8FC7851F041FB94F81D39202B6A
:102C2000D9B21AD194F81C39012B16D0242384F878
:102C30001D39D4F8DC381A6822F001021A601A68CB
:102C400022F480521A601A681A601A6842F001026F
:102C50001A6084F81D1984F81C79002196F82B005D
:102C60004DF052FE96F82B3001241D4D5A0903F009
:102C70001F03002104FA03F345F8223096F82A00D6
:102C80004DF042FE96F82A305A0903F01F039C408B
:102C900045F82240BDE8F88F47F038FCD9F81C30E1
:102CA000C3F30213984498F8543CEBE6F44619E752
:102CB000013170E7BEF10F0FF8D1002397E700BF95
:102CC000601B00243C240024001C0058286B6E4E1E
:102CD00000001643002474490000704200FFFF000A
:102CE00000E100E028A109080044025808B10022D0
:102CF00034E6704770B50E4C94F8F865AEB104F543
:102D00008764002503E001352034B5420DD0237FD0
:102D1000002BF8D0E06800220028F4D00135217D96
:102D2000FFF71CFE2034B542F1D1012070BD00BF79
:102D30000400002070B590F8EE311C09013C082C0D
:102D40000DD8194E054603F00F0336F8140040FA6B
:102D500003F2D20703D595F8F121012A01D0012011
:102D600070BD9A402644013A104057F015F896F885
:102D7000643C0E4A034402EBC30452F83320A38898
:102D800010691840ECD0002395F8EF21022120466D
:102D900085F8F131FFF7E2FDD5F85021136843F0D3
:102DA00008031360DBE700BF28A10908C41B002447
:102DB00038B5BFF34F8F6A4A6A49A2F58653C1F806
:102DC000683220339342FAD1BFF34F8FBFF36F8F36
:102DD000654C94F84D28B4F85C38022A11D094F868
:102DE0004D28012A00F08D80D4F810580C2B0CD8F7
:102DF000DFE803F0110B0B0B300B0B0B4D0B0B0B28
:102E00006A00002384F85E3838BD00236B6201231A
:102E100084F84D3838BDD4F83408544B544AC36450
:102E200090F83430C263012B00F09780012290F8B3
:102E30003530934280F8342000F0858000234FF431
:102E4000006280F8343042656B62EB6843F40073D3
:102E5000EB60DCE7D4F83808444B454AC36490F88B
:102E60003430C263012B61D0012290F83530934297
:102E700080F8342053D000234FF4006280F83430BF
:102E800042656B62EB6843F48063EB60BFE7D4F8A4
:102E90003C08364B364AC36490F83430C263012B89
:102EA0004ED0012290F83530934280F8342040D043
:102EB00000234FF4006280F8343042656B62EB68A7
:102EC00043F40063EB60A2E7D4F84008274B284A9C
:102ED000C36490F83430C263012B1DD0012290F8F6
:102EE0003530934280F834200FD000234FF4006235
:102EF00080F8343042656B62EB6843F48053EB60DA
:102F000085E7022284F84D286EE740F22A4305F156
:102F10004002184946F038FB00236B62ECE740F2B0
:102F20002A4305F13802134946F02EFB00236B6259
:102F3000A8E740F22A4305F13C020E4946F024FB83
:102F400000236B62BBE740F22A4305F134020949D2
:102F500046F01AFB00236B6277E700236B6274E78D
:102F6000A041012400ED00E0601B0024A15E0808E0
:102F7000F95E0808E0300124014B53F82000704747
:102F800050400058014B43F8201070475040005803
:102F900019481A4B01681A4A41F4807130B482B062
:102FA0000160D3F8F410FF24CA2041F48031C3F843
:102FB000F410D3F8F41001F4803101915321019DF4
:102FC000546250625162D3F8D030DB010CD40C4B08
:102FD00000220C495A659A65DA651A665A669A663D
:102FE000196502B030BC7047126D064B9A42EED1A3
:102FF00002B030BC704700BF00480258004402587D
:1030000000400058316665422DE9F84FD0F85C71F8
:103010000446534B00F59676FDB227F0FF0982680F
:1030200000F1E00A103D4846D2F80080A3FB0535C8
:103030002D09294650F048FAD4F81C210023B2F596
:10304000807F84F820317FD00DD8102A00F0848052
:103050005DD8012A46D0042A16BF6FF400616FF0D4
:1030600008013C230EE0B2F5805F71D0B2F5803FDD
:103070003BD0B2F5806F15BF6FF400616FF00801AF
:103080003C230423324608F11806404656F803C094
:1030900001EA0C01F150D4F81CB159464FF0C2FEC0
:1030A000BBF5807F2ED024D8BBF1100F3FD037D88E
:1030B000BBF1010F02D0BBF1040F34D14FF0080C6B
:1030C000336852462946484643EA0C03336040239E
:1030D000C4F8E83050F09CF93B6843F010033B60C3
:1030E000BDE8F88F6FF00801CCE76FF008013C23D2
:1030F000C8E7BBF5805F22D0BBF5803F1AD0BBF597
:10310000806F10D108F11C064FF0080CD8E7402A58
:1031100015BF6FF400616FF008013C230023B1E795
:10312000BBF1400FCAD03C364FF4006CC8E74FF4F7
:10313000006CC5E708F154064FF0080CC0E708F131
:103140001C064FF4006CBBE76FF00801042399E7FD
:103150006FF40061042395E76FF4006192E700BF0C
:10316000ABAAAAAA2DE9F8432422D0F85051002393
:103170008168C0F8D02104462A6800F5A87622F0BC
:1031800001022A602B606B60AB604279C0F8D831D5
:1031900080F8CC31C0F8D031C0F86831C0F8D431F3
:1031A000C0F870319302C0F8541103F48053BC4945
:1031B000C0F8583113038D4203F40053C0F85C315A
:1031C0004FEA022303F48063C0F8603100F0AB8162
:1031D0002379D80703F0020100F14081002940F073
:1031E0007181C4F8641194F8F0314BB1D4F878319E
:1031F00043F00803C4F878314FF40043C4F8883131
:1032000012F00802D4F8D03100F06E81002B00F0EB
:10321000AD8124233046C4F8D0312B6823F001035C
:103220002B6047F007FD012817D0D4F87831002B28
:1032300040F09F816B68304623F490436B60AB682D
:1032400023F02203AB60AB6843F00803AB602B684C
:1032500043F001032B6050F0F9F994F8048018F062
:10326000010F6FD0D4F82C71002F00F06C81002377
:103270004FF4807C04F13C09E7632366E36648462B
:10328000C4E91133C4E91433C4E91933D4F834312F
:10329000C4F8B8304FF48063E3644FF48033C4E97A
:1032A00016C351F0DFFB484645F0CEFFD4F8D431C9
:1032B000C4F8C891202B666741D1E368626998B26F
:1032C000EAB3B0FA80F14909C8B394F8CCC1BCF1B3
:1032D000010F34D04FF0220CC4F8D811A4F8AC017F
:1032E0000120C4F8D4C1DFF8D0C1C4F8A821C4F8C3
:1032F00078C0DFF8C8C1C4F88C10C4F87CC0DFF80F
:10330000C0C184F8CC01C4F888C094F870C084456A
:103310000CD084F8700094F87100012800F031811D
:103320004FF4006384F87010C4F890301023C4F890
:10333000D831002384F8CC312023C4F8D0317B6805
:10334000C4F8443118F0020F00F08680D4F83051F0
:10335000002D00F0EC80D4F83821002304F1B407EC
:10336000C4F8C0303846C4F8C830C4E92D524022F1
:10337000C4F8BC204FF48062C4F8C4204FF48032FB
:10338000C4E93333C4E93633C4E93833C4F8D4204C
:1033900051F068FB384645F057FF002840F0A38005
:1033A000404B4149414A8D4218BF9D42404801F17E
:1033B0006001C4F8C4710CBF01230023C4F8EC60A1
:1033C000954208BF43F001033032854208BF43F005
:1033D00001036030954208BF43F0010330328D4253
:1033E00008BF43F0010301F56871954208BF43F03F
:1033F000010302F55C72854208BF43F0010300F54A
:103400006870954208BF43F0010330328D4208BF17
:1034100043F001036031954208BF43F001033032AD
:10342000854208BF43F00103954208BF43F0010302
:1034300030328D4208BF43F00103954208BF43F08C
:1034400001033BB91B4BEB1AB3FA83F35B09002B67
:1034500000F0AF8000236B60BDE8F8830423C4F85C
:10346000643171B10C23C4F86431D3077FF5BBAE6E
:10347000D4F878314FF4803143F00203C4F880115E
:1034800028E0D3077FF5AFAED4F8783143F00203DC
:10349000C4F878314FF48033C4F88031A3E600BF1C
:1034A000000C00581000024028000240400002407A
:1034B00058000240B8040240815F0808B55F080860
:1034C000B95F08080823D107C4F864317FF58BAED3
:1034D000D4F8783143F00103C4F878314FF4003365
:1034E000C4F87C317FE6FEE70BB194F8CC212423AD
:1034F00084F8CC213046C4F8D0312B6823F0010386
:103500002B6047F097FB01283FF4A7AED4F8783141
:10351000002B32D16B68304623F490436B60AB686C
:1035200023F02A0392E60423C0F8743150E6D4F85D
:10353000DC311A6842F080021A601A6842F04002D8
:103540001A60BDE8F883D4F8DC311A6842F480725E
:103550001A609A6842F001029A601A6842F02002EA
:103560001A601A6842F010021A60EBE684F8CC3157
:103570004FE6304647F05CFD5CE6304647F058FDCC
:10358000C8E79BB2484605F1240145F0FDFF00283D
:103590007FF4CCAE84F8CC012B6843F480732B60AD
:1035A000AB6843F00103AB60AB6843F04003AB6032
:1035B000C5E66B6050E700BF38B50409013C082C34
:1035C00018D80E4D00F00F0335F8140040FA03F23E
:1035D00012F0010210D00122254402FA03F3013B4C
:1035E000184056F0D9FB95F8643C054A034402EBB9
:1035F000C30038BD002038BD104638BD28A10908D9
:10360000C41B00242DE9F047984D05EB0013D3F8B7
:10361000F04B002C00F08F80B3F8FA7B06464FEA9F
:10362000001938464DF0D2FE01227B0907F01F0732
:10363000023BBA40082B0FD8DFE813F0BF00C700E9
:10364000CF00D700DF000900E700EF00B70088498E
:10365000CB6F23EA0203CB6705EB0903013693F82E
:10366000F40BF6B2FFF7A8FF074610B11223C6719C
:10367000837105EB090393F8F50BFFF79DFF824675
:1036800010B11323C671837105EB090393F8F60B90
:10369000FFF792FF804610B11423C67183714D4429
:1036A00050462E2195F8F82BFFF77CF995F8F92B69
:1036B00040460E21FFF776F995F8F72B2E21384674
:1036C000FFF770F923686B4A23F0010394422360EB
:1036D00033D0694B9C423ED1654BD3F8902042F4E5
:1036E0008042C3F89020D3F8902022F48042C3F89F
:1036F0009020E36843F00043E360A36823F4F07391
:10370000A3602368DA0716D4A1685C4A5C4B0A40C0
:103710001343A360E368DB0042D5E268594B1340D2
:1037200043F0E863E360236823F400632360236DC0
:1037300023F001032365BDE8F0874D4BD3F89820B3
:1037400042F48052C3F89820D3F8982022F4805293
:10375000C3F89820CDE74C4B9C4213D04B4B9C4276
:1037600063D04B4B9C426ED1414BD3F8982042F42E
:103770008012C3F89820D3F8982022F48012C3F85E
:103780009820B6E73A4BD3F8902042F40042C3F8B1
:103790009020D3F8902022F40042C3F89020A8E7AC
:1037A000236843F480532360B7E73149D1F89C3054
:1037B00023EA0203C1F89C304EE72D49D1F8983036
:1037C00023EA0203C1F8983046E72949D1F890303E
:1037D00023EA0203C1F890303EE72549D1F894303E
:1037E00023EA0203C1F8943036E72149D1F880304A
:1037F00023EA0203C1F880302EE71D49D1F8843056
:1038000023EA0203C1F8843026E71949D1F88C3045
:1038100023EA0203C1F88C301EE71549D1F888303D
:1038200023EA0203C1F8883016E7114BD3F8982039
:1038300042F40052C3F89820D3F8982022F40052A2
:10384000C3F8982055E7134B9C427FF452AF03F521
:103850000C33D3F89C2042F02002C3F89C20D3F80C
:103860009C2022F02002C3F89C2042E7601B002429
:10387000004402580030014000380040E0FFBF8F94
:1038800007000020FFFF39D8003C00400034014011
:10389000005001400014005808B51D20FFF78CFEB1
:1038A00010B190F9063053B11E20FFF785FE10B11C
:1038B00090F9063003B108BD5523C38008BD5523D8
:1038C000C380F1E7F8B50E4C94F8F875A7B104F58C
:1038D000C064C7F109070925013D0FD0A6683079FA
:1038E000FFF76AFE94F8DC10F27908B1FFF736F8BA
:1038F000AF4204F5B474EFD10120F8BDAB68FFDE30
:103900000400002008B548F0A1FE1B20FFF754FE7C
:1039100008B12923C3801C20FFF74EFE08B12923DC
:10392000C38050F055FE0B484DF096FE0A4B93F8BD
:10393000552C012A01D0012008BD084AD3F8340FC4
:10394000C3F8302F50F052FC0023054A184682F885
:10395000233008BD20040024601B002458040024E8
:1039600000ED00E0F8B50446EFF31185502383F332
:103970001288D0F830311B6803F001031BB1EDB29F
:1039800085F31188F8BDD0F8D021D0F8D4110A43BE
:1039900002F02102212AF2D0D0E90912914250D03E
:1039A00090B24BD8194623691B1A9BB2A162002121
:1039B00084F8E011D4F8D0112029E0D1A169891848
:1039C000DDD0B3FA83F25209002BD8D094F8CC01A1
:1039D0000128D4D02120A4F8A6314FF0010CC4F85E
:1039E000D821C4F8D001D4F8C401D4F85061C4F887
:1039F000A011A4F8A43184F8CCC160B31B4F90F897
:103A000034E0C7631A4FE64502650764194FC7647F
:103A10000AD090F8357080F834C0674515D04FF45F
:103A2000006380F834204365102100222023C4F86D
:103A3000D81184F8CC21C4F8D031A0E7081A83B299
:103A4000B4E7012380F8E03199E706F1280245F058
:103A50009BFD0028E8D100234022326284F8CC315B
:103A6000B36843F08003B36089E700BF595F08087B
:103A70007D5F0808B95F0808BFF34F8F0549064B03
:103A8000CA6802F4E0621343CB60BFF34F8F00BFFC
:103A9000FDE700BF00ED00E00400FA05002103206F
:103AA00008B5FFF76FFA72B6FFF7E6FF08B51D48D5
:103AB0000023C0F88430BFF34F8F436923F4803371
:103AC0004361BFF34F8FD0F8803043F6E074C3F307
:103AD0004E3CC3F3C90E4FEA4C1C0CEA040173467A
:103AE00041EA8372013BC0F874225A1CF8D1ACF150
:103AF000200C1CF1200FF0D1BFF34F8FBFF36F8F5D
:103B0000BFF34F8FBFF36F8F4369002223F400335D
:103B10004361C0F85022BFF34F8FBFF36F8F72B66F
:103B2000FFF7AAFF00ED00E003689B0AA3F58013EE
:103B3000522B00D970470F4A13441B7D0D2BF9D827
:103B40004FF04C0C10B40C4C42790CFB0340022398
:103B5000D0F8380FDA409340C26829B922EA03034B
:103B60005DF8044BC360704713435DF8044BC360BA
:103B7000704700BF28A10908601B002403689B0A46
:103B8000A3F58013522B11D8094A13441A7D0D2A2C
:103B90000CD84079022307494FF04C0CD8400CFB5D
:103BA00002128340D2F8382FDB431361704700BF05
:103BB00028A10908601B002401490248FDF700B94B
:103BC000442000240000014001490248FDF7F8B8F4
:103BD000442000240000014002494FF08040FDF7DE
:103BE000EFB800BF7020002401490248FDF7E8B893
:103BF0009C2000240004004001490248FDF7E0B881
:103C0000C82000240008004001490248FDF7D8B848
:103C1000F4200024000C0040F8B5164D164E2A6919
:103C2000EB681A404FF00040B2FA82F3EAB120FA92
:103C300003F3012A6FEA030302EA03012B610A4638
:103C4000F2D1D6F8E8758FB1013F0023BFB2C6F8B4
:103C5000E835D6F8E44534B123682046394698471C
:103C60006468002CF8D10022DCE7F8BDEF6ABFB22F
:103C7000EFE700BF00100040601B0024014902482C
:103C8000FDF79EB8782100240004014010B5064CD1
:103C9000064804F5C361FDF793F804F5CE610448C6
:103CA000BDE81040FDF78CB8601B00240004014003
:103CB000001C004001490248FDF782B8A4210024FD
:103CC0000018004001490248FDF77AB8FC210024A1
:103CD0000020004001490248FDF772B82822002464
:103CE0000040014001490248FDF76AB8542200240F
:103CF0000044014001490248FDF762B880220024D7
:103D000000480140800AA0F5801052280ED8084BC8
:103D100003441A7D0D2A09D8064B4C2101FB0233BE
:103D2000D3F8382F136843F001031360704700BFC6
:103D300028A10908601B00241F4B984210B50ED023
:103D400003F5806398420AD01C4A03F580439842E9
:103D500018BF904203D003F5806398421BD146F010
:103D6000D5FB174B1749DC69DA69C4F3022CC2F39F
:103D7000022201EB0C0393F8543C03F01F03D840DC
:103D80000F4B11491B69C3F3C03342EAC303CB5C39
:103D900003FB00F010BD46F0B9FB094B0949DC6993
:103DA000DA69C4F30214C2F302120B1993F8543CFB
:103DB00003F01F03D840E3E700000140004001404A
:103DC0000044025828A10908B0230A082DE9F04F41
:103DD000002391B0AE4C0093AE4BAF4FA3F54966B4
:103DE000AC4D4FF00009AD4BD5F800A093F8C622BA
:103DF0004FEA9A23A3F58013522B00F2D08033446C
:103E00001B7D0D2B00F2CB80012A17F903B000F0C7
:103E10001181022A02D1BBF1080F3CD14FF00008FA
:103E20004146584612F098FA12F01EFB90F900C075
:103E3000BCF1000F18BFBCF1540F14BF4FF0010CC0
:103E40004FF0000C40F0EA8008F104081FFA88F8EF
:103E5000B8F1100FE4D1009B002B00F0AB808C4A2E
:103E60000BE033441B7D0D2B0ED8FB565B450ED06B
:103E700002F58672944200F0998091680B689B0A63
:103E8000A3F58013522BECD900235B45F0D14B797D
:103E900069799942ECD109F101091C35B9F1080F92
:103EA000A1D1009B04F586740133042B009397D1B4
:103EB0007B4A4FF0010B92F8F83502F58769013320
:103EC0000393039B5B4567D0744B99F81020D9F896
:103ED0000C6093F8DA320092002E5DD0704AD6F86A
:103EE00000A055686F48B288002D504401924FEAF7
:103EF000902040F3AE80664A002405E0013402F5CC
:103F00008672AC4200F0A28011688142F6D1604B0B
:103F10004FF48672019D02FB0434009B0322C9F812
:103F20000C6089F81030019BC9F81840B3FA83F788
:103F3000C7F11F035800C9F80430B27186F807B002
:103F400002FA00F6A16C0122D4F854C0314302FAFF
:103F500000F002FA03F3A164216D0143D4F8AC0030
:103F600021654F490E7899B2002E00F04E8143EA48
:103F70000C036365CAF81850FCF794F80BF1010BB9
:103F80002046FCF763F809F1200940F20113BBF168
:103F9000090F29F8043C94D111B0BDE8F08F013A23
:103FA000012A7FF678AF4FF0000B37E7BCF1000F26
:103FB0007FF471AFA86800223B4904E001320C3164
:103FC000102A00F088834B689842F7D152B2697981
:103FD0005046FEF7F5F8354A406800235168013332
:103FE000884208D0102B02F124023FF454AF5168EC
:103FF00001338842F6D1DBB22D4A013B03EBC30308
:1040000002EB830393F9FC31002B7FF444AFC9EB3F
:10401000C909204B03EB8903A36042E7009B002BF7
:104020007FF41DAF09F101091C35B9F1080F7FF4C8
:10403000DAAE36E7BBF1010F3FF4F0AE09F101094A
:104040001C35B9F1080F7FF4CEAE2AE7042C00F03E
:1040500049824FF48671124A01FB052211690491CD
:10406000002900F00483906001304FF054019C4619
:10407000C4B20D4882F8101182F811416A1C084937
:104080004A60049A1168976802915179002216E0FB
:104090000C000020B8AD0908C4230A08582C0024DD
:1040A000040000200000FEA720010024E0010024FD
:1040B0000000002401320C30102A00F00C83436809
:1040C0009F42F7D152B20298CDF814C0FEF778F8AB
:1040D000944B4FF48672DFF87C8202FB053100229C
:1040E000059B0132D0E90170C1E90770414648687B
:1040F000874208D0102A01F124013FF44DAF4868EF
:1041000001328742F6D1D2B28749013A02EBC202AC
:1041100001EB820292F9FC1100297FF43DAF4FF4CC
:10412000867182F8FD410693542401FB05F37F4814
:1041300082F8FC419A107E49059300FB02F201F5DA
:1041400060747848C2EBC20C02EBC202184401EB67
:104150004C1104EB4212C0F80CA0C0F8B410C0F827
:10416000FC203322C0F8B8208C22C0F80021714A0C
:104170000298D418FFF7E0FD069B062B00F0B981EA
:10418000072B6D496D4B6E4A18BF1A466D4B18BF11
:104190000B464FF48671DDF808A0B0FBF3F3B0FBDB
:1041A000F2F2013B5F48013A01FB05019BB2A1F825
:1041B000BC20A1F874302366059B03F1580100F17F
:1041C0000803504619440023A4F858306366E36599
:1041D0004EF0A6FFDAF8003043F08003CAF8003052
:1041E000049B5B791A4606930C2A1CD8DFE812F070
:1041F00003021B001B001B00DD011B001B001B003A
:10420000BB011B001B001B009601C7F12F072D04EB
:1042100002FA07F3324643EA0C036365CAF8185002
:10422000FBF740FFAAE63F4A4FF4867302984FF02F
:10423000000A03FB05230222CDF828A05969036870
:10424000079123F00103CDF834A0CDF83CA0036022
:10425000602308934FF480730E93012309930A237C
:10426000CDE90B3208AA4EF0DDFD0799B1F5807F4C
:1042700000F0288240F24081B1F5805F00F00E82AC
:10428000B1F5803F00F00482B1F5806F15BF4FF4A7
:10429000006308234FF03C0A4FF0040A029A1832D8
:1042A00052F80A100B4342F80A30049B1879002890
:1042B00040F0CB81029A136843F00103136000239E
:1042C000D8F804200133974200F0BC81102B08F18C
:1042D0002408F5D14FF0FF330027134A03EBC30343
:1042E00002EB8303D3F8E001174B984214BFA120DF
:1042F000A0204DF06BF8069A0C2A00F2A081134B17
:1043000003EB4203B3F870CD4FF48673054A1048AF
:1043100003FB0523DDF808E000F23471A3F818C0B0
:10432000002320E004000020000000246B4CA407C0
:10433000E02801240C000020D0DD06004495080090
:104340001055220040771B000000024028A10908F8
:10435000FC100020E0010024964500F09D8101330F
:10436000042B00F0BB8151F83320002AF4D1D0F89F
:1043700054270132C0F8542700EBC300029ADB0037
:10438000C0F8342719443846234690228F884CEAD7
:10439000070C0027A1F804C0C349FDF785FF4FF4BF
:1043A0008673C24A40214FF4403CC14803FB052AB2
:1043B0004FF48052DAF81C502B6843F010032B6046
:1043C0002B6843F014032B60C4E91F77C4E92777F7
:1043D000C4E92977DAF82030A167E9B2C4F894304B
:1043E000069310394FF48063C4F898C0A0FB010114
:1043F0004FF4804CC4F88430DAF8B8000909059B02
:10440000C4F8900025F0FF00DAF80C80C4F888208A
:1044100008F118020491029008F11008226703F1D4
:104420007002A44B1A44DAF8B430C4F88CC0636745
:104430004EF0EEFFD5F800C0059BC4F820C0D5F8BB
:1044400014C003F1B8029B4BC4F824C0D5F804C0D3
:104450001A44069BC4F828C0D5F808C00499C4F8CB
:104460002CC0D5F80CC0C4F8DC304FF48063C4F81D
:10447000C870C4F8CC304FF40033C4F830C0C4F86E
:10448000E0300298C4E93077C4E93977C4E93B7772
:104490004FF40067DAF80031C4F8B880C4F8D0707F
:1044A0004FF48047C4F8D830DAF8FC30C4F8D47040
:1044B000C4F8BC304EF0ACFF2B68D6F800A06363A4
:1044C0006B69A3636B68E363AB682364EB68636445
:1044D0002B6843F010032B602B6843F014032B6010
:1044E000B5881AE50323744A82F8DB3211B0BDE8BF
:1044F000F08F724A724B4CE6102900F0E98000F20E
:10450000BD80012900F0E280042915BF4FF400634B
:1045100008234FF03C0A4FF0000ABFE602984FF420
:10452000867262494FF0020A036802FB05124FF4DB
:10453000805123F00103516108AA036000230A930C
:104540000D930F93602308934FF480730E93012310
:1045500009930A23CDE90B3A4EF064FC4FF0040AAC
:104560004FF400639AE602984FF486724F494FF079
:10457000020C03684FF0040A02FB05124FF480712D
:1045800023F0010351616022036000230E910A931E
:104590000D930F930123CDE908230A2308AACDE93F
:1045A0000B3C4EF03FFC082378E602984FF48672ED
:1045B0003E494FF0000A03684FF0020E02FB05125D
:1045C000102123F00103CDF828A0516108AA03604F
:1045D0006023CDF834A008934FF48073CDF83CA04D
:1045E0000E93012309930A23CDE90B3E4EF01AFCEA
:1045F0004FF4006352E602984FF486722B494FF055
:10460000000A03684FF0020E02FB0512012123F09D
:104610000103CDF828A0516108AA03606023099125
:1046200008934FF48073CDF834A00E930A23CDF88D
:104630003CA0CDE90B3E4EF0F5FB08232EE64FF0F3
:10464000000C61E6DFB27B1E47E6FEF7B5FF82464F
:1046500038B1049B0221DA79FEF780F95423AAF8D5
:104660000630029A536C43F40043536422E602235B
:10467000114A82F8DB3211B0BDE8F08F402915BF36
:104680004FF4006308234FF03C0A4FF0000A05E6A0
:1046900008234FF03C0A01E6DB0073E64FF40063A9
:1046A0004FF0040AFAE500BF0100000004000020FA
:1046B000ABAAAAAA0C000020582C0024882A1100BA
:1046C000A0BB0D0008234FF0040AE7E50823E5E549
:1046D0004FF40063E2E500235B68FFDE00239B8864
:1046E000FFDE00BF2DE9F04FB04D8FB095F8DC82B2
:1046F000B8F1000F03D100200FB0BDE8F08F002209
:104700002F21404611F006FF06460028F3D090F80E
:104710000590A74FD0F800A0A7F85C98FDF77CFDA6
:104720000028E8D0D0E901430193002CE3D0DFF862
:10473000B8B20022594601E0102ADCD04B680132A1
:1047400024319C42F8D1D2B29A4B013A02EBC20218
:1047500003EB820292F9FC31002BCCD12F21504681
:104760000293A2F8FC11C7F810A8FFF7E5FA924AE5
:10477000029B904280F0FA801A4601230393504630
:104780000292FFF7D9FA029A039BC7F814288B49C3
:10479000B0FBF3F2120A8A48A1FB02210022C7F8FB
:1047A0002028C7F818280A090909A0FB0202C7F83F
:1047B0001C185208A5F8E0225200A5F8DE2297F84E
:1047C0004D2802F0FF01002A00F0DE800222504650
:1047D0007C4987F84D2846F06FF90122404687F85A
:1047E000582887F84E2887F84F2887F8502887F8E8
:1047F000512887F8522887F8532887F8542887F8D3
:10480000552887F8562887F8572887F84D28FEF747
:10481000D3FEC5F8E40228B12F21C1804E21F279E0
:10482000FEF79CF8684A0021019B4FF4806CC5F8A4
:10483000F412B9F10C0FC5F80413C5F80C13C5E94F
:10484000BA43C5E9C511D2F8D80040F00100C2F85A
:10485000D800D2F8D80000F0010004900498D2F8F3
:10486000D80040F00200C2F8D800D2F8D82002F0F8
:1048700002020592059A4FF04002C5F8F0224FF46B
:104880008052C5E9BEC24FF48042C5F800234FF400
:104890000032C5F808234FF00302C5F8102376D87C
:1048A0004A4A02EB4902B2F88C8DC246484A08F1E6
:1048B00008084849C5F8202307EB8802C2F81018F9
:1048C000594600224B68013224319C4262D0102AA2
:1048D000F8D14FF0FF32374B02EBC20203EB8202FA
:1048E000D2F8E0013C4A904214BFA120A0204CF035
:1048F0006DFD0022DBF8043001320BF1240B9C42E9
:104900004BD0102AF6D1002007EB880753466022CF
:104910003249FDF7C9FCD7F8100844F095FC00288F
:104920007FF4E9AEB479002760260C9063004A4614
:1049300006A9274803F002030893E300CDE90667C0
:1049400003F00803002600270993CDE90A674BF01E
:104950004FFC00287FF4CFAEA30749461C481ED564
:1049600046F01EF9B0FA80F04009C5E65046FFF760
:10497000E3F91B4A1B490244A1FB0212920D531E8C
:104980009AB2531C0393FAE687F84C181EE78A463E
:1049900088468BE7D2B2013A9DE7D0B2B4E745F042
:1049A000FFFFB0FA80F04009A6E600BF582C0024B3
:1049B000601B002400000024006CDC02598B4F01B6
:1049C000ABAAAAAA742300240044025828A109080B
:1049D00070230024402F002400000240D502000074
:1049E00000366E01819F5E16E0010024830AA3F564
:1049F0008013522B00D970472DE9F0410F4C23440E
:104A00001E7D0D2E18D80E4C4FF04C08013915465E
:104A100008FB064789B2C7F8441FFFF78DF907F670
:104A20003C71B0FBF5F2013AD7F8380FC7F83C2FCC
:104A3000BDE8F04146F040B8BDE8F08128A1090882
:104A4000601B0024830AA3F58013522B70D82DE934
:104A5000F043734D85B02B441E7D0D2E65D84C233D
:104A6000704F9046044603FB06F907EB0905D5F89D
:104A7000382F824259D00139C5F8380F89B2C5F8AC
:104A8000441FFFF759F909F1080307F638710022AE
:104A90000B44C5F8402FB0FBF8F00138C5F83C0FC7
:104AA000C3E9022295F8753F03F0FF02002B40D0C6
:104AB0004C25022305FB061105FB06750431D5F8CC
:104AC000388F85F8753F404645F0F6FF012385F89D
:104AD000803F85F8763F85F8773F85F8783F85F801
:104AE000793F85F87A3F85F87B3F85F87C3F85F8EC
:104AF0007D3F85F87E3F85F87F3F85F8753F4A4BBF
:104B00009C4219D0B4F1804F16D0A3F57C439C424F
:104B100012D003F580639C420ED003F580639C4263
:104B200060D003F578439C425CD005B0BDE8F083CB
:104B3000704785F8742FBBE74C2303FB067393F88B
:104B4000742F012AF1D0022283F8752F374AD8F842
:104B500008100A40C8F80820012283F8752F0022A7
:104B600083F8742F00224C232F4903FB0673039212
:104B70008845CDE901224FF0020283F8752FD8F85D
:104B80000420D8F8083028D001F58061884524D069
:104B900022F07002C8F80420254A90450DD0B8F1E3
:104BA000804F0AD0234902F50062904518BF88451E
:104BB00003D002F54062904503D123F08003C8F88A
:104BC00008304C230121002203FB067383F8751F74
:104BD00083F8742F05B0BDE8F08317491140C8F879
:104BE0000410EAE74C2303FB067393F8742F012AA1
:104BF0009BD0022283F8752F0C4AD8F808100A407F
:104C0000C8F80820012283F8752F002283F8742F3A
:104C10000A4B9C42A6D003F578439C42A2D084E77D
:104C200028A10908601B0024000001408800CEFF75
:104C300000040040000800408FFF0FFF000C004000
:104C400037B590F867380446032B2FD10023204D49
:104C50008DF807309DF8073094F868289A4201D8FB
:104C600003B030BD9DF8073005EBC30393F8643300
:104C70008BB181F0010383B19DF8073005EBC303CD
:104C8000D3F86003FDF75EFE9DF807300133DBB219
:104C90008DF80730DEE70B46EDE79DF8073005EBB2
:104CA000C303D3F86003FDF753FEEDE7D0E910032B
:104CB0009B7903F00103994204D003B0BDE8304072
:104CC000FDF740BE03B0BDE83040FDF741BE00BF78
:104CD000582C002438B5044600790D4650B1FEF733
:104CE0006BFC08B10323C380E2792946BDE8384054
:104CF000FDF758BE38BD10B504462221FFF7EAFF84
:104D00002046FEF73BFF20460121BDE81040FEF79C
:104D10000BBF10B504460121FFF7DCFF0021204640
:104D2000BDE81040FEF700BF38B510F8133CA0F600
:104D30006C041BBB94F858388BBBD4E909239A4206
:104D40001CD05A1CA169A262CB5C21695B008A421B
:104D500028BF002243F40073A262A4F85C380A233F
:104D600084F85A38012384F8583894F86738012BAE
:104D700001D0042B02D1606CFFF7CBFF94F85438BC
:104D8000002B6DD194F855380133DBB2092B84F830
:104D9000553825D12046BDE83840FBF75BBA94F979
:104DA0005A586DB1B4F85C18013D20464B0801F02B
:104DB0000101A4F85C38FFF743FF84F85A58DDE797
:104DC000D4E9092384F858589A42D7D194F867381F
:104DD000012B01D0042BD1D1606CFFF78CFFCDE704
:104DE0000A2B3DD194F857382BB9B4F85E3843F00C
:104DF0000103A4F85E382379D9070AD5B4F85E0810
:104E0000820501D4C30718D4B4F864380133A4F878
:104E100064380122002384F8542894F8572884F831
:104E20005538012A1CD16179606C84F8573801F03B
:104E30000101BDE838404AF0DDBEE36AC0F3470037
:104E400013B1216B9847E4E7E3696269D054E369E1
:104E5000E2680133B3FBF2F102FB1133E361D8E7FF
:104E600038BD00BF2DE9F043BFB0BFF35F8FA24A4A
:104E70000020516A0346044621F480315162014604
:104E8000C2F89400C2F898300133C2F89C10112B7C
:104E9000C2F8A010F6D10523C2F89430536A43F447
:104EA00080335362BFF34F8FBFF36F8F9348944AA1
:104EB0009449121A54F062FD9348944A9449121A84
:104EC00054F05CFD934BDA6D042A00F0FB8005D8AA
:104ED000012A00F07283022A00F08583864A0023AB
:104EE0008D4C0120D2F888108C4E41F470018C4D0D
:104EF000C2F8881020602361216841F080012160A0
:104F0000216801432160216841F4803121602168DA
:104F100041F480512160A361E3612362A362E362F3
:104F200023636363A363E36323646364216821F4FD
:104F3000802121607B492366C1F808014FF00061A0
:104F40004FF6FF00784B9160D16801400B43D3606E
:104F500045F0BAFAA36902460F20C3F30323A169FF
:104F6000334493F8543C03F01F0322FA03F3C5F8CB
:104F7000A03443F0E7FD6D4AD36813F0040FD36803
:104F800040F0A2806A4B0021684A0591D96A21F05D
:104F90000101D962DB6A03F001030593936943F4CD
:104FA00040439361936903F440430593059B9369E0
:104FB0009B04FCD54C2200210EA85E4C54F03CFD15
:104FC0005D4A42F203031268B3EB124F4FF0000345
:104FD0000893A4F1140308BF1C46E268002A4DD0D0
:104FE000534B5249D86A20F00100D862DB6A03F0C3
:104FF000010308938B6923F4404313438B618B694E
:1050000003F440430893089B484A93699F04FCD5E6
:10501000414B4FF4403749480321D3F8E02042F098
:105020008002C3F8E0200122D3F8E03003F08003CF
:105030000793079B87610D9B0091019300234FF01D
:105040007BF9022322690EA8CDE91733A3781E92BB
:1050500001221993A3881A93A3791B93E3791C93D4
:10506000237A1D9300231F934FF48033CDE90E2341
:1050700044F072FF03283BD098B1FEE72B4A2C4B3B
:10508000916941F440419161926902F44042089271
:10509000DA6A42F00102DA62DB6A03F00103089384
:1050A000B1E7274B1A6812F00E0F4DD11A6822F0A3
:1050B0000F0242F002021A601B6803F00F03022B7A
:1050C00042D0FEE7DC6509E723F007031D4C43F0FF
:1050D0000203D360D4F8541A06E0D4F8543A5B1AA9
:1050E000B3F57A7F3FF64EAF53689804F5D549E79C
:1050F00072B6FEF7C1FC00BF00ED00E0000000004A
:10510000F849000090B50A080000002004000020C3
:10511000DB250B08004000580044025828A109086C
:1051200000000024008000510003FA0500480258E6
:10513000000400588C0400240010005C001C02587D
:1051400000200052601B00246E4A936903F0700334
:105150003F2B05D8936923F0700343F0400393611C
:10516000684AD36903F070033F2B05D8D36923F055
:10517000700343F04003D361624AD36903F4E063F0
:10518000B3F5806F05D2D36923F4E06343F4806301
:10519000D3615C4A136A03F070033F2B05D8136A8E
:1051A00023F0700343F040031362564B9A691007D3
:1051B00005D49A6922F00F0242F008029A61514A1E
:1051C000936923F470639361136899017FF579AF54
:1051D000136941F288304C4C23F0070343F003037A
:1051E0001361D4F8541A05E0D4F8543A5B1A834298
:1051F00000F29B81136903F03803182BF4D19369F3
:1052000003F00F03082B05D9936923F00F0343F034
:10521000080393613D4A136803F00F03022B0BD977
:10522000136823F00F0343F002031360136803F0C5
:105230000F03022B7FF445AF324A936903F07003EA
:10524000402B05D9936923F0700343F04003936129
:105250002C4AD36903F07003402B05D9D36923F09E
:10526000700343F04003D361264AD36903F4E0633B
:10527000B3F5806F05D9D36923F4E06343F4806309
:10528000D361204A136A03F07003402B00F245817A
:105290001C4F45F019F90346D5F8A404BA69B96959
:1052A000C2F30322164496F8542C02F01F02D34096
:1052B000C5F8A03443F046FC002840F07D8110235F
:1052C000159017900EA80E9344F046FE002840F06B
:1052D00023813B680E4A43F080033B60D7F8F430EB
:1052E00043F00203C7F8F430D7F8F43003F00203B8
:1052F0000493049B136A43F001031362054BD4F833
:10530000541A0CE000440258601B00240020005294
:105310000004005800E20400013B3FF4E9AED4F879
:10532000542A9142F8D0D4F8542AD4F8543A9B1A0B
:105330000A2BFAD9AF4C4FF480224FF440130EA839
:105340000E924FF000082F934EF0ACF9D4F8EC30E9
:1053500041F20302A849032643F002030EA8C4F851
:10536000EC30D4F8EC3003F002030393039BD4F841
:10537000943043F00203C4F89430D4F8943023F00E
:105380000203C4F894300B689C49B2EB134F9C4B5A
:105390009C4A28BF0A465A601A6822F47C5242F49A
:1053A00000521A601A6842F060021A600E96CDE947
:1053B0002B884EF077F94FF4E0430EA8CDF8E48047
:1053C0000E93CDE925884EF06DF918230EA8CDF87F
:1053D000B8800E93CDF8CC804EF064F94FF40023E2
:1053E0000EA80E934FF4003336934EF05BF9D4F8C9
:1053F000E0304FF48071844843F00103C4F8E0309A
:10540000D4F8E03003F0010309934346099A0222DD
:10541000CDE900684EF090FF23694FF400717B489E
:1054200023F0FE7343F088732361D4F8E03043F037
:105430000403C4F8E0304346D4F8E02002F004024C
:105440000692069A0222CDE900684EF075FF2369A4
:1054500023F07E4343F0FC43236145F035F86C4B69
:105460006C4A4146C5F8A0041846D21A54F0E4FA32
:1054700069486A4A6A49121A54F080FABFF35F8F8A
:10548000684D4646684C01276B6A23F480336B6293
:10549000C5F8948023E0002946D0D4F80090637AC0
:1054A000103414F8060C1B0643EA007343EA410368
:1054B00014F8051C43EA814314F8041C43EA4143F1
:1054C00014F8031CC5F89860013643EA0143C5F897
:1054D0009C90032E43F00103C5F8A03026D06368EA
:1054E000217A002BD7D0D4F800900029D7D129F009
:1054F0001F01A3EB0108B8F1200F38BF4FF02008BF
:10550000404654F079FA431E014607FA03F08045FD
:1055100008BF1946C9B2C2E7FEE7136A23F0700359
:1055200043F040031362B3E6FEE7CAE50523C5F87E
:1055300094306B6A43F480336B62BFF34F8FBFF3D9
:105540006F8FBFF34F8FBFF36F8F0022C5F85022CC
:10555000BFF34F8FBFF36F8F6B6943F400336B6101
:10556000BFF34F8FBFF36F8FC5F88420BFF34F8F0A
:10557000D5F8805043F6E0762A49C5F34E34C5F39A
:10558000C905640104EA06002B4640EA8372013B28
:10559000C1F86022F9D2203C14F1200FF2D1BFF300
:1055A0004F8F4B6943F480334B61BFF34F8FBFF391
:1055B0006F8F3FB0BDE8F08383E50E4A02201B49A0
:1055C000D865D2F8F4300343C2F8F430D2F8F4309E
:1055D00003400E930E9AD1F8003883F30888D1F86F
:1055E00004389847FEE704210320FDF7CBFC72B690
:1055F000FEF742FA004402580010005C7FBB220014
:10560000008400407FBB223000000258000802588E
:1056100020E6002400E7002460E3002420E60024C4
:10562000DF250B0800ED00E0A80400240090F01F27
:1056300030B4EFF31182102383F312880C4B4FF038
:10564000E0200C4C0025D3F8B817D2B20131C3F8D2
:10565000B8178169C4F8A013C4F8A453016982F390
:105660001188D3F8542A013230BCC3F8542A704749
:10567000601B0024582C0024254B5B68C3F30803EF
:1056800030B4FBB9EFF31183E3B9224C4FF0E02CB7
:10569000214BD3F8B827DCF81800D3F8B8178A42A2
:1056A000F7D1D4F8A0138842F3D8D3F860484FF468
:1056B0007A7101FB04F3181AB0FBF4F030BC01FB63
:1056C00002007047EFF31182102383F312884FF02A
:1056D000E023104C9D691969C90303D50121C4F861
:1056E000A4139D690C49D2B2D1F8B807D4F8A433F9
:1056F00082F311884FF47A72D1F86018034402FBE8
:1057000001F0401BB0FBF1F030BC02FB030070471E
:1057100000ED00E0582C0024601B00242DE9F84324
:105720001B4EFFF7A9FF7568002D1BDD07464FF0E4
:1057300000084FF4867900231C4609FB03620133FD
:1057400092F80521AB4244EA0204F6D1FFF794FF38
:10575000C01BB0F5FA6FCCBF002304F0010333B1D6
:105760009846E8E7FFF788FF0020BDE8F88344EAA1
:10577000080010F0FF00F8D0064B93F8A823542A35
:10578000F3D1B3F8B0230132A3F8B023BDE8F88316
:1057900004000020582C0024BE4803780BB90120D7
:1057A00070474368BC4A002B2DE9F04FD2F8B86728
:1057B00087B018DD00F108050024B849D5F8F430A9
:1057C000BFF34F8F03F59072C1F85C3220339342E0
:1057D000FAD1BFF34F8FBFF36F8F0134436805F5E4
:1057E00086759C42EADB90F8F8154FF00009AC4A48
:1057F0000491A2FB0612AB4BAB4D5209DFF8C0B2CD
:10580000A3FB0213DB0803EB8303A2EB4303DAB22F
:1058100005EB830A05F5387305920093049B9945BF
:1058200000F01681DBF81830DBF80470D3E93D4650
:10583000FFF722FFDFF88CC29C4901229CF8A88365
:1058400071180190B8F1540F9CF8BC0302FA07F2EA
:1058500004EB410104EB400301D1ACF8B2039942DF
:1058600040F26B811F88174200F060815F88174209
:1058700000F071819F88174200F06F81DF88083344
:105880001742ECD11C1B99424FEA640440F2558147
:10589000301B452828BF452003EB4000834280F0A1
:1058A000508100261F46B6463146CDE90298B3F82E
:1058B000008008EA020888451CD1B3F8028008EA93
:1058C0000208414540F01B81B3F8048008EA020851
:1058D000414540F01681B3F80690083309EA020901
:1058E000494508D1984209D9B3F8008008EA02086E
:1058F0008845E2D00233984200F2E680BEF1110FF3
:10590000DDE9029840F21D81DEF1150200F11981F6
:105910006749DCF8C003D1F8D8349C4238BFC1F8DD
:10592000D844019C231A002B14DB624B03449C4295
:1059300001D923460533CCF8C033D1F8D834052B30
:1059400040F20D81053BDBB28CF8BC334FF0FF33E6
:10595000C1F8D8343AB106FA02F2CEF1140E01269B
:1059600006FA0EF61643544BC6F3C43203EB82021A
:10597000D2F8A80D06F01F0203EB8202D2F8A81D90
:10598000C6F34412C6F3842603EB820241EA0031D7
:10599000D2F8A82D03EB860341EA0211D3F8A83D03
:1059A00041EA0321454B81EA1122D3F8403A82EAC9
:1059B0001212013302F00F020F2A40F0A480B1F559
:1059C000803F80F0A080B8F1540F4FEA111147D00A
:1059D0003A4AB1F5606FC2F8403A4DD0009B9981C8
:1059E00095F858300598834210D0DAF808202B68D3
:1059F0009B1A2B606B68DAF830209B1A6B600023CF
:105A0000CAF80830CAF8303085F858002B680133DE
:105A10002B60DAF808300133CAF808304FF6FF730C
:105A2000994207D16B6801336B60DAF8303001338B
:105A3000CAF83030009B09F101095C350AF15C0AB3
:105A40001433B9F1080F0BF1200B00937FF4E6AE8D
:105A500001231A4A012082F83C3B07B0BDE8F08FD1
:105A6000BCF8AC23B1F5606F02F10102ACF8AC23D5
:105A7000124AC2F8403AB1D1074A537803EB4303C4
:105A800002EBC3034B445B7C0D2BA7D18023009A10
:105A90009377A5E704000020601B002400ED00E0E0
:105AA0001F85EB51CDCCCCCC54180020C7FFFF7F15
:105AB0000000002420A1070028A10908FC100020F4
:105AC0003C040020582C0024A3EB0708254F33F892
:105AD000021C4FEA6808114008F1010887FB08978B
:105AE000A7EBE8774FF00108012FB8BF0127BE40B0
:105AF000BE44013F08FA07F73E431F46D7E604338A
:105B0000F9E60633F7E6B8F1540F04D1BCF8AC233C
:105B10000132ACF8AC23144A4FF6FF71C2F8403A98
:105B2000D2F83C3A0133C2F83C3A59E702331C1B25
:105B300099424FEA64043FF6ABAE10B101388CF8DD
:105B4000BC03B8F1540F7FF475AFBCF8AE3301332A
:105B5000ACF8AE336EE7043394E6063392E60023E6
:105B6000F2E600BF56555555FC100020264B70B587
:105B70001A785B789A4242D1244E7368002B22DD5A
:105B800006F108000025224CD0F8AC30BFF34F8F4F
:105B900003F1E002C4F8683220339342FAD1BFF334
:105BA0004F8FBFF36F8F337813B1037F012B20D05A
:105BB00042690135716800F586701368A94243F0A7
:105BC00001031360E0DCFFF757FD124BD3F8544795
:105BD000002C0DDD03F2347303EBC40419680833A1
:105BE00033F8042CC8689C4242EA0002CA60F5D12E
:105BF00070BD002380F8FC30FAF728FAD8E751F09E
:105C000007F80028B8D170BD601B002404000020F4
:105C100000ED00E0FC10002001302DE9F04F5FFAAC
:105C200080FA83B0544E4D1E544C4FF01008544F20
:105C3000D3464FF4FA7949F01FFD0195FFF71CFD9B
:105C40004FF0E0214FF47A7C4FF0010E7B68C3F3F4
:105C50000803002B72D1EFF31183002B6ED1D4F81F
:105C6000B8378A69D4F8B857AB42F8D1D6F8A05300
:105C7000AA42F4D8D4F860A80CFB0AF5AA1AB2FB21
:105C8000FAF20CFB03231B1AB3F57A7FDED3B9F1CA
:105C90000109D3D1019D4FF47A79584649F042FE6B
:105CA0000195FFF7E9FC4FF0E0214FF47A7C4FF0CB
:105CB000010E7B68C3F308031BBBEFF3118303BB27
:105CC000D4F8B8378A69D4F8B857AB42F8D1D6F8C7
:105CD000A053AA42F4D8D4F860A80CFB0AF5AA1A7B
:105CE000B2FBFAF20CFB03231B1AB3F57A7FE0D365
:105CF000B9F10109D5D1019D013D9AD203B0BDE8AA
:105D0000F08FEFF3118388F312888D690A69D2034B
:105D100002D5C6F8A4E38D69D4F8B827DBB2D6F86B
:105D2000A4A383F311885244D4F860A80CFB0AF3AF
:105D30005B1BB3FBFAF30CFB0233D5E7EFF31183E4
:105D400088F312888D690A69D20302D5C6F8A4E3E4
:105D50008D69D4F8B827DBB2D6F8A4A383F31188F1
:105D60005244D4F860A80CFB0AF35B1BB3FBFAF3B4
:105D70000CFB023387E700BF582C0024601B002473
:105D800000ED00E02DE9F04F484D85B02B781BB9B0
:105D9000012005B0BDE8F08F454BD3F8B847FFF7B9
:105DA0006BFC95F8F8350193002B00F0C881414B4E
:105DB00005F5C065404E0027A3FB042300955B0951
:105DC000A6FB03263D4AF60802F5EB6806EB8606BD
:105DD000A3EB4606D2F8483BC11A1346F2B203F6CB
:105DE000382A08EB860689460392B9F1000F05DBD5
:105DF000009BD3F824314B4500F388814FF4B473F2
:105E00002A4A03FB072393F82037002B00F0C080B9
:105E1000009D2B48D5F85C11AB681A68CBB221F015
:105E2000FF01103BA0FB030326481B09C35C0B4486
:105E3000A9895C68D368A4B223EA0103C4F11604FB
:105E4000D360072C40F2A4801C4A0121D5F864518C
:105E5000D2F8403A8B46AE4602970133C2F8403A38
:105E600000222868944614E0BCF1140F2CDC13F1D6
:105E7000080748BF03F117073B110CEB271C5F1EF7
:105E8000013102FA03F30BFA07F78C4247EA0302E7
:105E90001AD303468C425EF8040FA0EB0303E3D849
:105EA000CCF115034FF0150CE9E700BF040000200A
:105EB000601B00241F85EB51CDCCCCCCFC10002006
:105EC000ABAAAAAAD4230A08BCF1150F029F40F07E
:105ED00013819F48C2F38423C2F3441100EB830370
:105EE00000EB8101D3F8283ED1F8281E1B0243EABB
:105EF000011302F01F01C2F3C43200EB810100EB79
:105F00008202D1F8281ED2F8282E0B4343EA02332E
:105F100083EA132282EA121202F00F020F2A40F0E3
:105F2000EB80C3F30F134FF6FF72934200F0E4804F
:105F3000B3F5606F00F0EE80AAF80C3098F85820A6
:105F40000398824210D0B168D8F80020521AC8F8DD
:105F50000020D8F80420316B521AC8F8042000221F
:105F6000B260326388F85800D8F800200132C8F8CF
:105F70000020B2680132B2604FF6FF72934207D13F
:105F8000D8F804300133C8F80430336B013333637D
:105F9000009C013708F15C085C3620460AF1140ABF
:105FA000FDF732F804F5B4730093019BBB427FF414
:105FB0001CAF68490122002381F83C2BC1F8483B03
:105FC0006549D1F8083691F8D8261B6812F0020FFF
:105FD000D1F81C171A6A0CBF0A4342EA81021A62FE
:105FE000019B012B3FF4D4AE5B49D1F8703791F897
:105FF00040281B6812F0020FD1F884181A6A0CBFEF
:106000000A4342EA81021A62019B022B3FF4C0AEAE
:106010005149D1F8D83891F8A8291B6812F0020F1D
:10602000D1F8EC191A6A0CBF0A4342EA81021A62DB
:10603000019B032B3FF4ACAE4749D1F8403A91F8AD
:10604000102B1B6812F0020FD1F8541B1A6A0CBFF8
:106050000A4342EA81021A62019B042B3FF498AE84
:106060003D49D1F8A83B91F8782C1B6812F0020F3B
:10607000D1F8BC1C1A6A0CBF0A4342EA81021A62B8
:10608000019B052B3FF484AE3349D1F8103D91F8C4
:10609000E02D1B6812F0020FD1F8241E1A6A0CBF03
:1060A0000A4342EA81021A62019B062B3FF470AE5A
:1060B0002949D1F8783E91F8482F1B6812F0020F59
:1060C000D1F88C1F1A6A0CBF0A4342EA81021A6295
:1060D000019B082B7FF45CAE204A52F8203C92F8DA
:1060E000B0001B68D2F8F41080071A6A4CBF42EA6D
:1060F00081020A431A624BE6164AD2F83C3A01334F
:10610000C2F83C3AAFB14FF6FF7317E7002005B075
:10611000BDE8F08F12494A7802EB420201EBC2025D
:106120003A44527C0D2A7FF407AF80228AF81E2061
:1061300004E7294658220B4853F020FCE3E71946B0
:106140000122044BC3F8481B83F83C2B20E600BF18
:1061500028A10908FC1000200400002004100020E1
:10616000601B0024E01B002038B50546FFF784FAC9
:106170000446FFF781FA001BA842FAD338BD00BFDE
:106180002DE9F047294D00F1FF38294C1027294E01
:10619000FFF772FA4FF001094FF0E02C4FF47A7ECE
:1061A0007368C3F3080303BBEFF31183EBB9D4F8AF
:1061B000B837DCF81810D4F8B8279342F7D1D5F8DF
:1061C000A0239142F3D8D4F860A80EFB0AF2521A29
:1061D000B2FBFAF20EFB03231B1AB3F57A7FDFD36F
:1061E000B8F10108D4D2BDE8F087EFF3118387F34B
:1061F0001288DCF81810DCF81020D20303D5C5F89B
:10620000A493DCF81810D4F8B827DBB2D5F8A4A30F
:1062100083F311885244D4F860A80EFB0AF35B1A8A
:10622000B3FBFAF30EFB0233D6E700BF582C002471
:10623000601B002400ED00E0154C08B5D4F8C43311
:1062400094F8CA03ABB91420FFF79AFF00BFD4F843
:10625000C4335BB1196894F8CA239B8809690B4061
:1062600012B91BB1FDF71AFC002BFBD0FAF732FC78
:10627000ECE719689A880B69134020B1002BE2D132
:106280000B691340FAE7002BDDD00B691340FAE7E6
:10629000582C00242DE98848431C0A265A4DDFF863
:1062A00070815FFA83FB594C4FF4FA79B24649F09A
:1062B000E3F9FFF7E1F901264FF0E0214FF47A729C
:1062C0006368C3F30803002B7BD1EFF31183002B2A
:1062D00077D1D8F8B8C7D1F818E0D8F8B8379C45C6
:1062E000F7D1D5F8A0339E45F3D8D8F86038D8F860
:1062F000607802FB03F3A3EB0E03B3FBF7F302FB9F
:106300000C331B1AB3F57A7FDAD3B9F10109D0D176
:106310004FF47A79584649F005FBFFF7ADF90126AD
:106320004FF0E0214FF47A726368C3F3080333BB84
:10633000EFF311831BBBD8F8B8C7D1F818E0D8F831
:10634000B8379C45F7D1D5F8A0339E45F3D8D8F897
:106350006038D8F8607802FB03F3A3EB0E03B3FBBD
:10636000F7F302FB0C331B1AB3F57A7FDCD3B9F1D8
:106370000109D2D15646013E96D149F00DFDEFF309
:10638000118C102383F312888B691F460B69DB0382
:1063900003D5C5F8A4638B691F46D8F8B8E75FFA40
:1063A0008CFCD5F8A4338CF311887344D8F860E8DA
:1063B00002FB0EFCACEB070CBCFBFEFC02FB03C3B8
:1063C000D1E7EFF3118C102383F312888B691F46FA
:1063D0000B69DB0303D5C5F8A4638B691F46D8F8A6
:1063E000B8E75FFA8CFCD5F8A4338CF311887344BA
:1063F000D8F860E802FB0EFCACEB070CBCFBFEFC23
:1064000002FB03C37DE700BF582C002400ED00E031
:10641000601B00240246074B02209A4208D8013331
:106420005B0840009A4280B202D2FF28F8D9704738
:10643000704700BF7FF0FA02CB0700D5704710B558
:106440000446FAF757FE94F82830012B00D010BD0F
:10645000616A0248FFF7DEFF888010BD00E1F505A4
:106460002DE9F0470546086888B00C464FEA902CA5
:10647000BDF84080ACF5801C9DF844A0BCF1520FE3
:1064800058D819462E4B63441E7D0D2E52D806EB6C
:10649000C6032C4F06EB430307EB8307FEF7D2FA44
:1064A00094F80590A379BAF1000F01D083F00103AD
:1064B0005A004FF48071DB00384602F00202CDF83A
:1064C000088003F0080303924A4604936023019373
:1064D0004FF40073CDE90613002301A9059349F099
:1064E00087FEA379384649469F0726D444F058FAD8
:1064F0004C22154B02FB063393F8752F012A10D15D
:106500000221D3F8382F83F8751F104B91680B4088
:10651000062B06D0B3F5803F03D0136843F0010388
:1065200013602168637901F1340269600021D01899
:106530002860D15008B0BDE8F08744F031FBD7E7C0
:1065400028A10908982A0024601B002407000100E4
:1065500010B4284C94F8303763B3226D904234D095
:10656000012B27D0D4F82C21824236D0022B21D007
:10657000D4F80822904232D0032B1BD0D4F8E42266
:1065800090422ED0042B15D0D4F8C02390422AD0AC
:10659000052B0FD0D4F89C24904226D0062B09D08E
:1065A000D4F87825904222D0072B03D0D4F8542673
:1065B000824210D0DC22591C02FB034284F83017BF
:1065C000106518465DF8044B70470023DBB25DF898
:1065D000044B184670470723F8E70123F6E7022328
:1065E000F4E70323F2E70423F0E70523EEE70623AD
:1065F000ECE700BFFC1000200548D0F8843723B139
:10660000DB6A13B100F2847018470248704700BF7C
:10661000601B0024D0AF090870B5104C4FF0000C7F
:10662000234693F800E00633864512D00CF1010CA6
:10663000BCF1060FF5D10A4ED6F8F053052D07D060
:106640000CFB05430135C6F8F053187059809A8049
:1066500070BD062303FB0C43F7E700BF2430002482
:10666000582C002438B51D4CD4F8F4331B8843B99A
:106670001B4D002384F8FF3385F87C37C5F8783745
:1066800038BDD4F8F023002AF2DDD4F8F813012A3B
:10669000488806D00123124DA4F8FC0384F8FE3389
:1066A000E7E78A880132121A9A42F3D10C4D002290
:1066B000D5F8843705F28470C5F8B0271B69984770
:1066C000D5F884379B68002BD3D005F284709847A7
:1066D0000028CED149F068FBCBE700BF582C00243E
:1066E000601B00240748D0F880371BB1064B93F895
:1066F000FE330BB100207047D0F8843700F284706D
:106700005B681847601B0024582C0024184A10B4FA
:10671000184C92F87C3744602344174C036092F87D
:106720007C0794F8FF33834218D892F87C078342A1
:1067300007D300235DF8044B1A461846C1E900321E
:10674000704792F87C071A1E5DF8044BC0F1800375
:106750000CBF01200220C1E90032704792F87C474B
:10676000002201201B1B5DF8044BC1E90032704779
:10677000601B002440E60024582C0024104B114AD2
:1067800093F87C1792F8FF0393F87C27904293F8D4
:106790007C270FD8904204D3D3F8783700201844D0
:1067A000704793F87C27D3F87837C2F18002104401
:1067B00018447047801AD3F878371844704700BFE0
:1067C000601B0024582C002438B5194D194CD5F8FD
:1067D000F423937B012B08D0D4F8783703F2FF73AE
:1067E0006FF30A03C4F8783738BDD4F884375B6A8E
:1067F00063B104F284709847D4F884379B681BB166
:1068000004F28470984778B1D5F8F423D4F8783737
:106810005288013B514213440B4003F2FF736FF364
:106820000A03C4F8783738BD49F0BEFAECE700BF78
:10683000582C0024601B0024F0B51C4C85B01C4B68
:1068400094F87C271B4D0393134495F8FF1394F899
:106850007C270293914294F87C3716D899420CD247
:1068600094F87C670F46C6F18006D9B933460122F9
:106870003F2BCDE900670DD860B994F87C07401A2A
:10688000B0FA80F0400905B0F0BDCB1A0027012214
:106890001E46EDE76946002302A850F0EBFE95F88E
:1068A000FF13EAE773180222E2E700BF601B00242F
:1068B00040E60024582C00242DE9F047174684B008
:1068C00000293ED0441E294DDFF8AC904FF0000A5D
:1068D00004EB0108264E0DE096F87C3708469942F5
:1068E00096F87C371DD2C3F1800318443F281BD88B
:1068F000A04526D095F8FF0314F8013F411C4844F9
:10690000C9B280F820300B0685F8FF13E4D50020CB
:1069100096F87C3785F8FFA30146994296F87C37B4
:10692000E1D3C01A3F28E3D996F87C379942DFD0EB
:10693000104B5B78002BDBD00020FFF77DFFA045DC
:10694000D8D1694602A8FFF7E1FEDDE90032134421
:106950003F2B00D910B904B0BDE8F08702463B4692
:1069600002A850F087FE04B0BDE8F087582C002440
:10697000601B00240000002420E6002430B585B010
:10698000694602A8FFF7C2FE58B9094C04F28475A3
:10699000D4F8843728465B6898470028F8D005B0BB
:1069A00030BD0246012302A850F064FEEDE700BFAF
:1069B000601B002438B50023124C134DC5F88037F6
:1069C00048F044FBC4F8F803FFF716FED4F8F83398
:1069D000C4F8F403A3B19A885B88D21A436802FB17
:1069E0000333C5F88037FAF741F894F8FF230446DB
:1069F00095F87C379A4201D0FFF7C0FFC5F8784779
:106A000038BD00BF582C0024601B00242DE9F04144
:106A1000104E154682180446D6F880370F469A4223
:106A20000D4A88BF1D1A92F8FF2396F87C379A42C8
:106A300001D0FFF7A3FF002021462B463A46C6F8B7
:106A4000B007D6F88407846A0448A446BDE8F0413C
:106A5000604700BF601B0024582C0024E42200245F
:106A60008C461346014662461846CFE72DE9F04FA3
:106A700000218BB041F69462B84852F0DDFF04204B
:106A8000FCF77AFA01460520FCF776FA51EA000392
:106A900040F05781B24B03934C220021AF480124B0
:106AA00052F0CAFF00214C22AC4852F0C5FF039BB4
:106AB000AA4AD3F80C35AB4D164614711560D36154
:106AC000136253624AF002FDFFF774FF002108468B
:106AD0000EF0E4FAF9F7CAFFB0F1000840F39B8129
:106AE0000024A14DDFF8A4E206F14C092746A34695
:106AF00005F5806A9D4E0294CDF804E004E00BF5A4
:106B0000006BD84540F3AE80019AD2F8B837C2F88E
:106B1000BC37F9F7DFFF202251465846FFF776FFD2
:106B200012229349504653F077F80028E7D1BB452D
:106B300025D002998F4B01EB410203EB82034A1CE3
:106B40008D4918460293ABEB07030592049301F0BD
:106B50005DFB029B4946059A41F84C3B049BC9F8F2
:106B60000C700292C9E90433D9F81C30C9E9083322
:106B70000123C9F80830814BC9F828308946039BA6
:106B80005F461222D3F80C35C9F81C30A918335DC2
:106B9000013291F8001499420BD00024202AF5D13B
:106BA00020375146B845384653DBFFF72FFF002208
:106BB000ECE70134152CF1D1D019714F2022394660
:106BC000FFF724FF384600230A2209A9099701F09C
:106BD00051FC0746099800230A2209A901300990AF
:106BE00001F048FC0790002309980A2209A9013006
:106BF000099001F03FFC0690002309980A2209A998
:106C00000130099001F036FC059009A9099800238C
:106C10000A220130099001F02DFC0023049009980C
:106C20000A221946013001F025FC97B10599DDE9EA
:106C3000063243EA4212049B5B0143EAC123A7F2F6
:106C4000BC7143EA600342EA412243EA0243C9F8C5
:106C50001C30029B642B43D05F460BF5006BD8457C
:106C60003FF752AF029B642B1ED0BB451CD00C22B9
:106C7000404C5E1C404902FB0344ABEB0705324627
:106C8000204601F0C3FAD9F81C20C9F80040C9F821
:106C90000C700296C9E908220122C9F80820374A77
:106CA000C9E90455C9F82820029B002B03F1010112
:106CB00017DC4FEA4803B3F1805FC0F2AD80274B89
:106CC0009C6834B91A461B791BB11368002B40F03D
:106CD000D980002108460BB0BDE8F04F0EF0DEB9B8
:106CE00065214C261D48DFF8A8A04FF0010906FBDE
:106CF00001F432460021234F0519284652F09CFE2C
:106D000032460021284652F097FE1C4E134804F1EB
:106D1000100204F11803029940F804A0C5F8089085
:106D200002312F62AE6240F8028002440430C2F8A1
:106D30000480039AD2F80C25C25003445A606A6258
:106D4000B7E74FF47A72002351F064FA0E4B40F229
:106D5000B27240F26D14B0FBF3F31DE0C03E0024AC
:106D600000000024C0230A08582C002454230A08D9
:106D700030230A087830002444230A08616A040892
:106D8000583000240068214C80510100601B002411
:106D90006C230A085B1A013212F0030514BF214666
:106DA0004FF4B7718B42F5DA8649002D64D0039118
:106DB0000399D1F8DC148B42C0F29C80824D0124EF
:106DC0005B1A55F8041F01349942F9DD0133A2F230
:106DD000BC72039D43EA44133C2443EA42237B4AAA
:106DE000B0FBF2F102FB11024FF46160B2FBF0F173
:106DF00000FB11221C20C5F8E004B2FBF4F004FBF8
:106E00001022521042EA401242EAC12242EA0343EF
:106E1000C5F80C3540E621464C266D4BDFF8BC9199
:106E2000012706FB01F4324600214FF0020A1D192A
:106E3000284652F001FE32460021284652F0FCFD61
:106E4000634B039A04F1180143F80490C8F10063FE
:106E5000D2F80C0504F11002BB405D4C5D4E85F884
:106E600005A0AF602E62A35022445360231D5850EA
:106E700019444860686222E70C4603911D21C4F85A
:106E8000E01495E7524800220023214626468464F8
:106E9000C463C0E910230246D56C02F14C035DB314
:106EA00098684D1E9E64A842C2E92366DE630DD039
:106EB0004D1CA84210D113F8481C00293FF409AF1B
:106EC0001A6401461A4643F8083CE5E700293FF4F6
:106ED00000AF53F80C2C014600293FF4FAAE814272
:106EE0007FF4F7AE106CC56B0135C563186493640D
:106EF0001A46D1E7012469E7354A0226294613E0FC
:106F0000D36B16635B01C2E9041120D003F6FF7353
:106F100000EB133318465363C31A906352F84C7F47
:106F2000461C1D440134C7B11379701E002BE7D1F4
:106F3000136916637BB103F6FF7300EB13335769D4
:106F4000536337B107F6FF7700EB1730E4E73346BA
:106F5000E0E73046E0E73346F1E7DFF884E0013868
:106F60001D4B0EF5FC62CEF80C48CEF800583E24BE
:106F70003F25CEF8E4374023CEF8FC07C2E90245AE
:106F8000CEF8F037840F8300D0B140F2FF155B19C3
:106F900044F100045B0A43EAC45303F140040C4982
:106FA0002344CEF8F44703EBC000CEF8F837440290
:106FB000CEF8E007C30DC2E9091142E9024388E6B1
:106FC0000123EAE700000024DC04002480510100D2
:106FD000C03E00240068214C88230A087C230A084C
:106FE000601B00242DE9F043484F93B0484DFFF754
:106FF00039FB97F87C3795F8FF239A4201D0FFF7C9
:10700000BDFC0024D7F88067C7F87847002E6DD004
:10701000DFF800810AE097F87C3795F8FF239A4261
:1070200001D0FFF7ABFC2034A6421BD922464146D3
:10703000684601F0EBF8684650F08EFC01220146EC
:107040006846FFF739FCA3B2002BE4D1D7F8C0376C
:10705000002BE0D09A881B6859690A4218BF1204B5
:107060009A61D8E7FFF7B0FB97F87C3795F8FF23D4
:107070009A4201D0FFF782FC0023DFF898909846EF
:107080001C46C7F878372246494609A801F0BEF8E1
:1070900021220021684652F0CFFC2022694620467A
:1070A000FFF7B4FC2022054609A9684652F0B4FD5A
:1070B000A3B2203450B9202D08D15BB1A642E2D84A
:1070C000B8FA88F0400913B0BDE8F08308F1010870
:1070D000002BF3D1D7F8C037002BEFD01A689B886C
:1070E00051690B4218BF1B049361E7E7FFF76CFB84
:1070F00097F87C3795F8FF239A4201D0FFF73EFCC2
:1071000000230120C7F87837DDE700BF601B0024AB
:10711000582C002490230A080A4B93F810251AB91A
:10712000094A92F8D00870470849CA6D032AF7D176
:107130000020054A4FF0010C83F8100582F8D0C8F2
:10714000C865EEE700000024582C002400400058D9
:1071500008B503220E4BDA6572B60E4B53E90212E4
:1071600051EA020306D100231A4609490A664B6612
:10717000FCF79CFC084B4EF6602CD3F8B8370CFBA0
:1071800000F05B1842F10002C31842EBE072ECE73A
:107190000040005838350024601B002410B58C18BE
:1071A000A14215D001F1FF3E013C41F2210C1EF835
:1071B000012F082380EA022002B24000002A8CEA54
:1071C000420180B2B8BF88B2013BF5D17445EED11F
:1071D00010BD00BF704700BF2DE9F047002BDDF860
:1071E00020A0884607460CBF4FF020094FF0300919
:1071F0005646002A144616F8011B23DD11B3334608
:1072000001E0002C05DD13F8012B2546013C002A86
:10721000F7D1023D3CB149463846C047013DFAD25C
:107220009AF8001059B13846C047334616F8011B8A
:107230000029F8D1A4EB0A041819BDE8F08720460C
:10724000BDE8F087002C04F1FF35E4DC00240029C0
:10725000E9D1F4E703685A1C02601970704700BF57
:1072600010B56FF000440246044404E0B3EB0E0096
:1072700015D1A24214D012F8013BA3F14100192804
:1072800011F8010BA0F1410C98BF203300F1200E42
:10729000BCF1190FEAD91B1A04D10028E9D110BD9D
:1072A000002010BD184610BD884230B54FF00104D3
:1072B0003AD301FB04F4B0FBF4FC8C45F9D2BCB129
:1072C00002BB06E0A14203F8015B11D81446B0FBF3
:1072D000F2FCBCF1090F0CF157050CF1300E04FB68
:1072E0001C00B4FBF1F2EDDCA14203F801EBEDD997
:1072F00000221A7030BDA14203F8015BF8D8144691
:10730000B0FBF2FCBCF1090F0CF137050CF1300EAB
:1073100004FB1C00B4FBF1F2EDDCA14203F801EB2D
:10732000EDD900221A7030BD8446002AEAD1D0E798
:10733000002870B503DA2D23404201F8013B0928EB
:1073400086464FF0010307DD03EB83035B00B0FBD0
:10735000F3F2092AF8D89BB10F4CA4FB030CBEFB37
:10736000F3F2092A4FEADC0C02F1570602F130056C
:1073700003FB12EE07DD092B01F8016B6346ECD825
:1073800000230B7070BD092B01F8015B6346E4D844
:1073900000230B7070BD00BFCDCCCCCC0378202B6C
:1073A00003D110F8013F202BFBD0092BF9D02D2B56
:1073B00000F0A9802B2B75D0B7EE000AA3F13002A4
:1073C000D1B2092977D8F2EE046ADFED5F7A07EED1
:1073D000102A10F8013FB8EEC77AA3F13002D1B2FB
:1073E000A7EEA67A0929F0EE477AF0D92E2B66D0BF
:1073F00003F0DF03452B40F0838010B442782D2A40
:1074000000F096802B2A00F08380A2F13003013037
:10741000092B00F284800024002303EB830302EB9A
:10742000430310F8012FA2F13001303B0929F4D9B0
:10743000B3F59A7F1A46B7EE007A28BF4FF49A72D6
:10744000072B09D91346DFED416A083B27EE267A60
:10745000072BFAD802F00702DAB1F2EE046A012A29
:1074600027EE267A15D0022A27EE267A11D0032A93
:1074700027EE267A0DD0042A27EE267A09D0052A8F
:1074800027EE267A05D027EE267A062A18BF27EEA1
:10749000267A002C45D0C7EE877A5DF8044B20EEA3
:1074A000270A70474378B7EE000A0130A3F1300293
:1074B000D1B2092987D92E2BDFED237A98D14378D1
:1074C0000130A3F13002D1B2092991D8B2EE047A89
:1074D000F0EE475A06EE902A10F8013FB8EEE66A41
:1074E000A3F13002D1B2C6EE076A092927EE257A48
:1074F00077EEA67AEED903F0DF03452B3FF47DAF9C
:1075000020EE270A70474378BFEE000A013055E7A6
:1075100082780230A2F13003092B7FF67CAFB7EE00
:10752000007A67EE877A5DF8044B20EE270A7047F1
:1075300082780230A2F13003092B01D801246BE7D5
:10754000B7EE007AA7E700BF0000000020BCBE4CE9
:10755000F0B5067906F0E003402B03D145794FF0F2
:10756000FF3406E0602B4FF00105F8D1447905FAAD
:1075700004F40023012006F00706AB4200D1F0BD61
:10758000052E0FD8DFE806F00308101D242448B1AB
:10759000C85CD75C78400FE020B1C856D756C71BEF
:1075A000784278410133E8E70028FBD031F8130036
:1075B00032F81370784080B220420CBF01200020C6
:1075C000F0E70028EED031F9130032F91370E6E746
:1075D0000028E7D051F8230052F82370DAE7F8B515
:1075E0000C4E054633788BB9F8BD25B12388C3F31B
:1075F0000B039D4204D0A288D4E9020152F0BEF9E7
:107600001C34BC42F1D300233370EDE7024C034F2E
:10761000F7E700BF585D002490FF0A0850080B08E8
:10762000037903F01803102B1DD003D833B9B0F839
:107630000B007047182BFAD000207047114BB0F8A0
:107640000B0093F90030591C0BD10F4B1B7803EB47
:10765000430203EB820303EBC30300EB430080B25E
:107660007047DBB2F3E7074BB0F80B0093F901303A
:107670005A1C04D1044B5B7800EB4310EFE7DBB2FC
:10768000FAE700BFC805002438350024032870B588
:1076900018D80D4BC943C60003EBC00001F001012F
:1076A000057A427A81EA0504A2420BD042683AB1D7
:1076B0004D1B106892886942694109018A408261C4
:1076C00033445C7270BD00BF585D00240379062B03
:1076D0000FD1C9B20D290AD8074B59560123C268E8
:1076E0008B40134214BF08464FF0FF307047002113
:1076F000F4E7481C704700BFC4230A08092917D0C3
:10770000B1FA81F35B0999B1013903604A0001F0D4
:10771000030102F00802C1EB01119300C1EB01115A
:10772000A3EB92038900C3EB031381809B0043808A
:10773000704700BFB5EEC00ADFED357A0023F1EEE9
:1077400010FA30B5C8BF30EE270A87B0D8BF30EE88
:10775000670ADFED307A054603A9029320EE270A77
:10776000CDE90033FDEEC07A17EE904A84EAE4706A
:10777000A0EBE47045F022FF002C03A8B4BF2D233A
:1077800020238DF8003050F0E7F801282AD0022895
:1077900034D003281ED003A9684652F055F9684634
:1077A00050F0DAF8044669462846033CE4B2224623
:1077B00052F0E4F8002328462B5550F0CDF82E2245
:1077C000431C0DEB04012A54E81852F06AF92846CC
:1077D00007B030BD302303A968468DF8013052F060
:1077E00033F9DCE743F23002302303A96846ADF8F1
:1077F00001208DF8033052F027F9D0E743F230032F
:1078000003A96846ADF8013052F01EF9C7E700BF82
:107810006F12033A00007A440DF094B838B505466B
:1078200058B14C1E14F8011F284619B9BDE838405C
:107830000DF09CB80DF086F8F4E738BD70B505463C
:10784000B0F8090041F0D2F8054B044628461E78EE
:10785000FFF7E6FE16B1E368184470BDA368FBE7C6
:10786000585D002438B505460C46FFF7E7FF2A7936
:1078700002F0070302F0E002602A29D1052B0CD8A0
:10788000DFE803F0030B0F0B1B1B6A790123934006
:107890000278DBB214B11343037038BD22EA03034C
:1078A000FAE76A790123934002889BB214B113432B
:1078B0000380F2E722EA0303FAE76B7901229A4098
:1078C000036814B113430360E7E723EA0203FAE70E
:1078D000052BE2D8DFE803F0030305050707047072
:1078E000DBE70480D9E70460D7E708B5202152F030
:1078F000BAF8034618461BB102780133202AF9D0A2
:1079000008BD08B5CB0701D4FCF7D0F808BD2DE9B8
:10791000F3410023124D044600EB8106114F05F898
:10792000243FB44203D1104802B0BDE8F08139468B
:1079300028464FF0000852F087F82146684652F07A
:10794000B0F82021684652F08EF828B969462846DA
:10795000043452F079F8E4E780F80080F1E700BFE2
:10796000585D00249F9F0A087C5D00242DE9FF4795
:10797000914604468A461E46FFF7A8FE421CBDF803
:1079800030700546DDF834801FD0B9F1FF3F1FD0BD
:10799000154A3146CDE9000938462368C0474A46B2
:1079A0005FFA8AF12079FAF7C3FB024600B1028838
:1079B000D3B2314638460393C2F30323120B02932A
:1079C000CDE90052094A2368C04704B0BDE8F087FA
:1079D0007B06FAD40C90314623683846044AC446E4
:1079E00004B0BDE8F0476047CE930A08DB930A086D
:1079F000FF930A082DE9F043154685B089461946DC
:107A00006A1CBDF830600D9F28D04FEA101800F0B6
:107A10000F04194A304608F14008CDE900454346B5
:107A2000B847C0B1EBB2D9F8000099F805100F2B98
:107A300011D82A46FAF7C4FB68B1038800210278FE
:107A400030460392C3F303221B0B02920B4ACDE98B
:107A500000434346B84705B0BDE8F0837306FAD447
:107A6000030900F00F00064ABC460C904033304634
:107A700005B0BDE8F04360470E940A0820940A0858
:107A800049940A082DE9F043070987B091461E463C
:107A9000DDF83880403700F00F0439B30EF002FCF7
:107AA000C3790546164A49463046CDE900433B4670
:107AB000C047C0B12868FAF773FEAA796B7912F053
:107AC000020F10494FEA93030F4A18BF0A46E9799B
:107AD00001330094CDE90321CDE901030B4A3B4674
:107AE00000213046C04707B0BDE8F0833B46084A56
:107AF00049463046C4460E9407B0BDE8F04360479F
:107B00005D940A0854980A08C9A90A086F940A08DB
:107B100091940A080823484041B240000029C0B2AD
:107B2000B8BF5040013BF7D1704700BF30B5056882
:107B300004468D4218D901F1FF3E681E00231EF84D
:107B400001CF082183EA0C034FFA83FC5B00BCF1F0
:107B5000000FDBB2B8BF53400139F5D17045EED10B
:107B60006A1C22602B7030BD00236A1C22602B70BF
:107B700030BD00BF9FED067AF7EE007A60EE870A0F
:107B800060EE800A30EEA70A80EE800A704700BFE0
:107B9000DB0FC94010B52DED028B08EE101ADFED9A
:107BA000807ADFED800A0446B8EE488A28EE008A23
:107BB00028EE278AB0EE480A51F0D6F99FED7A7A7E
:107BC000F0EE407AB4EEC70AF1EE10FA40F3BD8051
:107BD0009FED746ADFED756AB0EE677A77EEC67A6C
:107BE000B4EEE67AF1EE10FAF6DC9FED717AF4EE7F
:107BF000C77AF1EE10FA40F3C5809FED6B7A77EE0D
:107C0000677A27EEA76ADFED6B5ADFED6B6A9FEDAF
:107C10006B7AE6EE256A9FED660A67EE865ADFED1F
:107C2000610A38EE000AA6EE267AE5EE877AB0EE13
:107C3000678A51F099F9DFED5C7AB4EEE70AF1EE6C
:107C400010FA5BDDDFED576A9FED587AF0EE407A6F
:107C500030EE660AF4EEC77AF1EE10FAF6DCDFEDEC
:107C6000547AB4EEE70AF1EE10FA62DDDFED4E7AF7
:107C700037EEC00AF7EE007A9FED517A20EE004A07
:107C8000DFED4C6ADFED4C4A0023B0EE673A9FED22
:107C90004B5AE4EE264AC4ED097A60EE043AA36139
:107CA000A8EE073A6361F0EE675A2362F8EE006AC5
:107CB000E361A4EE245AE8EE475A87EE836AA3EE06
:107CC000850AB6EE007ABDEC028B77EEC07A26EE1E
:107CD000077A66EE266A27EE865A67EE277A25EE41
:107CE000866A26EE807A84ED015AC4ED007A84ED2E
:107CF000046AC4ED027A84ED037A10BDDFED317AB7
:107D0000B4EEE70AF1EE10FAA9D5DFED266A9FED91
:107D10002E7AF0EE407A30EE260AF4EEC77AF1EED3
:107D200010FAF6D4DFED227AB4EEE70AF1EE10FA9B
:107D30009CDCDFED267AB4EEE70AF1EE10FA99D575
:107D4000DFED207A37EEC00A94E79FED1E7AB4EE9D
:107D5000C70AF1EE10FA7FF548AF9FED126ADFED2A
:107D60001A6AB0EE677A77EE867AB4EEE67AF1EECA
:107D700010FAF6D49FED0E7AF4EEC77AF1EE10FA0F
:107D80003FF73BAF9FED117AF4EEC77AF1EE10FAB0
:107D90007FF537AF9FED0B7A77EE677A31E700BF5B
:107DA00027D4D236DB0FC940DB0F4940E4CB164164
:107DB000DB0FC93F92E741B99730083C15A82ABEAE
:107DC000F304353FDB0F49C0E4CB16C1DB0FC9BF5D
:107DD000DFED2D0A08B551F0C7F8DFED2C7AB4EECF
:107DE000E70AF1EE10FA28DDDFED276A9FED287A29
:107DF000F0EE407A30EE660AF4EEC77AF1EE10FA51
:107E0000F6DCDFED247AB4EEE70AF1EE10FA2FDDAE
:107E1000DFED1E7A37EEC00A20EE007A9FED1E6A73
:107E2000DFED1E6ADFED1E7AE7EE066A20EE076AD6
:107E3000E6EE877AA6EE270A08BDDFED1A7AB4EEE1
:107E4000E70AF1EE10FADCD5DFED0F6A9FED167A46
:107E5000F0EE407A30EE260AF4EEC77AF1EE10FA30
:107E6000F6D4DFED0C7AB4EEE70AF1EE10FACFDCCF
:107E7000DFED0E7AB4EEE70AF1EE10FACCD5DFEDC5
:107E8000097A37EEC00AC7E7DB0FC940DB0F49406C
:107E9000E4CB1641DB0FC93F92E741B99730083C6C
:107EA00015A82ABEDB0F49C0E4CB16C1DB0FC9BF42
:107EB000B0EEC07AF0EEE06AF0EE407AC6FE875A85
:107EC000F5EE405AF1EE10FA3BD086FEC75A85EE29
:107ED000256A9FED1D2A9FED1D3A9FED1D4ADFED9E
:107EE0001D4ADFED1D2AF7EE005ADFED1C3A9FED2B
:107EF0001C5AA6EE423AE6EE223AA6EE034AE6EE17
:107F0000235AE6EE044AA6EE245A85EE250AF4EE3C
:107F1000C76AF1EE10FA03D59FED127A37EE400AE8
:107F2000F5EEC00AF1EE10FA03D59FED0F7A37EEA9
:107F3000400AF5EEC07AF1EE10FA48BFB1EE400A01
:107F400070479FED070AE2E739094E3DE3B59E3ED3
:107F500088FA163E45FE7F3F99FB243F69A2163EF4
:107F6000A7DFA834DB0FC93FDB0F49402DE9F04FF5
:107F7000884689B01E461178531C0393002900F0EF
:107F80001681002514460746A94609E03846013502
:107F9000C047039C621C21780392002900F08F8067
:107FA0002529F3D16078A31C3028CDE9033923D0EB
:107FB000A0F130034FF0000ADBB2092B26D96C2860
:107FC0002AD078287FD8572878D9A0F15803202BB9
:107FD00079D8DFE803F0BD787878787878787878A1
:107FE0007882AF787878787878787878AA7878789E
:107FF000789E788A7878BD00E31CA0784FF0010A5B
:108000000393A0F13003DBB2092BD8D804AA03A94B
:1080100046F0F4FF6C28D4D1039B1A785C1C782AB4
:108020000394B7D8572A40F28E80A2F15803202B30
:10803000B0D801A151F823F06F810408957F04089E
:10804000957F0408957F0408957F0408957F0408B0
:10805000957F0408957F0408957F0408957F0408A0
:10806000957F0408DD8004088B810408957F04084F
:10807000957F0408957F0408957F0408957F040880
:10808000957F0408957F0408957F0408957F040870
:108090002D810408957F0408957F0408957F0408C6
:1080A000957F040815810408957F04089B810408C6
:1080B000957F0408957F04086F81040828B9284635
:1080C00009B0BDE8F08F039C64E72528FBD1039C31
:1080D000252138460135C0475CE7039C56F8041B50
:1080E00038460135C9B2C04754E70DF1140B0022E0
:1080F0000A2156F8040B5B46039CFFF7D5F853465C
:10810000049A41463846CDF800B0FFF765F80544BB
:1081100040E7039C56F8040B0023049A4146009064
:108120003846FFF759F8054434E7039C56F8043BFA
:108130001D602FE70DF1140B56F8040B039C5946F4
:10814000FFF7F6F8DBE7002AB9D0252AC0D021E7EF
:10815000A0F158020DF1140B102156F8040BB2FADD
:1081600082F25B465209FFF79FF8039CC7E7A2F132
:1081700058020DF1140B102156F8040BB2FA82F2DA
:108180005B465209FFF790F8B9E70DF1140B56F86A
:10819000040B5946FFF7CCF8B1E70DF1140B0022A0
:1081A0000A2156F8040B5B46FFF77EF8A7E70D4659
:1081B00085E7F8B5104C07460D461646A06CA0B1F1
:1081C0000E49FFF72BFB3946A06CFFF727FB0C4944
:1081D000A06CFFF723FB0B4933462A46A06CFFF740
:1081E000C5FE0949A06CFFF719FB94F84C3013B198
:1081F000012384F84D30F8BD585D0024A3940A088B
:10820000C0AE0A0819780408B0940A080EB400B584
:1082100084B0084905AB019001A853F8042B0393DF
:10822000FFF7A4FE0022019B1A7004B05DF804EB76
:1082300003B0704755720408F7B5114E0746002386
:108240000C46304615460F494E3600F84E3F04EBBB
:1082500045050D4B002F18BF19460C4F51F0F4FB8C
:10826000AC4202D10A4803B0F0BD394634F8022BC3
:108270006846FFF7CBFF6946304651F0E5FBEFE774
:10828000585D0024BD940A08B4940A08C6940A08EC
:10829000A65D0024F7B500230B4E044600EB410514
:1082A0000A4F06F87F3FAC4202D1094803B0F0BD47
:1082B000394634F8022B6846FFF7A8FF6946304676
:1082C00051F0C2FBEFE700BF585D002401980A0897
:1082D000D75D0024F8B54E1E054601F11F04054F79
:1082E00016F8012F284639460235FFF78FFFA642C0
:1082F000F6D1F8BDCB940A0802460846531C05D1B6
:10830000034B1A681B790A600B71704701497DE7BE
:1083100009940A0802980A0810B5013114460DF0B4
:10832000C1FF28B9054B1A681B792260237110BD63
:10833000C27920460249BDE8104067E709940A085F
:108340006A940A0803685A1C02601970090A0368D3
:108350005A1C02601970704702681346511C016074
:1083600013F802CB0360D31C5178036093781B048D
:1083700043EA0123111D43EA0C030160D07843EA6C
:1083800000607047A0F13003092B07D920F02000CE
:10839000413819288CBF0020012070470120704708
:1083A000303809288CBF0020012070474138192837
:1083B0008CBF002001207047613819288CBF002035
:1083C0000120704720280BD0092809D00A2807D09F
:1083D0000D2805D00B3801288CBF002001207047E4
:1083E00001207047A0F14103192B98BF203070473E
:1083F000A0F16103192B98BF2038704702B384465F
:1084000010B5841803E0981A15D1A44514D01CF8AF
:10841000013BA3F14100192811F8010BA0F1410E15
:1084200098BF203300F12002BEF1190FEBD91B1ABF
:1084300004D10028E9D110BD002010BD184610BDA0
:108440001046704770B5044608460D464FF084FA52
:10845000064602E014F8013F43B132462946204661
:10846000FFF7CCFF0028F5D1204670BD1C46204602
:1084700070BD00BF2DE9F043064686469EF800C059
:1084800074460EF1010EBCF1200FF7D0BCF1090FBC
:10849000F4D0BCF10A0FACF10B00EFD0ACF10D053C
:1084A000B5FA85F56D09002DE8D10128E6D9BCF1B2
:1084B0002B0F3DD0BCF12D0F39D0102A3ED04FF0FC
:1084C000FF3E9046BEFBF2FE02FB0EF7FF43FFB2FB
:1084D000002014F801CBBCF1390F4CF02009ACF1AD
:1084E000300C0DD85FFA8CFC944510DA70452646A6
:1084F00002D819D1674517D21D404FF0FF30E8E789
:10850000A9F1570CB9F1600F5FFA8CFCECD801B1FE
:108510000E6003F00103D5B9002803DA002B18BF61
:108520006FF00040BDE8F08300FB08C0D1E70125F3
:10853000102A94F801C004F10104C0D1BCF1300F3D
:1085400010D06FF0704E0F274FF01008C0E7B0F159
:10855000004F04D91BB14FF00040BDE8F08340420A
:10856000BDE8F08360786FF0704E0F274FF0100871
:10857000A0F14106192E04F1010698BF2030782899
:108580000CBF02343446A3E773B50E4610490546C6
:10859000FEF766FE18B93070012002B070BD2C786D
:1085A000602C8CBF613C413C082C0FD80135012365
:1085B0000A2201A92846FFF75DFF019BAB4205D0C7
:1085C0000F2803D8013440EA0410E4E70020E4E770
:1085D00009940A0801230A2200214BE770B50D46D1
:1085E0001446FFF782F90646A0B1FFF7F3FF40F605
:1085F000340319229842A8BF1846B0F5617FB8BF6E
:108600004FF46170A0F56173B3FBF2F32B70237824
:10861000013323703046FFF768F90646A0B1FFF733
:10862000D9FF40F6340319229842A8BF1846B0F586
:10863000617FB8BF4FF46170A0F56173B3FBF2F3D3
:108640006B70237801332370304670BD2DE9F04103
:1086500016461F46404D0446394630464FF47A725E
:1086600000234FF0D7FD3D4B05443D4F3D4E83FB6E
:108670000510E9172844C1EB601183FB0103C817FB
:108680000B44C0EB631087FB003CC317C3EBAC0388
:1086900086FB03764FEAE37ECEEBE61EC1EB0116C6
:1086A000A5EB860CC0EB00154FEA8E0684F806C0D9
:1086B000A1EB8501617103EB4301A0EBC10040F226
:1086C000B55101FB1E332071B3F5896F33DA40F2E7
:1086D000DA218B4237DCB3F5B77F234FB4BF4FF0BD
:1086E000000E4FF0010E0EEB4E0175464FEA4E089C
:1086F00007EBC101C88A08EB0E0C0B2107EBCC0C71
:108700000CF1160C01E03CF8020D984210DD013925
:10871000F9D1F044012137F8380006F5FA6E01333B
:10872000A17075441B1A22812580E370BDE8F08199
:108730000131C9B2F1E7032540F296500A4F4FF0DC
:108740000608AE46D7E7022540F22940064F4FF013
:108750000408AE46CFE700BF80BC92C789888888EE
:10876000ABAAAA2A73B06D1684BB09080D4B10B5CD
:10877000D3E9004354EA03020AD10146002340F240
:10878000011218460B80C1F802208B710B8110BDBD
:10879000054A1268121943F10003FFF757FF012041
:1087A00010BD00BF30350024182300242DE9F0410E
:1087B0000446154608469442B4FBF2F607D205FB80
:1087C0001644134B1B5D00F8013BBDE8F081964257
:1087D000B6FBF2F70CD20E4B05FB176705FB1644F0
:1087E000DA5D1B5D00F8012B00F8013BBDE8F0816C
:1087F000BA42B7FBF2F807D905FB1878044B13F817
:10880000082000F8012BE7E74046FFF7CFFFF3E72A
:10881000E0230A08794B9A88B2F57A7F02D94FF49F
:108820007A729A80DA88B2F57A7F02D94FF47A7236
:10883000DA801889B0F57A7F03D94FF47A7210463E
:108840001A81B3F80AC0BCF57A7F02D90022944697
:108850005A819A89B2F57A7F4BD94FF47A72D989C5
:1088600091429A8149D900228445DA8180F0B08012
:10887000598B9A8B914201D900225A83604B1B88F5
:10888000002B41D010B55F4C82B0A278062A63D984
:108890002179002940F09E809FED5B7A5B4A07EECC
:1088A000903AA3791178F8EEE77A06EE901AB8EECE
:1088B000E66AC6EE276A0BB137EE077AB4EEE67ABF
:1088C000F1EE10FA67DC524A5378032B5FD8514916
:1088D00001EB43111078504B0328C3F8D0144ED845
:1088E000EA2203F5947300FB02334C4A136002B092
:1088F00010BDD989B1F57A7F3CD8844519D291420F
:10890000B6D300229A81B3E7414A5378032B13D898
:108910004049107801EB43113F4B0328C3F8D014B2
:1089200013D8EA2203F5947300FB02333B4A136029
:10893000704700201881E2E7002310783549537012
:108940000328354BC3F8D014EBD9002103F59473F9
:108950001170324A136070473149207901EB82016E
:1089600091ED187A002899D0531F032BABD9002A18
:10897000A9D035E000218445D981C0D3D9E70021B1
:1089800003F594731170254A136002B010BD0023E3
:10899000204953709EE767EE877ABCEEE77A8DED4B
:1089A000017A9DF8043007EE103AB8EEC77AF4EE7B
:1089B000C77AF1EE10FA01DD0133DBB2E3B1102B1F
:1089C000A8BF1023DBB28B4238BF0B4613707AE787
:1089D0001A814DE7053A032A7FF675AF9FED0A7AB3
:1089E000B7EE000A80EE070A50F0F0FA23888342BF
:1089F00028BF0346238066E70123E3E7003700240E
:108A0000A01D00200C2F00246F120338B436002460
:108A100038350024005E0024585D0024BC36002454
:108A200084BB09082DE9F04F924B83B01B7800AF4F
:108A3000A3F11702022A00F2D5828F4E8F4C4FF01D
:108A4000000A94F8DC3404F5B06804F5A1697B6091
:108A5000D9F8005015F0010B40F0828299F90420FA
:108A6000142A11D0284651F097F9AA0340F16A82DE
:108A7000012809D0082807DCBBF1000F00F075823F
:108A80007F4B1D4240F061827E497F483FF0C4FF2A
:108A90000023022084F8843512F00AF894F888350F
:108AA0007A4A022B156800F01483002800F06083D6
:108AB000DFF8F091764B4FF47A7A94F8E1C54FF0F5
:108AC000000E03F56A7B4FF06408C7F804C033F862
:108AD000082CB2F57A7FB3F8462088BF23F808AC9B
:108AE000B2F57A7F33F8062C88BFA3F846A0B2F51A
:108AF0007A7F33F8042C88BF23F806ACB2F57A7F6E
:108B000002D9002223F804EC33F8061C9142B3F892
:108B10005A10B3F85C2098BF23F806EC914293F802
:108B20006B2003F1650102F1FF3288BFA3F85AE020
:108B3000632A93F86C2002F1010288BF83F86B80EE
:108B4000D2B2092A4FF0000288BF83F86CE013F814
:108B50003200013211F801CF844538BF81F800E0BE
:108B6000032AF4D17A68EA33012A18BF03F864ECC7
:108B70009B45ACD1DFF830A19AF80230042B00F00D
:108B8000D6822BB9BAF80030B3F5F07F00F23F82FD
:108B9000FFF740FE3F4894F8F415FEF7AFFD1030A4
:108BA00094F81316FEF7AAFD103094F82316FEF77A
:108BB000A5FDB4F83226B4F830361343B4F83426A1
:108BC00013431BB213B10123A4F83636324B2B40AA
:108BD000002B00F0DC82E80700F18B82690400F1D1
:108BE00025822A0740F162822C4A284B15401D60DD
:108BF000D9F800301340C9F8003015F4004300F0F4
:108C00003A82002384F8E33484F8F334E80440F132
:108C10003C8294F84336022B02D1012384F8433678
:108C2000DFF87C80434608F1780B02E006339B4571
:108C30000CD01A780A2AF9D19978DA78914202D3BD
:108C40005A79002AF2D00A201EF05EFA00234FF46F
:108C5000806084F8843511F02BFF002800F07C82BE
:108C60000F490D467960687960B3297839B3434676
:108C70001FE000BFE435002484BB0908585D0024D0
:108C8000BC02020060620024DC010B08603B00248F
:108C90008A5E00245C63002409600002FE9FFFFDE1
:108CA000A0630024683500240C2F002406339B4564
:108CB00008D01A788242F9D15A79002AF6D00846AB
:108CC0001EF022FA0635AB45CDD19AF802807968BC
:108CD000B8F1080F00F0EF8194F8E135D9F8000001
:108CE000A3F10103C0F3C032B3FA83F384F8C326BF
:108CF0005B0984F8C03694F8E235A3F10103B3FAB6
:108D000083F35B0984F8C636A54B5A78032A01D948
:108D100000225A70A34DA44A2B6813400240A34876
:108D20002B60807BC9F80020002800F0EE81A04D68
:108D3000AB88002B40F0DF819E4A1368B3F5000F2B
:108D400001D30023136093689B48184010B140F290
:108D5000022393601379013B042B01D90123137182
:108D6000A8F10508954BB8F1030F93F8009040F275
:108D70007981B9F1000F28D00025DFF860827D608D
:108D80003E6045464E46894606E0A8F10608A8EB37
:108D90000A039E4240F24C81A84615F8010F0028B4
:108DA000F3D00DF0A3FA0028EFD083799B07ECD520
:108DB0007D6849463E6801223DB19AF8113053B9A9
:108DC0009AF80530012B00D02AB19AF8063013B179
:108DD00000238AF806307A4BDA8802F00F00042864
:108DE00003D8C2F30312022A02D94FF42062DA80B8
:108DF0001A8902F00F00042803D8C2F30312022AD2
:108E000002D940F601221A8194F8D90694F8E52691
:108E100094F8D836904205D9002284F8D92653B167
:108E2000A4F8DC2694F8E4269A4204D2002384F8BD
:108E3000D836A4F8DC3694F8DA2694F8CE379A427D
:108E400002D9002384F8DA36DFF894C10CF1800AE5
:108E5000634613F8032D02EB4202324492F8549118
:108E600092F8558192F856E113F8015F98794D45D3
:108E7000DA78A8BF4D464045A8BF404672451D70F0
:108E8000A8BF724663459871DA70EDD103F1200CEA
:108E9000D445DDD1D4F80025002A00F03D8100251D
:108EA000012002E006318B450ED00B782B2BF9D137
:108EB0004B78043300FA03F31342F3D0063122EA6D
:108EC000030201258B45F0D10DB1C4F800253D4DBD
:108ED0006E4605F108082B4602E0434500F0AD80E0
:108EE00013F8012F072AF8D9002305F8013F0133B1
:108EF000082BFAD1B4F8DA25B546B4F8D8359A4239
:108F000002D3314BC4F8D835304BFF22304D03F13A
:108F1000780084F8002813F9082C142A05D053F897
:108F20000C1C35EA010100F0FF800C339842F2D1AD
:108F3000284B5A79022A01D100225A710C37BD46BA
:108F4000BDE8F08F01283FF795AD09F10C09C84540
:108F50007FF47EAD0AF1FF32022A7FF699AD93E5E8
:108F60000AF1010A5FFA8AFA7CE56B067FF58CAD9F
:108F700015F4057F09D07B680F2BE6D0012BE4D0D8
:108F80009A1E052AE1D9102BDFD0134AAA437FF499
:108F90007BAD09F10C09C8457FF45AADDAE700BF93
:108FA00000370024603B0024BCD455183835002419
:108FB0006C360024C4360024FDFDFFFF481C002051
:108FC000383A00241E2F0024AE014A016C620024AE
:108FD00001000200B027002440000200132F0024EB
:108FE000055E00246E4A12F83310A9B9DB001A445A
:108FF0006C4E5278002A3FF421AD334493F87C3014
:10900000002B7FF41BAD1823674A137016E54FF44D
:10901000F073AAF80030BBE502EBC301DB0049683E
:109020000029E4D1172160480170E0E75F4ADCE5E0
:109030007D6849463E680022BEE688B02022FF21B6
:10904000E946484650F0F8FC594A04E0424549F8E0
:1090500023303FF44FAF12F8013F59F8231001318C
:10906000F4D041E700238AF80430B9F1000F00F092
:109070008C80012581E694F8E324002A3FF4C6ADF4
:10908000E80484F8F3343FF5C4AD29067FF5C1AD9B
:10909000454B1A78182A04D8464BD340DA073FF5D7
:1090A000B8ADDFF8248108F1780BCFE5AB047FF58C
:1090B000A4AD414A99E59AF80630002B3FF40CAE76
:1090C0009AF81130012B7FF407AE02238AF8113091
:1090D00002E600283FF4ECAC90F904904FF0FF0A50
:1090E00001E080F808A048460EF064FF0028F8D19F
:1090F000DEE4324A79E5287879600DF0F7F879688E
:1091000000287FF419AEA88016E62D4803430243D9
:109110002B60C9F800200AE62B2079601DF0F4FFCF
:10912000D4F800257968BAE684F8002800E7254BD2
:1091300025F480551D60D9F8003023F48053C9F818
:109140000030BAF82030B3F57A7FBFF421AD4FF488
:109150007A73AAF820301BE51A4A136823F00063DB
:109160001360D9F8003023F00063C9F8003077E5C8
:10917000144B25F08005DFF854901D60D9F80030BD
:1091800023F08003C9F8003094E44A4615E6D9F884
:10919000003045F0080543F00803C9F8003023E526
:1091A00090B2090884BB0908E4350024F6DFFFFD0E
:1091B0001E2F002400410001F6BFFFFDF79FFFFDB9
:1091C00000040500603B0024A063002468350024EF
:1091D0002DE9F04F704F83B0704BFA68DFF8E481EF
:1091E00002F2DC524345FA6080F0D280DFF8D89179
:1091F00001229B466A4D09F102060192B9F802105C
:10920000002900F0AF80052906EB010240F2AA8098
:10921000AA4280F0A780BBF800003446C0F30B00E0
:109220000BE0118814460A44002900F09B80AA42F2
:1092300080F09880052940F2958061888142F0D1C4
:1092400061798B07EDD123885846DBF8081094F834
:1092500004A000933FF0E0FBBBF80010BAEB113F15
:1092600000F0868000230193BBF804100BF11C0B67
:109270005BF8140CC1F30B015BF8044C45F02CFABD
:10928000C3452060BAD3474A474C484B1268DFF8C1
:109290003C811A60FFF7C6FB98F80010EA2204F53B
:1092A0009473434D434E01FB023398F801202B6029
:1092B00004F1A80303EB4213C4F8D0341DF0EAF91B
:1092C0004FF0FF332868736025F01CFA1DF062FF31
:1092D00004F5C96304F5D86102E00633994251D020
:1092E0001A78002AF9D19D78D878854202D3587926
:1092F0000028F2D094F84036327203EB8303B4F8BE
:10930000442603EB83039B00642BB8BF64237B607C
:10931000642303FB02F20023642A7B61BB84B8BF91
:10932000642287F82630C7E90333BA603A62224ADA
:10933000C7E90633214B936226F0A2FEB4F8040875
:1093400094F806181FF020FE34F0E0FC16F042FE00
:109350001B4B012201981B6887F82520FB6003B096
:10936000BDE8F08FDBF8081058463FF055FB79E771
:10937000009BA11D58469A1F3FF084FB00287FF4F4
:1093800073AF6FE798F80F20003A18BF0122B1E7DA
:109390000123019377E700BFD436002490FF0A0829
:1093A00000000408603B0024585D00246835002458
:1093B000BC360024C8050024302300208863002424
:1093C0001823002450080B08000002083835002438
:1093D000104B0122032810B504461A7005D9601CF1
:1093E000BDE81040C0B211F077BDEA210A480B4A2F
:1093F00004FB01000A4B1470186025F083F922F079
:1094000098FB22F079FC601CBDE81040C0B211F05E
:1094100063BD00BF00350020805E00243835002485
:10942000BC360024044A01200449136881F8080866
:1094300043F4001313607047B0360024585D0024D5
:10944000F8B5164D6B78BE2B26D1AC1C144F0222FA
:1094500029464FF6FF70FDF7A1FE22884AB1A618F3
:10946000BE4219D2052A17D921463446FDF796FE89
:10947000F3E721460222FDF791FE0222A1180634ED
:10948000FDF78CFE074B641BA3F80A4841F60F5307
:10949000C31A58425841F8BD0020FCE700000208FA
:1094A00000000408585D002470B5046886B00546C5
:1094B0000E46C4F310033BBB01220393CDE90133F5
:1094C0002023CDE9042304F17843B3F5801F19D399
:1094D000A4F10163B3F5801F10D2A4F5801302221A
:1094E00003F17843694601A802925B0C039340F0B4
:1094F00069FB48B14FF0FF3006B070BD0520FCF7A6
:10950000C9FEFBE72346EBE73146204646F04AF822
:1095100018B92B6820332B60EEE76FF00200EBE701
:109520002DE9F0416A4E90B03378B12B7ED1FFF730
:1095300087FF80F00104E4B2664B04F00104664D3D
:10954000B3F86331654FADF80030BD4270D3002CE5
:1095500000F0BC802822002106A850F06DFA604B74
:1095600004969B1B05935F4BDA68D40770D45D4B60
:10957000D3F80C21D00774D44FF4807302226946CB
:1095800004A8ADF83C304DF0C7FB022269464FF607
:10959000FF70514DFDF702FE4FF000080446BD423A
:1095A00069D30025022201A904A8ADF804504DF0AA
:1095B000B3FB022201A92046FDF7F0FD40BA0222CA
:1095C00002A9C043ADF8080004A84DF0A5FB0E9811
:1095D00088B106ABC0F120022946184450F02CFA9D
:1095E0009DF93C0018B906A904A8FFF75DFF002308
:1095F0008DF83C000E939DF83D307BB1394BDA6815
:1096000042F00102DA60DA68D20707D5D3F80C21FC
:1096100042F00102C3F80C21D3F80C319DF93C0053
:10962000B0FA80F0400910B0BDE8F081012483E772
:10963000AB691C3535F8181CD3F8008055F8140CAC
:10964000C1F30B0145F048F8804518BF01247CE7C1
:10965000254A5A6002F188325A60DB68D90786D5FC
:109660008AE7214AC3F8042102F18832C3F80421B1
:10967000D3F80C3180E7AE8802A904A88DF80D80DC
:10968000C6F30B061C35B31DADF8083035F81C3C8D
:10969000C3F30B021B0BADF80A2006228DF80C3029
:1096A0004DF03AFB062202A92046FDF777FD04465D
:1096B00055F8141C324604A84DF02EFB204655F8F0
:1096C000141C3246FDF76AFD044668E70120AAE74C
:1096D0000000020884BB090890FF0A0850080B0824
:1096E00000000408002000522301674570B5164DA4
:1096F000FFF798F90324154EEB6803F2DC53EB6097
:10970000FFF70EFF58B13378B12B08D1FFF798FE61
:10971000013C16D040B9FFF703FF0028F3D1013C0C
:10972000EED10520FCF7B6FD09490022094B0120C6
:10973000096883F80C2885F82500E96083F80D286E
:1097400070BD0028F0D1ECE7D436002400000208F8
:1097500018230024585D002410B5074A0124074B44
:1097600014709C73FFF7C2FFFFF732FD2046BDE87F
:10977000104011F0B1BB00BF003500203835002487
:1097800090F89230B7EE007ADFED6A6A014607EE94
:10979000903A90F89630684AB0EE476A05EE103A73
:1097A00090F89430F8EEE77A04EE903A90F895301D
:1097B000B8EEC55A05EE903A90F8983067EEA67A62
:1097C00004EE103A25EE265AF8EEE44AF8EEE55A91
:1097D000B8EEC44A25EE275A64EEA64A65EEA65AAC
:1097E00024EE264A64EE854A65EEA75A24EE274AFF
:1097F000B0EE473AF0B590F8917000F16F0602F1C3
:109800001A050024137807EE903AF8EEE77A67EE2F
:10981000857A67EE867AFDEEE77A17EE903AFA2BB4
:10982000A8BFFA2323EAE3730B72537807EE903A4A
:10983000F8EEE77A67EEA47A67EE867AFDEEE77ACD
:1098400017EE903AFA2BA8BFFA2323EAE3734B7280
:10985000937803EE903AF8EEE33A63EEA57A67EE7A
:10986000877AFDEEE77A17EE903AFA2BA8BFFA2333
:1098700023EAE3738B72938807EE903AF8EEE77A67
:1098800067EE847A67EE867AFDEEE77A17EE903A15
:10989000D5ED007AB3F57A7FF8EEE77AA8BF4FF4FA
:1098A0007A7323EAE3738B812B68002B3FDD90F8FA
:1098B0009730B0EE436A02EE903AF8EEE22AA2EE5A
:1098C000E66A63EE863A83EEA76AA2EEA66A65EEC2
:1098D000A77A013467EE877A67EE867AFDEEE77A3B
:1098E00017EE903AFA2BA8BFFA23BC4223EAE3739F
:1098F00006F8013F00DDF0BD012C13D190F8933044
:1099000007EE103A90F89B3006EE103AB8EEC77AA0
:10991000B8EEC66A27EE267A26EE266A04350832A5
:1099200008316FE7B7EE007AB0EE476AF6E7B7EEB8
:10993000006ACCE70AD7233CEABC090890F89930C2
:109940006BB3B0F864308BB190F89A20642102EBCD
:109950008203C3EB0313B3FBF1F3A0F86430962347
:1099600012FB03F3B3FBF1F3A0F8663043884BB16D
:1099700090F89A30642203EB8303C3EB0313B3FB29
:10998000F2F34380B0F850304BB1962290F89A3001
:1099900013FB02F36422B3FBF2F3A0F850307047DC
:1099A00090F821304BB3438B83B190F82230FA22E8
:1099B000642113FB02F203EB8303B2FBF1F2B3F574
:1099C0007A7F4283A8BF4FF47A738383838843B13D
:1099D000FA2290F8223013FB02F36422B3FBF2F375
:1099E0008380C3884BB190F8223003EB8303B3F537
:1099F0007A7FA8BF4FF47A73C380704770B50A4C62
:109A000000250A4E94F8913013B12046FFF7B8FEB6
:109A100020460135FFF792FF3046FFF7C1FF042DC6
:109A200004F1EA04EED170BD805E0024003700240A
:109A300010B5064C4FF48072002104F60E004FF072
:109A4000FBFF0023C4F8103910BD00BF585D00248F
:109A5000034BD3F8140908B10AF088BF704700BF60
:109A6000585D002408B50B4605490246D1F8140993
:109A700028B10449FEF77AFABDE80840E8E708BDD6
:109A8000585D002419780408024B0146D3F81409E4
:109A9000FDF7C4BE585D00240048F5E7C7A90A08D1
:109AA0000CB4C30607B500D561B905A904980191A6
:109AB000FFF7D8FFFFF7F0FF012003B05DF804EBDC
:109AC00002B070470020F8E70FB407B504A951F8B9
:109AD000040B0191FFF7C6FFFFF7DEFF03B05DF84F
:109AE00004EB04B070470349034801F500610EC957
:109AF000EAE700BF00E0F11FD0940A0870B5002427
:109B0000144E96F82330651C2341DB071CD5E4B2C4
:109B100029461148FFF7D8FF7521204628F072FE2C
:109B200001460E48FFF7D0FF1A21204628F06AFEB2
:109B300001460B48FFF7C8FF1B21204628F062FEB4
:109B400001460848FFF7C0FF022D4FF00104D8D1AD
:109B500070BD00BF00370024E4940A08F0940A089E
:109B600003950A0816950A0808B5FFF78DFFBDE8AA
:109B7000084091E72DE9F04385B0224EFCF73CFD0B
:109B80000269838900250188044602928268DFF811
:109B9000888001924288DFF884901B4F00924268CF
:109BA0001A48FFF791FF15B91948FFF7DDFFD8F8FC
:109BB00000309D4212DA3378052B20D809EB83035D
:109BC000D3F88C21B38829460135384600930636F0
:109BD00036F8043CFFF778FF062DE4D145F036FA5D
:109BE0004288838864689B1A03FB0444FCF7C6FD23
:109BF00002460848214605B0BDE8F04364E700226C
:109C0000E0E700BF2430002493950A0829950A084C
:109C100087950A08A2950A084830002484BB0908E1
:109C200010B504460348FFF72FFF2046BDE810405B
:109C30009AE700BFBF950A0808B5034610460AB95F
:109C4000002008BDDB0601D50029FAD0FFF7E8FFA8
:109C5000F6E72DE9F04F724C8DB0DFF8D0910A464F
:109C600004F1B00A00218346FFF7E6FF03900025C8
:109C7000A37A99F80060AB4200F392801034544507
:109C8000F5D140F216200DF1180A3EF0AFFE002784
:109C9000002E4FF015024FF00001D0E9024550466A
:109CA00004BF254634464FF0C7FE2E78002E3ED026
:109CB0006978304605910CF0F5FA95F90290049018
:109CC00009F1010253425341002C00F0A68000220A
:109CD0000599A05CB04240F09C80224492F9028039
:109CE000C14540F0948052788A4208BF0123012286
:109CF00003F001030AF8072083F00101039A584694
:109D00000593FFF799FF059B039044B1454A304600
:109D10000499CDE900B24246FDF76CFE059B424A2C
:109D200030460499CDE900B24A46FDF763FE01379B
:109D30000335152FB9D184B3564604F13F07DFF838
:109D4000E480DFF8E49016F801ABBAF1000F21D1FE
:109D50002078F8B194F9023001331BD061780CF00F
:109D6000A1FA0546039A01215846FFF765FF94F9C9
:109D700002205346294603902078CDE900B8FDF72C
:109D800039FE207853464FF0FF322946CDE900B91D
:109D9000FDF730FE0334BC42D5D10DB0BDE8F08FE5
:109DA000E0883EF023FE002E627AD0E90231207A6C
:109DB00004BF1946334605FB00228F5623B39E5637
:109DC000B742039A5846049313BF012100214FF074
:109DD00001084FF00008FFF72FFF049B039043B1E9
:109DE000104B324629462046CDE900B34346FDF7E5
:109DF000BDFD0D4B29463A4620460135CDE900B35D
:109E00004346FDF7B3FD33E74FF0FF36D8E70023B5
:109E10006DE703323F2A7FF45CAF4FF0FF386BE70A
:109E2000D4050024A19F0408A19A0408585D0024C9
:109E300010B508460749FDF713FA002815BF01249D
:109E4000002405480548FFF7EBFE2046BDE810401A
:109E50000AF02ABAC4950A08CD950A08F4950A08AA
:109E60002DE9F04F0C4607468BB040F216203EF02D
:109E7000BDFD2246054600213846FFF7DDFE404B7A
:109E8000064615221B78002104A8002BD5E90245BF
:109E900004BF25461C464FF0CFFD05F13F03039359
:109EA00095F80090B9F1000F30D095F801A0002C82
:109EB00063D0224600231178494557D1283392F8C0
:109EC000018001226B4403F8182CD04532463846F5
:109ED00013BF012100214FF0010B4FF0000BFFF7E2
:109EE000ABFE064654B1B8F1000F07D0254B5A46D9
:109EF0004146484600933B46FDF7C4FD224B5A4677
:109F00005146484600933B46FDF7BCFD0335039B95
:109F10009D42C5D13CB3651C0DF110084034DFF8FB
:109F20006490DFF864A018F8013BCBB915F8013C48
:109F3000B3B116B13046FFF773FE29783B4615F8EA
:109F4000010C0022CDF800900026FDF79BFD0022B9
:109F500015F8010C3B461146CDF800A0FDF792FD27
:109F60000335A542DFD10BB0BDE8F08F01330332DA
:109F7000152BA0D14FF00008A7E7A046A5E700BF2A
:109F8000585D0024A19F0408A19A0408034B0146D0
:109F9000D3F8140908B10AF0D5BC7047585D002405
:109FA0000CB407B510F020000BD079B92320FFF7CF
:109FB000EDFF05A904980191FFF754FDFFF76CFD33
:109FC000012003B05DF804EB02B070470020F8E711
:109FD0002DE9F04F914687B00C461A460021804685
:109FE0004D46FFF729FE00270646B9F1000F63D062
:109FF0002946062220464FF073FE0028324640468E
:10A0000013BF012100214FF0010A4FF0000AFFF7B2
:10A0100013FE0646287815F069FF8346F8B1687983
:10A0200015F064FF4FF461714FF0190CAB78EA78CA
:10A030009BF805E01CFB03131CFB021295F801B012
:10A04000297900B14079CDE90410CDE902325146B9
:10A050003B461A4A4046CDE900EBFFF7A1FF2078C6
:10A0600015F044FF8346F8B1607915F03FFF4FF4D7
:10A0700061714FF0190CA378E2789BF805E01CFBA6
:10A0800003131CFB021294F801B0217900B140794E
:10A09000CDE90410CDE9023251463B46074A40461D
:10A0A000CDE900EBFFF7FCFC013706340635142F31
:10A0B0009BD107B0BDE8F08FCA46D0E710960A08DA
:10A0C0002DE9F04F904689B01A460C460021814692
:10A0D0004546FFF7B1FD3A4E08F178030746DFF831
:10A0E000E4B0079394F904000DF064FF00285CD0FD
:10A0F000B8F1000F61D029460C2220464FF0F0FD48
:10A1000000283A46484613BF012100214FF0010ABA
:10A110004FF0000AFFF790FD074695F9040043F061
:10A1200037FAEA790346514606EB82024846D2F8EE
:10A13000A42104922A7A06EB8202D2F8A421039287
:10A14000AA7906EB8202D2F8A42102926A7906EB80
:10A150008202D2F8A42101922A6800925A46FFF79F
:10A160001FFF94F9040043F013FAE27903465146C5
:10A1700006EB82024846D2F8A4210492227A06EB2A
:10A180008202D2F8A4210392A27906EB8202D2F8CD
:10A19000A4210292627906EB8202D2F8A4210192F4
:10A1A000226800925A46FFF77BFC0C35079B0C3463
:10A1B000AB4297D109B0BDE8F08FC246D1E700BFEE
:10A1C00084BB090829960A082DE9F04F90468BB008
:10A1D00000264FF0190A45464FF461790C461A469D
:10A1E00000210746FFF728FD0990B8F1000F49D07C
:10A1F00029460A2220464FF073FD0028099A384666
:10A2000013BF012100214FF0010B4FF0000BFFF7AE
:10A2100013FD2A890990334606925946EA88384642
:10A2200005922A790492EA780392AA781AFB02929C
:10A2300002926A781AFB029201922A780092124ADC
:10A24000FFF7AEFE2289334601365946069238465C
:10A25000E2880A35059222790492E2780392A27884
:10A260001AFB0292029262781AFB0292019214F88F
:10A270000A2B0092044AFFF713FC1E2EB5D10BB037
:10A28000BDE8F08FC346DDE746960A082DE9F04F9A
:10A29000804691461E460C4615460027DFF81CA155
:10A2A0002DED088B95B094ED008AB5EE408AF1EE65
:10A2B00010FA7BD0D4ED019A94ED029AD4ED038A82
:10A2C000B9F1000F49D0D5ED00BA95ED01BAB4EE61
:10A2D0006B8AD5ED02AA95ED03AAF1EE10FA6AD1C8
:10A2E000F4EE4B9AF1EE10FA65D1B4EE6A9AF1EE03
:10A2F00010FA60D1F4EE4A8AF1EE10FA0CBF012197
:10A30000002132468B46404681F00101FFF794FC64
:10A31000B0EE6B0A064611A8FDF70CFAB0EE4B0A38
:10A3200007900EA8FDF706FAB0EE6A0A06900BA891
:10A33000FDF700FAB0EE4A0A059008A8FDF7FAF911
:10A340000599069A079B039040460291594601924F
:10A35000524600933B46FFF723FEB0EE480A11A891
:10A36000FDF7E8F9B0EE690A83460EA8FDF7E2F9B9
:10A37000B0EE490A06900BA8FDF7DCF9B0EE680ACA
:10A38000059008A8FDF7D6F9069B059A00210390D1
:10A3900040460292524610341035CDE900B33B4698
:10A3A0000137FFF77DFB082F7FF47DAF15B0BDECC3
:10A3B000088BBDE8F08F0021A3E700BF69960A086B
:10A3C0002DE9F74F92460C461A4600218146564623
:10A3D000FFF732FC00258046DFF864B0BAF1000FC9
:10A3E0002CD03146042220464FF07AFC0028424609
:10A3F000484613BF0121002101270027FFF71CFC5D
:10A40000738880465A46019339463AF825304846C3
:10A4100000932B46FFF7C4FD63885A4639464846E9
:10A420000193043634F8043B00932B460135FFF7C3
:10A4300037FB042DD2D103B0BDE8F08F5746EBE7D0
:10A440007D960A082DE9F04F8FB089461746002106
:10A450001A4606460024FFF7EFFB0DF1240B0546D4
:10A46000DFF86CA059F82480594602A8CDF808807E
:10A4700043F03EF84FB357F824302A46304698450B
:10A48000039313BF012100214FF001084FF0000892
:10A49000FFF7D2FB04A9054603A843F029F804A955
:10A4A00023465246009130464146FFF779FD234648
:10A4B0000134524641463046CDF800B0FFF7F0FA7D
:10A4C000202CCFD10FB0BDE8F08FB846EFE700BF2A
:10A4D0008E960A082DE9F04F924685B00C461A4632
:10A4E000002181465546FFF7A7FB00268046DFF88E
:10A4F0006CB0BAF1000F2FD02946042220464FF04D
:10A50000EFFB00284246484613BF012100210127E6
:10A510000027FFF791FBEB7880465A4602933946B5
:10A52000AB78484601932B8800933346FFF738FDFC
:10A53000E3785A463946484602930435A378019396
:10A5400034F8043B009333460136FFF7A9FA102E86
:10A55000CFD105B0BDE8F08F5746E9E798960A08D5
:10A560002DE9F04F85B014461A46054602910021A8
:10A57000FFF762FB4FF00008064606234FF0000984
:10A5800003FB08F7C037029B13F807B0002C7AD002
:10A59000E35D324628469B45039313BF012100210A
:10A5A0004FF0010A4FF0000AFFF746FB039B0646F7
:10A5B000374A51462846CDE900934346FFF7F0FC61
:10A5C0004346334A514628460137CDE9009B09F1FD
:10A5D0000109FFF765FAB9F1060FD4D108F10108B6
:10A5E000B8F1060FC9D1E427029BA7F1E40913F8DB
:10A5F00007A0002C49D014F807B032462846DA45A7
:10A600000DBF4FF001084FF0000801210021FFF7B6
:10A6100013FB062306461E4A41462846CDE9009B09
:10A62000FFF7BEFC01370623194A41462846CDE90B
:10A63000009AFFF735FAEF2FD6D1029B93F8EF700F
:10A64000ACB194F8EF8032462846474513BF01214C
:10A65000002101240024FFF7EFFA00230C4A2146D1
:10A66000009328460723CDF80480FFF799FC0023C8
:10A67000074A21462846009307230197FFF710FA5F
:10A6800005B0BDE8F08FA2469AE7A046CAE700BF32
:10A69000AA960A082DE9F04F0E46154689B01A46CB
:10A6A00000210446B046FFF7C7FA2F4681464FF017
:10A6B000000B002D7AD039460C2240464FF010FB9B
:10A6C00000284A46204613BF012100214FF0010A0D
:10A6D0004FF0000AFFF7B0FA97F90B2081465B466E
:10A6E0000492514697F90A2020460392B7F90820B0
:10A6F0000292B7F906200192B7F904200092364A77
:10A70000FFF74EFC98F90B205B460BF1010B51460D
:10A710000492204698F90A200C3708F10C0803929D
:10A7200038F9042C029238F9062C019238F9082CD9
:10A730000092294AFFF7B4F9BBF1080FB9D14FF0E5
:10A74000000BDFF898800C2303FB0BF985B300277F
:10A7500055F80900012356F8092003FA07FA424088
:10A760003AEA020214BF1946002110EA0A0F07D084
:10A770005B464246204600970791FFF711FC079978
:10A7800056F809201AEA020F05D05B4642462046D9
:10A790000097FFF785F901370E2FD9D10BF1010B87
:10A7A000BBF1080FCFD109B0BDE8F08FAA46A9E7E9
:10A7B0002F46012356F8091003FA07F20A4206D081
:10A7C0005B464246012120460097FFF769F90137B1
:10A7D0000E2FEED1E2E700BFBE960A08D6960A0811
:10A7E0002DE9F04F89468DB0164600211A460746DE
:10A7F0000024FFF721FADFF8DCA00546C4EBC40310
:10A8000009EB030259F80300918840F30748927955
:10A810000890ADF824108DF82620B8F1000F53D021
:10A82000002E54D0F218F0589188937907220A909C
:10A8300008A8ADF82C100AA98DF82E304FF050FA68
:10A8400000282A46384613BF012100214FF0010B92
:10A850004FF0000BFFF7F0F99DF82E3005465246F9
:10A86000069359469DF92D30384605939DF92C30B5
:10A8700004939DF82B3003939DF92A3002939DF8A1
:10A88000293001939DF8283000932346FFF788FB79
:10A890009DF8263052465946384606939DF9253094
:10A8A00005939DF9243004939DF82330CDE902836C
:10A8B0009DF8213001939DF8203000932346013408
:10A8C000FFF7EEF8102C99D10DB0BDE8F08FB3462C
:10A8D000DEE700BFEB960A082DE9F04F924600260E
:10A8E00089B04FF019095546B3464FF461780C46CC
:10A8F0001A4600210746FFF79FF90790BAF1000FAB
:10A9000027D02946062220464FF0EAF90028079A68
:10A91000384613BF012100214FF0010B4FF0000B0F
:10A92000FFF78AF96A790790334619FB0282594684
:10A93000384605922A7919FB02820492EA7803923A
:10A94000AA7802926A7801922A780092104AFFF758
:10A9500027FB627933460136594619FB0282384695
:10A9600006350592227919FB02820492E27803925D
:10A97000A27802926278019214F8062B0092044A9F
:10A98000FFF78EF80A2EB9D109B0BDE8F08F00BFED
:10A9900008970A082DE9F04F14468BB00F461A4667
:10A9A00000210646FFF748F90546002C00F0D78045
:10A9B00022783B789A42024630460DBF4FF001089C
:10A9C0004FF0000801210021FFF736F923780546F2
:10A9D0009B4A41463046FFF7E3FA3B784146984AA6
:10A9E0003046FFF75DF8002C00F0BB8062783046FF
:10A9F0007B789A422A460DBF4FF001084FF00008BD
:10AA000001210021FFF718F9637805468D4A414678
:10AA10003046FFF7C5FA7B7841468A4A3046FFF751
:10AA20003FF807F1C90307F1020A04F1CA0B0593C5
:10AA3000A31C4FF000090693822307933B784B45F4
:10AA400000F39180002C00F0F58097F8EA30304652
:10AA500094F8EA209A422A460DBF4FF001084FF0C1
:10AA6000000801210021FFF7E7F894F8EA300546D5
:10AA7000754A41463046FFF793FA97F8EA30414667
:10AA8000714A3046FFF70CF8002C00F0D58004F135
:10AA9000EA0307F1EA0204F1FA014FF0010833F882
:10AAA00002CF32F8020F844518BF4FF000089942D8
:10AAB000F5D188F001012A463046C9B2FFF7BCF84B
:10AAC0000821054604F1EC00FDF7E4FB5F4A03466C
:10AAD00041463046FFF764FA97F8EA1007F1EC00B8
:10AAE000FDF7D8FB594A034641463046FEF7D8FFEA
:10AAF000002C00F0A3804FF0FC094FF0010807EB99
:10AB0000090104EB0900FCF7ABFB09F1040900287B
:10AB100018BF4FF00008B9F58E7FF0D188F0010121
:10AB20002A463046C9B2FFF787F8082104F1FC0035
:10AB3000FCF7EDFE464A034641463046FFF730FA41
:10AB400097F8EA1007F1FC00FCF7E1FE404A0346E3
:10AB5000414630460BB0BDE8F04FFEF7A1BFA0461E
:10AB60003BE7A04657E7079BFB180993002C5FD0F3
:10AB7000079B0998E31819460893FCF771FB059B9E
:10AB80005A789BF800309A424FD1B0FA80F84FEAD9
:10AB90005818069AAAF102030AF10E01023A33F894
:10ABA00002CF32F8020F844518BF4FF000088B42E5
:10ABB000F5D188F001012A463046C9B2FFF73CF8CA
:10ABC0006278069905469BF81800FDF735FB029060
:10ABD0009BF8003041461F4A30460193089B009382
:10ABE00009F10103FFF7DCF9059B51467A7809F179
:10ABF0000109587E0AF1100AFDF71EFB059A029022
:10AC0000414612F8013F30460BF1010B0193099BBD
:10AC1000059200934B460F4AFEF742FF069B103306
:10AC20000693079B0933079308E74FF00008B0E746
:10AC3000A046D9E7A04620E7A0464DE7A0467FE71B
:10AC400021970A0833970A0861970A0879970A0832
:10AC500090970A0848970A082DE9F04F0F4690464A
:10AC600089B0002187EA08080646139A0025039355
:10AC7000FEF7E2FFDFF884906FEA080304460693CC
:10AC800028460CF0B3FF129B184230D0069BDFF829
:10AC900070B0034014BF4FF0010A4FF0000A049354
:10ACA00010EA070328460CBF4A465A460593079206
:10ACB0000CF0AEFF039B8046079A51460090304649
:10ACC000FFF76EF9049B22463046B3FA83F1490937
:10ACD000FEF7B2FF059A0446039B002A0CBF5A46B2
:10ACE0004A4651463046CDF80080FEF7D9FE013580
:10ACF000172DC5D109B0BDE8F08F00BFA7970A088E
:10AD000077960A082DE9F04F3B4C89B00A4600219E
:10AD10000546FEF791FF059094F900000AF08AFAC3
:10AD2000814660883DF062FE344BD0F808B01F7851
:10AD300017B15F46D0F80CB0A3790026012B38BFBD
:10AD4000012306932279637906FB02331BF8038003
:10AD5000002F3AD0FB5C4345059A2846079313BF62
:10AD6000012100214FF0010A4FF0000AFEF764FFB5
:10AD7000079B0136059053B303F00F021B095146A0
:10AD80002846403302921E4ACDE900634B46FFF746
:10AD900007F9B8F1000F24D008F00F034FEA181894
:10ADA000174A5146029308F140032846CDE9006353
:10ADB0004B46FEF775FE069BB342C3DC0834114BCD
:10ADC000A342A9D109B0BDE8F08F3B46C3E7002FED
:10ADD000DFD04B460C4A514628460096FFF7E0F874
:10ADE000D7E76B06E7D44B46074A514628460096FC
:10ADF000FEF756FEDFE700BF68BD0908585D002476
:10AE0000AE970A0870BE0908C4970A080FB407B5C0
:10AE100004A951F8040B0191FEF724FE03B05DF87C
:10AE200004EB04B070472DE9F041037903F0E00230
:10AE3000402A4DD009D83ABB03F00703052B1ED892
:10AE4000DFE803F0181D181D0910602A47D0802A7A
:10AE500041D0BDE8F081D0F805102348BDE8F041AD
:10AE6000FEF732BED0F8052051422048BDE8F0413F
:10AE7000FEF72ABEB0F80720B0F80510F5E7B0F9E4
:10AE80000720B0F90510F0E746790024184D19485D
:10AE900005EBC605FEF7F8FD012395F8F072A74211
:10AEA00003D8BDE8F041FEF7F7BDD5F8EC624FEAF4
:10AEB000840856F824204AB113B90F48FEF7E4FD80
:10AEC00056F808100D48FFF7A1FF00230134E6E70C
:10AED00041790B48C2E7827941790A48C6E70A48B6
:10AEE000BDE8F041FEF7F0BDD8970A08EE970A08D2
:10AEF00084BB090805980A0880990A087DAE0A08EB
:10AF000016980A0827980A083E980A08194B1B68E1
:10AF10002DE9F0415BB30025174FDFF86880174833
:10AF2000FEF722FEFEF794FDFBF79CFBFBF7DAFB36
:10AF3000044648B113200FF025FFFEF7ADFD104881
:10AF4000BDE8F041FEF710BE3B78012BF2D0404641
:10AF50006E1CFFF75BFF792D02D12646FEF79CFDA4
:10AF6000FEF776FD64203546FBF70AF9DEE7BDE81B
:10AF7000F08100BFE02200245630002456980A08D1
:10AF800070980A0847AF0A08BD4B42F201011A68DF
:10AF9000B1EB124F4FEA12432DE9F04F91B000F0A0
:10AFA000F58142F20302934200F0F28141F2030282
:10AFB000981A43424341B34A0025B34E116806EB49
:10AFC000C303B24AB24CB348B34F04F5126BDFF877
:10AFD0008483B946DFF880A3B1FBF2F2D3F8A8145A
:10AFE000FFF714FFB4F818294FF47A730A20B2FB64
:10AFF000F3F103FB1122B4F91A3992B2B2FBF0F269
:10B00000A648FEF761FDA64AA649A748FFF7FEFE3F
:10B01000FEF742FDA54BA64A997BA64B06EB8101A4
:10B02000A548D31AB4F80A28D1F8C414FEF74CFD89
:10B03000FEF732FDA148FEF727FD94F81C19A04841
:10B04000FFF7E4FE9F48FEF71FFD9F4B94F81D1984
:10B050001A889E4892B2FFF7D9FEFEF71DFD9C4963
:10B060009C48FFF7D3FE2B4698F81F202A41D107B2
:10B070002ED513B19848FEF707FD691C5046FFF71F
:10B08000C5FE15F80B30954806EB8303D3F8CC14B6
:10B09000FFF7BCFE99F86A352B41DA0702D59048D4
:10B0A000FFF7B4FE97F81831032B09D08D48FFF74E
:10B0B000ADFE97F81831012B02D18B48FFF7A6FEA1
:10B0C000FB6C5B7B012B02D98848FFF79FFE0123B5
:10B0D00007F5CE77002D00F05D81002B40F05C81FC
:10B0E0008348FEF741FD834FD4F82489DFF86C9242
:10B0F00007F1180A0123AB4013EA080F15D019F81D
:10B10000052057F825305AF8251053F822207A48A0
:10B11000FFF77CFE012D06D1784B93F8211011B179
:10B120007748FFF773FEFEF7B7FC0135062DE1D136
:10B130007448FEF7A9FC744B1B681B0640F1608144
:10B1400094F84439032B8CBF70487148FEF79CFC7F
:10B1500094F88835022B40F022816E48FEF794FC6B
:10B1600094F84439042B00F242816B48FEF78CFCC2
:10B1700094F85439002B00F0418106EBC303D3F857
:10B1800060156648FFF742FEFEF786FC644B654893
:10B190001D68654B1B7806EB8303D3F89415FFF706
:10B1A00035FE25B12A7A697A6048FFF72FFEFEF74F
:10B1B00073FCFBF721FA016921B182685C48120D2A
:10B1C000FEF782FCFEF768FC5A4B5B4819684FF4A7
:10B1D0007A73B1FBF3F1FFF719FE05A8FDF7C6FA84
:10B1E00038B105A908A84CF067F908A95348FFF73A
:10B1F0000DFEFEF751FCD4F8E079002F00F0048139
:10B2000007EE907ADFED4E6AB8EEE77AC6EE877AFF
:10B21000FDEEE77A17EE903A4A4D15F8600C30B122
:10B22000494A039392ED310A4DF0D0FE039BD4F8C6
:10B2300060495CB107EE904ADFED416AF8EEE77ACB
:10B2400086EEA77AFDEEC77A17EE904A2B4AB2F83F
:10B2500070103A466429CDE90004A8BF64213B4838
:10B26000FEF732FC35F85C2C64233948B2FBF3F16D
:10B2700003FB112215F84B3C06EB830670E000BF80
:10B280000010005CA004002484BB090840420F00A9
:10B29000585D00247E980A08A01D002090980A0896
:10B2A000F8FF012000080000B2980A083835002491
:10B2B0000000040800000208C4980A08DB980A0885
:10B2C000ED980A08F5980A08B8250024F7980A08A6
:10B2D0000B990A0810990A0880990A08AA990A087D
:10B2E0007B9E0A081A990A0822990A0827990A08CF
:10B2F0002F990A08B0C00908A2A60A080035002044
:10B3000034990A0838990A08683500243E990A08D1
:10B310004A990A085A990A0858B00A089E990A08D0
:10B32000B03A0024BA990A08AC3A0024C3990A0832
:10B33000CD990A0818230024E8990A08029A0A08F5
:10B3400000247449506E0024C8050024159A0A0888
:10B350005B9A0A080037002415990A08840600241D
:10B3600092B2D6F8A835314E009315F84C3C012521
:10B37000FEF7AAFB2E48FEF787FB2E4B1C68002C1D
:10B3800044D1FEF789FB11B0BDE8F08F022312E62D
:10B39000032310E6012567E6FEF77EFBA3E6022005
:10B3A0000FF0A4FB054608B92348D7E690F904003E
:10B3B00042F0EEF8074632F093FC06EB8000394687
:10B3C000D0F8A4211D48FFF721FD94F88B35012BFF
:10B3D00004D11B48FEF758FB1A48BFE6AB791A4860
:10B3E00006EB8303D3F8A411FFF710FDF4E794F8FC
:10B3F0008A350BB91548B9E61548B7E61549C0E6D0
:10B400001548FEF741FBBFE63B4605E794FAA4F07A
:10B41000B0FA80F005FA00F024EA00040CF0CEFB4C
:10B4200001463046FFF7F2FCA9E700BFAA990A08D7
:10B43000809A0A08B036002460990A086A990A08B6
:10B440007A990A087F990A0842960A0883990A0895
:10B4500093990A0876980A08AE990A082DE9F04FE0
:10B46000DFF86C8199B098F80330002B00F09380DE
:10B470004E4800254E4EDFF85CB1FEF775FB2F46B7
:10B48000DFF85491DFF854A10BA9E8B216F0D2FE10
:10B490009DF83430002B53D0139C54B107EE904AE2
:10B4A0009FED440AF8EE677A80EE270A4DF08EFD94
:10B4B00004460B9A29465846FFF7A8FC109A002A22
:10B4C0006BD002FB04F04FF47A73B0FBF3F30993F3
:10B4D000DDF848C0BCF1000F61D00CFB04F142F272
:10B4E0001073B1FBF3F1082D98F8033018BF7F18E3
:10B4F000002B56D017984FF47A7E0A2307901598A0
:10B500000690169805901198B0FBFEFECDF810E05D
:10B510000998B1FBF3FE03FB1E11CDE902E1099985
:10B52000B1FBF3F103FB1100BCFBF3F3CDE9001019
:10B5300021465046FEF7C8FA0023B362C6E90D3330
:10B54000013540361D2D9FD198F8033003B31A4CB6
:10B550004FF47A73194854E91212B1FBF3F3D2088D
:10B5600054F8401CFEF7B0FA0A22154897FBF2F196
:10B5700002FB1172FEF7A8FA124B1B78432B04D181
:10B58000114854E90F21FEF79FFA002344F8403C8C
:10B5900019B0BDE8F08F0D486BE7099298E7614656
:10B5A000A1E721464846FEF78FFAC5E7969A0A08B2
:10B5B000B06600248096184B506E00243D9B0A080C
:10B5C0005D9B0A0800300024819B0A08F49A0A084F
:10B5D00038350024FE9A0A08299E0A080D9B0A089D
:10B5E00010B5114B86B0114904460493104B114815
:10B5F0000393114B114A0293114B0193114B00938A
:10B60000114BFFF703FCFEF747FA10491048FEF70D
:10B610005BFA3CB10F4A1049104806B0BDE8104033
:10B62000FEF752BA06B010BDEB9B0A08B59B0A089C
:10B63000F09B0A08C09B0A08FB9B0A08AB9B0A0800
:10B64000049C0A08109C0A083F3500241A9C0A082A
:10B65000229C0A08339C0A08419C0A08469C0A0856
:10B660000120BDE7234870B5FEF70EFA224B13F810
:10B67000603C002B38D0214B93ED310A4DF0A6FCF5
:10B6800001461F48FEF720FA1E4C1F48FEF7FCF942
:10B690001E4B94F8F5041E4A00280CBF10461846AD
:10B6A000FEF762FA94F8F53413B31A4C1A48B4F85A
:10B6B0000611FFF7ABFB194E94F80401184D002852
:10B6C0000CBF30462846FEF74FFAB4F8081115486B
:10B6D000FFF79CFB94F8050100280CBF3046284674
:10B6E000BDE87040FEF740BA0F48FEF73DFACBE7E1
:10B6F00070BD00BF839C0A08506E0024C80500245A
:10B700009D9C0A08585D0024AC9C0A0853980A08BE
:10B710001CB50A0800350020BD9C0A087C9C0A085C
:10B72000739C0A08E49C0A08A29C0A0838B50B4DD1
:10B730000C4605EBC00595F9E40109F07BFD0146D7
:10B740000748FFF763FB95F8EA3133B1611C054800
:10B75000C9B2BDE83840FFF759BB38BD84BB090802
:10B760007DAE0A0801980A086B4B1B782DE9F04F53
:10B7700087B0002B00F0CA80684D4FF00008684881
:10B78000A968FEF7A1F969686648FEF79DF9664B5E
:10B790006648D3E90031C91A654B1A68B1FBF2F269
:10B7A000FEF792F9FEF778F96248FEF7DDF9624894
:10B7B000FEF7DAF9614B5FFA88F41B78A34221D8CF
:10B7C0005F4D00245F4EFEF767F9013455F8041F02
:10B7D0003046FFF71BFB162CF7D15B4D0124594E69
:10B7E000FEF75AF92B466968013430461B68043568
:10B7F000C91AFFF70BFB162CF4D107B0BDE8F04FC8
:10B80000FEF74AB9514B14264FF03C0B671C03EB73
:10B81000840306FB045693ED450A4DF0D7FB96F8DA
:10B820001EA081B2B6F80E901AF0010F80B20CBFC4
:10B830002D2252221AF0020F049045480CBF2D23EE
:10B8400054231AF0040FB1FBFBF10CBF4FF02D0C89
:10B850004FF0560C1AF0080F05914FF064010CBF21
:10B860004FF02D0E4FF0430E1AF0800F01FB09F13F
:10B870000CBF4FF02D0A4FF0530ACDE900CECDE9B1
:10B8800002A13946FFF7C2FAB37FDB073AD55C2342
:10B89000304A6343D118D05891ED010A70B1B8EE27
:10B8A000400ADFED2D7A20EE270A07EE900AF8EE27
:10B8B000677A80EE270A4DF089FB00B2642290FB84
:10B8C000F2F102FB11022548FFF7A0FA14212448E7
:10B8D00008F1010801FB075701FB0454F988628A4B
:10B8E0000491218B02F0030392080391E18A0291F3
:10B8F000A18B0191A18A009119214B43218AFEF766
:10B90000E3F857E71748FEF7BFF8DFE7164807B038
:10B91000BDE8F04FFEF728B904000020341B0020DA
:10B92000049D0A08149D0A083C1C00202B9D0A084F
:10B93000C0230024589D0A08B49D0A08481C002012
:10B94000DC1B0020649E0A08E01B0020003500205C
:10B95000109E0A085418002000401C462D9E0A081C
:10B96000429E0A08399E0A08689E0A080EB403B56A
:10B9700003AA52F8041B0192FCF71BFC064BD3F8F8
:10B9800014291AB90549986CFBF748FF02B05DF815
:10B9900004EB03B0704700BF585D0024C7A90A0834
:10B9A0002DE9F04798460B7981460F4603F0E005F4
:10B9B0001646402D32D10024634DDFF8A881DFF810
:10B9C000B09116E03B7903F00703013B042B04D848
:10B9D000DFE803F014171A1D2100315D5A48FFF704
:10B9E00015FA7B79013BA34202DD4846FEF74CF88D
:10B9F00001347B79A342E5DCBDE8F0873157284666
:10BA0000EDE736F81410FAE736F91410F7E756F8B0
:10BA100024104046E3E756F82410F0E703F007034C
:10BA2000052B57D8DFE803F0031F27292C3E347875
:10BA3000602D55D02CD8002D75D1B7F80550B7F82A
:10BA4000076021464048FFF7E1F9AC4239DBB442D8
:10BA500037DCB8F1000FCFD0324629463B48BDE86D
:10BA6000F047FFF7D3B996F90040602D38D00FD8D2
:10BA7000002D58D151E03488DAE7B6F90040F4E7F8
:10BA8000D6F800A0202D54464DD034D9602D27D0B3
:10BA9000802DB1D132782E4B2E48002A14BF31466A
:10BAA000194635E0202D34683DD0EFD82146264890
:10BAB000FFF7ACF9D7F80510A14202DB4B42A342D5
:10BAC00021DDFDF7E9FF23463A6848462249BDE8F3
:10BAD000F0474BE7202D25D01ED9602DD8D100246A
:10BAE0007B7944FA03F3DB07BDE8F0474CBF1B4802
:10BAF0001B48FFF78BB951461A48FFF787F9D7F86B
:10BB000005108A45DDD8B8F1000F3FF475AF16482F
:10BB1000BDE8F047FFF77AB90024B7F90550B7F947
:10BB200007608EE700247A79104B03EBC20393F889
:10BB3000F022A242C5DDD3F8EC3253F82400BDE870
:10BB4000F047FDF7A1BF00BF02980A0801970A0855
:10BB500020B00A087DAE0A088A9E0A0853980A088F
:10BB60001CB50A08EB970A08849E0A0884BB0908DA
:10BB7000F5980A082DE9F04F164685B0334C1A4661
:10BB80004FF00009A246CDE9010100213046FEF741
:10BB900053F806F0100300900393FDF759FF237943
:10BBA000029A03F01803934203D0002A44D1182BC1
:10BBB00042D14FF00D0B0BFB09A3B3F809003CF089
:10BBC00015FF80462046FBF72BFD0746D8E90221EA
:10BBD000024401442046FBF7BBFC80F0010105460E
:10BBE000009AC9B23046FEF727F8039B009003B1D4
:10BBF00015BB0BFB09FBB3065AF80BB00ED56DB99C
:10BC000059461348FFF702F9D8F808202B46214679
:10BC10003A440198FFF7C4FEFDF73EFF59460D4830
:10BC2000FFF7F4F8D8F80C20002321463A44019895
:10BC3000FFF7B6FEFDF730FF09F1010940F263237B
:10BC40000D349945A9D105B0BDE8F08F5CCA09084B
:10BC5000A49E0A08A59E0A0870B5164605460C461D
:10BC60000846FBF7EBFD3346024621462846BDE871
:10BC7000704095E60EB403B503AA52F8041B019276
:10BC8000FCF797FA044B0549986CFBF7C7FD02B027
:10BC90005DF804EB03B07047585D0024C7A90A089B
:10BCA0000049E7E7AF9E0A0838B50C460546154936
:10BCB0002046FBF7D5FA30B9FDF7A0FE1248BDE8E3
:10BCC0003840FDF751BF11492046FBF7C9FAA8B922
:10BCD0000F4B83F8B90183F8C10183F8A30283F8FD
:10BCE000AB0283F88D0383F8950383F8770483F818
:10BCF0007F04084B83F821000748E0E72846BDE8A9
:10BD00003840CDE7BE9E0A08C49E0A08DF9E0A0896
:10BD1000585D002400370024E79E0A080049A9E77F
:10BD2000039F0A08F8B50C4606460846FCF752FC85
:10BD30002021054620464DF096FE044618B93046AF
:10BD4000BDE8F840EAE7114F0134114E3B783278F4
:10BD50009A4201D0FAF712FE0E4B20461D604BF0BE
:10BD6000FBFD012201462046FAF7A6FD3B7832781A
:10BD70009A4201D0FAF702FE20464BF0EDFD2A462A
:10BD800001460548BDE8F840FDF79EBEDC220024D0
:10BD900057300024D82200241A9F0A082DE9F041C8
:10BDA0000D4688B006460846FCF714FC20210446E0
:10BDB00028464DF058FE20B9304608B0BDE8F041A5
:10BDC000ACE7FCF707FC2246054601460F48FDF7A5
:10BDD0007BFE85B1202D2A466946204628BF2022B9
:10BDE000E846FAF713FE00270646B74208DBAD1B0C
:10BDF0003444002EEDD1FDF74FFE08B0BDE8F081D0
:10BE000018F8010B0137FEF7C1F8EEE7309F0A087A
:10BE10002DE9FF47074608460D464BF09DFD0828D3
:10BE200046D105F1FF3801AE073531464246B146ED
:10BE300012F8010FFCF7DCFA01F8010BAA42F7D166
:10BE40000023DFF880A08DF80C30A84518D11C49DC
:10BE5000484624F069F81A4808231A4910F8012BBB
:10BE6000013B11F8014B02F110026A4402F80C4C3C
:10BE7000F4D101A914488DF80C30FDF725FE14E02B
:10BE800018F8010FFCF7B4FA0446014606F8010B56
:10BE900050464DF0E8FD28B1214630464DF0E3FD17
:10BEA0000028D2D03846FFF7FBFE04B0BDE8F0878B
:10BEB0000028D0D0384604B0BDE8F0472EE700BFD8
:10BEC0002C62002440330A08489F0A0807B50093F3
:10BED00013460A460249FFF7CDFE03B05DF804FBA6
:10BEE0004F9F0A082DE9F04F06468BB00D46DFF84C
:10BEF000908228464BF030FD034638B902469249FD
:10BF000001200BB0BDE8F04FFEF76ABC05228F4957
:10BF10002846FCF773FA044698B98D4D0146702205
:10BF2000A5F134004DF088FDEC63AC646C652C66C3
:10BF3000EC66AC67C5F88440C5F890400BB0BDE82E
:10BF4000F08F042241462846FCF758FA044628BBE5
:10BF50002846FBF7CAFC81460028EFD04BF0FCFCDA
:10BF6000DFF820B282465BF8047B37B92A4679496C
:10BF700030460BB0BDE8F04F7CE6524639464846A5
:10BF8000FCF73CFA40B92046734D22F05BFF39467E
:10BF90007248FDF799FDACE70134E4E707227049E8
:10BFA0002846FCF72BFA0746002877D1202128469F
:10BFB0004DF059FD044670BB6A4D6B48FEF726FFF5
:10BFC000214601342846FEF721FF0E2CF8D100252A
:10BFD000DFF8B491654FFDF75FFDDFF8B0810C2607
:10BFE0000024DFF8ACA129466E434846FEF70EFF59
:10BFF0000123F2595E48A340013413420CBF41466D
:10C000005146FEF703FF0E2CF2D10135FDF744FD3A
:10C01000082DE4D192E702AC564D01AA55494DF0E6
:10C02000E8FC002845D0022F11D1029A072A07D830
:10C03000039C0D2C04D80378722B13D06E2B23D0C5
:10C04000082300224C493046FFF740FF76E7FCF713
:10C05000C1FA01AA44F8040B2946002001374DF02B
:10C06000C8FCDEE70C233A4903FB02110123C96B2C
:10C07000A3400B4336490C2000FB02123849D3631E
:10C080003046FFF72FFF59E7314B0C20012100FB11
:10C090000233A140DB6B23EA0103EBE728460024CF
:10C0A00002AD344F01AA33494DF0A3FC80B1082CF6
:10C0B00003D13046FFF732FE40E7FCF78BFA01AAC6
:10C0C00045F8040B3946002001344DF092FCEDE7B1
:10C0D000082CEED1029B0F2B30D8DDF80CE0BEF11E
:10C0E000070F2BD8DDF810C0BCF10D0F26D8059F27
:10C0F00007F16402C82A21D8069DFF2D1ED8079893
:10C1000064281BD80899642918D8884216DA099C33
:10C11000032C13D8C3EBC3020D4B134403F82F1C9D
:10C1200003F834EC0C4903F833CC03F8327C03F801
:10C13000315C03F8300C03F82E4CA1E70F49304670
:10C14000FFF798FDFAE600BF1C6E0024689F0A08FE
:10C15000506E0024739F0A08C9A90A08849F0A0820
:10C160008E9F0A08969F0A087EAE0A088C6E0024ED
:10C170009B9F0A089F9F0A08A19F0A08A79F0A0879
:10C180006E9F0A0840C1090802980A0856AE0A08BC
:10C19000E9960A0810B504460748FDF7E5FCFAF7EA
:10C1A00021FF20B10548BDE81040FDF7DDBC204669
:10C1B0000349BDE810405DE5BD9F0A08C79F0A0816
:10C1C000CF9F0A082DE9F04F8FB004460846B249C8
:10C1D00002AA4DF00EFC054640B903460246AF499F
:10C1E0004120FEF7D7FB0FB0BDE8F08FAC49FBF75D
:10C1F00037F8064628BB02AAA7494DF0FAFBFCF720
:10C20000E9F90828054606D908233246A5492046FB
:10C21000FFF75CFEE7E7A44C94F8E43683420CDCBD
:10C2200084F8E456DFE731460136384630F02CFF1B
:10C2300094F8E436B342F6DCF2E7064604F2E4672B
:10C24000F6E79A492846FBF70BF80646E0B902AA3A
:10C2500091494DF0CEFBFCF7BDF90828054603D9FE
:10C26000082332469249D2E78F4C94F8E536834250
:10C2700002DC84F8E556B6E730460136294641F03F
:10C2800055F8082EF8D1F4E78A492846FAF7E8FF6E
:10C29000064600BB02AA80494DF0ABFB0028A2D0A5
:10C2A000FCF798F90828054603D908233246824945
:10C2B000ADE77D4C94F8CE37834209DD014604F2A8
:10C2C000E46030F027FF294604F2E46030F030FFEC
:10C2D00084F8CE5787E779492846FAF7C1FF064622
:10C2E00018BB06AD704BDFF8B0910146A84610228E
:10C2F000284693F8CE774DF09FFBBE4202AA80F20B
:10C300000A81494600204DF074FB10B93A466C4949
:10C310000AE1FCF75FF9013628F8020BEDE7694CFA
:10C3200095E80F0084E80F005DE767492846FAF7B3
:10C3300097FF0646C0BB5C4B06ADDFF85C9193F8F7
:10C34000CE77BE4202AA80F2F380494600204DF02B
:10C3500050FB014610B93A465C49E5E0AA464FF069
:10C360000008032228464DF069FC28464BF0F4FAF9
:10C37000404502D801360435E3E79AF8000008F199
:10C380000108FCF735F80AF8010BEEE7B6000446A1
:10C390004F4DB4423FF427AF06AB281903221919B9
:10C3A000043430F05BFEF4E74A492846FAF758FFB8
:10C3B0000746002840F0AC80DFF8EC8002AA36493E
:10C3C00098F8E4664DF015FB00283FF40CAFFCF73D
:10C3D00001F9451E01D4AE4203DC334601223E4939
:10C3E00015E72D4902AA00204DF003FB0146002865
:10C3F0003FF4F9AE00260DF10C09082203A88DF8D0
:10C4000014604DF01BFC03A84BF0A6FAB0421BD8F9
:10C4100002AA214900204DF0ECFA00283FF4E3AED7
:10C420000026037898F8E5A6B1460193564502AA7E
:10C4300019494FF0000080F285804DF0DAFA83460A
:10C4400050B9524625496FE099F800000136FBF7D4
:10C45000CFFF09F8010BD6E7A6B99BF80030303BB7
:10C46000092B0FD91E49FAF7FBFE38B11D49584672
:10C47000FAF7F6FE70B15A461B4955E04FF0010934
:10C480004FF0FF365846FCF7A5F8002830DA5A4638
:10C49000164949E0B146F3E79F9F0A083C6400242F
:10C4A000D69F0A08DC9F0A08585D0024E79F0A0807
:10C4B000F09F0A08FE9F0A080AA00A081CA00A08A2
:10C4C0000BA10A082865002446A00A082BA10A0827
:10C4D0003865002470A00A0875A00A084BA10A0854
:10C4E000B5940A0881A00A0888A00A08BDA00A0815
:10C4F0000EAB03EB4603013623F8200C96E75246B9
:10C500001F4911E033F8022B013724F8022F30E0E5
:10C510002A461C4908E01C4900204DF06AFA002810
:10C520003FF4FDAE3A4619492046FFF7A3FB5AE611
:10C53000154900204DF05DFA00283FF427AF3A4638
:10C540001349F1E74DF055FA0028D8D105EBC500A5
:10C55000104C082203A98230204404EB051430F06B
:10C560007DFD0198FBF744FF08EB050383F8AE0758
:10C5700006ABBE42C6DC454485F8C69733E600BF2D
:10C58000D2A00A08F5A00A089F9F0A0828A00A0856
:10C5900052A00A083C640024154B1B682DE9F041A9
:10C5A000044688B0F3B11A6804A91846D56A6A46E9
:10C5B000A847064688B104AC6D460027DFF83C80EA
:10C5C000013735F8022B34F8021B4046FDF77CFAA0
:10C5D000BE42F5DC08B0BDE8F08106492046FFF711
:10C5E00049FBF7E7044908B0BDE8F041FFF742BB5B
:10C5F000303700248AA10A08A2A10A0870A10A08FB
:10C6000070B5054608460C464BF0A6F9024670B1D7
:10C610000D2804D1214609484DF0FEFA38B12846CC
:10C62000064B074A0749BDE87040FFF723BB0349A3
:10C630000548BDE87040FDF747BA00BF339C0A08C3
:10C64000A9A10A08B4A10A08DEA10A0870B5054626
:10C6500008460C464BF080F9024670B1042804D11C
:10C66000214609484DF0D8FA38B12846064B074A0A
:10C670000749BDE87040FFF7FDBA03490548BDE82A
:10C680007040FDF721BA00BF419C0A08ECA10A08DE
:10C69000B4A10A08FCA10A082DE9F04307469BB0A3
:10C6A00008460C464BF058F906462022002101A806
:10C6B0004DF0C2F936B3402E08D0402332463A49F5
:10C6C00038461BB0BDE8F043FFF7D4BA01AD04F122
:10C6D00040084FF000090222214668464DF0AEFAAC
:10C6E0000023102209A968468DF80290FBF7C2FECC
:10C6F000099B0DF10202934223D1023405F8010B8C
:10C70000A045E8D109AC41220021284D20464DF03A
:10C7100093F9002E3CD095F89C60D6B1202205F10B
:10C720009D0101A84DF0DCFA98B105F19D0120466C
:10C73000FBF7D0FD23461E4A38461E49FFF79AFAFA
:10C7400004E01A7838461C49FFF794FA1BB0BDE89C
:10C75000F0831A4B1B78DBB9D6B901AB184E1A46D9
:10C76000083603CAA24246F8080C46F8041C1346D1
:10C77000F5D101232046124985F8BD30FBF7AAFD0B
:10C780001048FDF74DFA21460F48FDF79DF9DDE70A
:10C7900095F8BD301BB995F89C30002BF3D00849B3
:10C7A0002046FBF797FDEEE70FA20A08506E002423
:10C7B0004DA20A08B4A10A0831A20A08585D002453
:10C7C000ED6E002457A20A0866A20A082DE9F74F69
:10C7D000DFF82081834608460C464BF0BDF8D8F8B8
:10C7E0000070064628B1024633492046FBF706FE94
:10C7F00080B93946314840F051FE3149314821EA8B
:10C80000070140F04BFE3049304803B0BDE8F04F1F
:10C8100040F044BE23782D2B24D10134013E4FF04B
:10C82000010A2B4B4FF000094FF0FF3553F8041B62
:10C8300051B1324620460193FBF7E0FD0028019BF1
:10C840000ABF4D460021012109F10109A9B9B9F139
:10C850001D0FEBD122461F49584603B0BDE8F04FEB
:10C86000FFF708BA4FF0000ADBE73B431A49C8F864
:10C8700000301A4B12E01A4913E00123104AAB4072
:10C880001A40002AF7D007EA0302BAF1000FECD0F1
:10C8900027EA03031349C8F80030134B002A18BFD6
:10C8A0001946124B124803EB8503D3F82C2603B02C
:10C8B000BDE8F04FFDF708B9F99A0A089EA20A08E8
:10C8C000BCD45518A8A20A08432BAAE7B4A20A08A8
:10C8D000B0C10908739F0A0896A20A088FA20A0825
:10C8E00073A20A087FA20A0886A20A0884BB090864
:10C8F00077960A08603B00242DE9F74F019008461F
:10C900000E46174698464BF027F80446E8B9404DC6
:10C910004048FEF77BFA20460BF068F93B68184266
:10C9200006D020460BF074F901462846FEF76EFA51
:10C930000134172CEFD13B6813B93748FDF7A4F841
:10C9400003B0BDE8F04FFDF7A7B8024633493046C3
:10C95000FBF754FD0546A8B92C46314D3148FDF78B
:10C9600093F820460BF042F910EA080F06D0204653
:10C970000BF04EF901462846FEF748FA0134182C10
:10C98000EFD1DDE733782D2B29D10136013C01258C
:10C990004FF0000948F4000B48460BF039F92246E5
:10C9A000824601463046FBF729FD18BB48460BF08E
:10C9B0001DF91BEA000F1DD09DB1B9F1170F02D070
:10C9C0003B6840EA03081848C7F80080FDF75CF8A8
:10C9D0005146134803B0BDE8F04FFDF775B8002588
:10C9E000D6E7B9F1170F02D03D6825EA00050F48D8
:10C9F0003D60EBE709F10109B9F1180FCCD13246DE
:10CA00000B49019803B0BDE8F04FFFF733B900BF01
:10CA1000A9990A08C2A20A08CCA20A08F99A0A0827
:10CA2000AA990A08D3A20A0886A20A0896A20A08A6
:10CA3000739F0A0840F20223004A5DE7CC360024C7
:10CA4000014B024A58E700BFFFFF7F00C4360024B5
:10CA500010B50446012023F0DBFA28B92046054929
:10CA6000BDE81040FFF706B90348BDE81040FDF7E8
:10CA70002BB800BFDEA20A08EDA20A08074B10B5CA
:10CA80000446D3F8C00031F0A3F828B92046044981
:10CA9000BDE81040FFF7EEB810BD00BF506E002497
:10CAA000F8A20A0870B5054608461646FBF792FD3F
:10CAB0000D4B041E1A780EDB944205DA21460B4812
:10CAC000FDF702F8204670BD2EB1FF2C03D10848B7
:10CAD000FCF7FAFFF6E7013A064928464FF0FF3423
:10CAE000FFF7C8F8EEE700BF481C00200EA30A08B5
:10CAF0001FA30A0832A30A082DE9F04F074691B098
:10CB000082480E46824DFCF7DFFF00238149402416
:10CB1000062285F8C830304601230978C5F8C4D00C
:10CB200085F8C94007F0DCFE0A20F9F729FB95F8E3
:10CB3000C8300C2BDAB240F2E4809DF80C60FE2E77
:10CB40002CD0FF2E15BF0F2415240025012594425B
:10CB500040F0D780611E6846C9B235F0F9FD04F196
:10CB600040030DEB030414F8413C834240F0C480C1
:10CB70006A1E9DF80D30012A12D903F01F075C09C7
:10CB800061376548FCF780FF022D39D0013C042C49
:10CB900034D8DFE804F00B2D2F3331000225D6E71F
:10CBA0009DF80E701E469DF80F40EAE75B486C4604
:10CBB0004FF00008DFF8BC91FCF7D6FFDFF8B8A112
:10CBC000DFF8B8B15648FCF75FFF08F1010814F828
:10CBD000011B4846FEF71AF9B8F10C0F16D00AFBF4
:10CBE00008F3B3F1553FF0D85846FCF74DFFECE79A
:10CBF0004C48DCE74C48DAE74C48D8E74C48D6E7E5
:10CC000000230DF11F008DF83F30D0E7FCF744FF03
:10CC1000022D3AD064223B464648B6FBF2F102FBB5
:10CC20001162C9B2D2B2FCF74FFF85F001035B423B
:10CC3000DBB2012B59D8404A404B9DF810104048B8
:10CC400000290CBF114619463E4EFCF73DFF9DF8EA
:10CC500011103D4B3D4800290CBF31461946FCF7E9
:10CC600033FF022D41D19DF812403948FCF70CFFEB
:10CC70008CB1FF2C1FD00A233648B4FBF3F103FB21
:10CC80001142D2B2FCF720FF08E03A463146324862
:10CC9000FCF71AFFCFE73046FCF766FF9DF813401C
:10CCA0002E48FCF7F1FE44B1FF2C21D021462C4840
:10CCB000FCF70AFF04E02B48EEE72248FCF754FF9C
:10CCC0000DF1130500241F4E1F4FDFF8988015F853
:10CCD000013F7BB1FF2B14BF3A4642462146013447
:10CCE0002148FCF7F1FE042CF1D111B0BDE8F08F22
:10CCF0001C48E3E73246F1E71C493846FEF7BAFF25
:10CD0000F3E71B48FCF730FFEFE700BF78A30A0802
:10CD1000506E0024481C002089A30A0894A30A0826
:10CD2000BAA30A089BA30A08A3A30A08ABA30A088C
:10CD300076980A08CCA30A0861A30A0858A30A082F
:10CD400003A40A0868A30A0899AD0A081AA40A08E5
:10CD500021A40A0835A40A08E8A30A083DA40A0881
:10CD600002980A086CA30A084DA40A0858A40A08E5
:10CD700068A40A08CB940A08ABAAAAAA20B00A0899
:10CD80002DE9F84307460C46DFF8A09020464AF00C
:10CD9000E3FD064658B91D4B1D481A781D4B03EBA1
:10CDA0008203D3F8B815BDE8F843FCF78DBE024600
:10CDB00049462046FBF722FB60B1DFF86080002582
:10CDC00058F8041BB1B9224638461349BDE8F84368
:10CDD000FEF750BF114C124D1248FCF755FE54F8A7
:10CDE000041B19B12846FEF711F8F8E7BDE8F8432F
:10CDF000FCF752BE324620460135FBF7FFFA002809
:10CE0000DED1024B084C1D70C0E700BFE4350024A2
:10CE100071A40A0884BB0908739F0A0840C1090865
:10CE2000AA990A08D3A20A08C9A90A08F99A0A08FD
:10CE300038B50D460446052219492846FBF7DEFAA7
:10CE400068B9184B93F84C2022B9012183F84D2082
:10CE500083F84C101448BDE83840FCF785BE032227
:10CE600012492846FBF7CAFAA0B90E4D95F84C3086
:10CE700063B195F84D304BB10D492046FEF7FAFEEF
:10CE8000002385F84C3085F84D3038BD0948FCF753
:10CE90006BFEF5E720460849BDE83840FEF7EABEDC
:10CEA000F0AC0A08585D00247BA40A0842AE0A08C8
:10CEB00091A40A08C8A40A08DCA40A0870B5194C91
:10CEC000054694F84C307BB194F84D3063B1164967
:10CED000FEF7D0FE28461549FEF7CCFE002084F868
:10CEE0004C0084F84D0070BD114B93F8BD20B2B1D9
:10CEF00093F89C209AB903F19D0203F1CC0503F14C
:10CF0000BD061068083252F8041C2C46B24203C415
:10CF10002546F6D1012283F8072109F0CDFF012033
:10CF2000E1E700BF585D002491A40A08EBA40A08B9
:10CF3000506E00242DE9F04F80468BB008460D4618
:10CF40004AF00AFD0246A8B3A5492846FBF756FA5F
:10CF5000044678BBFCF7A0FDA24DA348A34EFCF706
:10CF600003FEA34F1420DFF8CC8240F0F3F9E11068
:10CF7000304604F007020131FDF748FF95F81D9097
:10CF800095F91C00B9F1000F0DD008F053F94A468D
:10CF900001464046FCF798FD01342435102CE6D1BB
:10CFA0000BB0BDE8F08F08F045F901463846FCF7B4
:10CFB0008BFDF1E7284605AA8E494CF01AFD05467F
:10CFC00020B901464120FCF744FEE9E78A49FAF717
:10CFD00047F920B989494046FEF74CFEE0E7884E04
:10CFE0000B27002431682846FAF73AF9002808BFD1
:10CFF0003446013F06F11006F4D154B98149284660
:10D00000FAF72EF928B12A467F494046FEF732FE4C
:10D01000C6E7002005AA77498DF813004CF0E9FC1B
:10D020000646002C4DD0002849D0FBF7D3FA031E4A
:10D0300042DB2279062A3AD10121E26801FA03F0A3
:10D04000104239D0DBB2714840FA03F2D20733D52F
:10D050009940013908404CF09FFE0546E0880027C2
:10D060003BF0C4FC6A4903970978D0E90223002900
:10D0700018BF1A46217A637A05FB0133D11812F9D9
:10D080000390029105AA5B4900204CF0B2FC834654
:10D0900000283FD101235F499CB3029A204692F9B0
:10D0A0000020CDE900312946FAF760FC78E75D1EE3
:10D0B00013B1A37A9D42D1DB32465749A5E7574EBB
:10D0C000FAE768B10DF11301FBF75EFA28B19DF89C
:10D0D00013502846F6F770FA20B93246504994E7C3
:10D0E0004E4EFAE72846F5F74FF88146284609F0F4
:10D0F000C5F803902846254609F0F8F8029407463B
:10D10000C0E7CDE900314A4639469DF81300FAF7E9
:10D1100071FC45E73849FAF7A3F8064600282FD1F5
:10D12000ACB1EDB23F4F72B229462079F5F700F865
:10D1300000283FF435AF028831460378384601367F
:10D140000093C2F30323120BFCF7BEFCEBE7386835
:10D150007979344C72B2F5F733F800283FF420AFF8
:10D16000028831460378013620460093C2F3032338
:10D17000120BFCF7A9FC102E38687979EAD10FE779
:10D1800029495846FAF76CF8002876D05846FBF73C
:10D1900021FA824642B29CB1E9B22079F4F7C8FF85
:10D1A00000284DD1266829462046FAF78FFA3246E4
:10D1B00003461E49CDF800B04046FEF75BFDEFE6A2
:10D1C0005FFA8AF6386879790F2E35D99DF81330D1
:10D1D00017491A09CDF800B003F00F034032EBE70E
:10D1E00009A50A08E00100240EA50A0824A50A08DA
:10D1F000AA990A089F9F0A08F99A0A0835A50A08F9
:10D20000D40500246BA80A0849A50A08FEF103000A
:10D21000585D0024A19A040858A50A08C9A90A085B
:10D2200068A50A087AA50A08CEA20A089BA50A08DA
:10D23000BEA50A0893A60A08F4F7C2FF0028C5D0C5
:10D2400006AE50463146FBF757F808A94846FBF7AB
:10D2500053F8CA4520D04FFA8AF38CB1029A294676
:10D26000204613702768FAF731FA08AB02463946B0
:10D2700014480096FCF728FC92E64FF0FF3ADFE7EF
:10D28000039A1148937008AB9DF81320009611097A
:10D2900002F00F024031EDE75CB1266829462046D6
:10D2A000FAF714FA08AB024631460848FCF70CFCC2
:10D2B00076E69DF8132008AB0548110902F00F022D
:10D2C0004031F3E7E6A50A0809A60A0831A60A08CC
:10D2D0004CA60A082DE9F04F07468DB008460D46CA
:10D2E0004AF03AFB044630B9014601200DB0BDE8D2
:10D2F000F04FFCF7B5BD0246A5492846FBF77EF87E
:10D3000030B9A44938460DB0BDE8F04FFEF7B2BCC5
:10D310002246A1492846FBF771F8002854D1FCF7B2
:10D32000BBFBDFF8B8A29D480E27DFF8B4B2FCF7CC
:10D330001BFC172040F00EF81AF9018BB8F1000F12
:10D3400036D00025414658462E46FDF75FFDB10018
:10D350004046013689B208F0FFFF814609F084F8A3
:10D3600090F900300446CBB10DB9FCF795FB99F864
:10D370000630657803F0020394F90000884A894C6E
:10D38000002B18BF1446B5B107F054FF22460346E0
:10D39000314685480095FCF797FB0125042ED6D130
:10D3A00015B98248FCF7E0FB013F17F0FF07C3D136
:10D3B0000DB0BDE8F08F07F03DFF22460346314631
:10D3C0007B48FCF781FBE8E7002407AA754928465B
:10D3D0008DF81B404CF00DFB18B93846FEF760FC89
:10D3E000E6E70DF11B01FBF7CFF881460028F4D0EA
:10D3F0009DF81B502846F6F7DFF820B96D493846EE
:10D40000FEF738FCD4E72346DFF8D8814FF0FF342D
:10D4100003EB430218F8022095420BD0002C02DAED
:10D42000002A08BF1C460133152BF1D1002C16DA57
:10D430006149E4E71C4607AA5A4900204CF0D9FA92
:10D440000646002800F097805149F9F709FF38BBDC
:10D4500004465A4FDFF84881DFF88C9117E04FF00F
:10D460000009E8E73068F5F79BF9B179737902466E
:10D4700011F0020F96F807A04FEA930348460CBF3D
:10D4800039464146013300915146FCF71DFB0134FA
:10D490002846214608F006FF06460028E2D187E725
:10D4A0004FEA151A0222464930460AF1400A05F0B1
:10D4B0000F0BFAF7A3FF002845D10390B01CFBF730
:10D4C00089F8039902460491013128460592039197
:10D4D00008F0E8FE059ADDE9031338B95B465246C9
:10D4E000384900963846FEF7C5FB61E7C07990429F
:10D4F000E9D11F466300B9F1000F31D01A19424437
:10D500005678013E7A1C23440AAC284614BF2946AB
:10D51000002108EB030208F803107B1C3946537006
:10D52000FF2393702246FAF7F7FE08AA31462846F1
:10D53000FAF7F2FEB74216D108AB5A4651462248D6
:10D54000FCF7C2FA34E721493046F9F789FE20B1E9
:10D550005B4652461E490096C4E74FF0FF37C9E7C5
:10D560004FF0FF36CEE708AB5A46514619480094B3
:10D57000FCF7AAFA1CE704EB4404174B02462846C2
:10D58000A0440093012398F80110FAF77BFA0FE703
:10D59000F99A0A0835A50A0809A50A0868A60A081A
:10D5A00054980A089F9F0A0888A60A08A9A60A088C
:10D5B0009AA60A08AFA60A08C6A60A08C9A90A08B0
:10D5C000EFA60A08F2A60A0844A70A08CEA20A088B
:10D5D0001EA70A0862A70A08A19A0408C4230A0819
:10D5E00081A60A08BC250024DAA60A082DE9F04F16
:10D5F00089B0074608469C4905AA4CF0FAF9054649
:10D6000030B901464120FDF77DFB09B0BDE8F08F40
:10D610009649F9F725FE044600283BD19448954DDC
:10D62000FCF7A2FA944E1420DFF88C823FF092FEB1
:10D6300095F9060007F0FEFD2968AA88034601F166
:10D6400027413046B2FA82F201F57E01C2F11F0293
:10D65000890A4131FDF7DAFBE97911B14046FDF75E
:10D66000D5FB0134FCF718FA0835902CE0D17E493F
:10D6700005AA00204CF0BDF98049F9F7F1FD00281A
:10D68000C3D138467949FFF725FE78493846FFF778
:10D6900051FCBAE70024DFF8F89119F9340007F0DB
:10D6A000C9FD804601462846F9F7DAFD40B101344C
:10D6B000212CF2D12A4672493846FEF7DBFAA4E75C
:10D6C00005AA69494CF095F9064690B3FAF782FF2E
:10D6D00005466C4B4FEAC40A03EBC40393F8EA31E6
:10D6E0004BBB002D29DC09EB0A03588893F8049002
:10D6F00093F805A03BF07AF9EBB2D0F808B003FB41
:10D7000009AA0093002E00F09A803378002B00F0D5
:10D71000968006A93046FAF737FF002800F08C8083
:10D720009DF818500DBB58480BF80A50FCF71CFA2E
:10D730006BE70546CDE7002D05DD012B1A4638BF06
:10D740000122954209DD012B4FF001024F49384675
:10D7500038BF0123FEF7BAFB57E705AA424900206C
:10D76000013D4CF046F90646BDE72846F5F724FF93
:10D77000814600285CD02B09454F4FF000080BF87C
:10D780000A504033029305F00F030393BB79002640
:10D79000012B38BF0123019397F804B097F805A037
:10D7A00078883BF023F906FB0BA38268D15CA94281
:10D7B00022D1444504D10099B1421DD00021D15459
:10D7C0005FFA86FB33485FFA88FADDE90212FDF75B
:10D7D0001DFB59465046FDF7A9FF444509D12E4887
:10D7E000FDF714FB50465946FDF7A0FF2B48FDF707
:10D7F0000DFB2B48FCF7B8F90136019BB342CBDC9B
:10D8000008F101080837B8F1210FBFD1D9F800108D
:10D81000B9F8042001F127412248B2FA82F201F559
:10D820007E01C2F11F02890A4131FCF74DF9ECE695
:10D830003846FEF735FAE8E632461B493CE71BF866
:10D840000A30013573B11A09184903F00F0306A80D
:10D850004032FAF7DBFC06AB2A4641461448FCF797
:10D8600033F9D2E6134BF7E79F9F0A0809A50A0888
:10D8700088A70A08C41B0024C6A70A08D1A70A085B
:10D88000D5A70A0884BB0908F7A70A08F1A70A0860
:10D8900068BD090809A80A086D980A082DA80A0891
:10D8A00047AF0A0837A80A0853A80A08BD970A080C
:10D8B0006FA80A0809940A0801980A0820B100789C
:10D8C000B0FA80F040097047012070472DE9F74F0A
:10D8D00081460846FFF7F2FF0E46054670B1002468
:10D8E00001A9204601343FF069FE01464846FFF792
:10D8F000EDFF122CF4D103B0BDE8F08F0846FAF723
:10D9000069FEC4B2112C72D83D4D701CF9F7EDFFC1
:10D910003C4E05EB44088346670098F808A1B8B967
:10D92000AAF102014B424B413D4495F80821B25CFB
:10D93000002B55D095F80931192040F2EE2100FB5B
:10D9400003132146304803B0BDE8F04FFCF7BCB8E4
:10D95000017830464CF087F880B1032C2B49A0EBBE
:10D96000060394BF0022012202EB42020A4452FA4B
:10D9700083F393F8A0A6BAF1030F05D1484603B08C
:10D98000BDE8F04FFEF78CB95846F9F7AEFFF0B19D
:10D99000BAF1020FF2D1FAF71DFE40F6CA0380B2C7
:10D9A0009842A8BF184640F2EE239842B8BF1846E6
:10D9B0001923A0F2EE20B0FBF3F088F80901AAF1D8
:10D9C000020253425341EA1982F808A1ACE7BAF1C6
:10D9D000020FF4D1484603B0BDE8F04FFEF79EB900
:10D9E00021460B4803B0BDE8F04FFCF76DB811239A
:10D9F0002A460849484603B0BDE8F04FFEF766BA2C
:10DA0000506E002450350A0883A80A0884BB090810
:10DA100093A80A08A0A80A082DE9F041054686B097
:10DA200008460F46FFF74AFF064640B100235C490F
:10DA300001201A4606B0BDE8F041FCF7C9BA084615
:10DA4000FAF7C8FD1328044600F3A08006258DF8D8
:10DA50001760544E4543781CF9F747FF074660B1FD
:10DA6000FAF7B8FDC0B212F05BFA30B1731902795F
:10DA700083F8482601238DF817303846F9F735FF2B
:10DA8000074668B1FAF7A6FD0D2809D8062303FB5F
:10DA9000046383F849069DF8173001338DF8173079
:10DAA000DFF8FC80A91C0DF1170238464144FAF753
:10DAB00095FDF9F71AFF074668B1FAF78BFD0128C3
:10DAC00009D89DF817300622013302FB04628DF855
:10DAD000173082F84C063846F9F707FF80B1FAF79D
:10DAE00079FDC0B212F01CFA50B19DF81730062231
:10DAF000017902FB0462013382F84D168DF817306C
:10DB00009DF817200623042A2FD103FB046300226B
:10DB1000A3F84C26062519F03DFB05FB046595F896
:10DB2000480612F0E3F995F84B1695F84A76192352
:10DB30004FF46172804695F84D0613FB012613FBE6
:10DB4000072712F0D3F94379214698F8052003936B
:10DB500095F84C3614480097CDE9016395F849369D
:10DB6000FBF7B2FF06B0BDE8F081052A05D103FB43
:10DB70000463002283F84D26CCE7062ACAD000238E
:10DB800008EB050248F805309380C3E713233246BB
:10DB90000649284606B0BDE8F041FEF797B900BF38
:10DBA000A0630024585D002410960A08F1A70A0813
:10DBB0002DE9F04F80468DB00846FFF77FFE054601
:10DBC00040B10023624901201A460DB0BDE8F04F74
:10DBD000FCF776BA09AF099007915E49C7E90100E1
:10DBE00007A84BF0D9FE06463FF0C8FB431C04468D
:10DBF0000CD12B460A2208A93046FAF73BFC089BB9
:10DC00001B781BB9C4B2132C15D944B2A31CDBB2C8
:10DC1000012B0AD94E4E002396F90420A24200F0AF
:10DC20008C8001330C360A2BF6D14046FEF738F8CB
:10DC30000DB0BDE8F08F333464B2E7E7002302256E
:10DC40000A221946FAF716FC09904FF0000BDFF88C
:10DC50000491DFF808A1494607A84BF09DFE20B3C8
:10DC6000FAF7B8FC3C4A002352F8041B884222D140
:10DC7000DBB20AEB8302D2F8A421904215D1BBF1AA
:10DC8000020F22D0BBF1030F24D05A1EBBF1010FAB
:10DC9000D2B215D00B2A03D88DF829300135EDB258
:10DCA0000BF1010BBBF1040FD5D1052D18D840465F
:10DCB000FEF734F8BCE70133102BD5D10023D8E7A9
:10DCC000052AEDD88DF82A30E8E7092BE8D88DF839
:10DCD0002C30E3E79A1E0D2AE2D88DF82B30DDE7D1
:10DCE00097E8070086E8070020463FF051FC1B4AF2
:10DCF0009DF82B10034602EB8101D1F8A411049189
:10DD00009DF82C1002EB8101D1F8A41103919DF82C
:10DD10002A1002EB8101D1F8A41102919DF829107B
:10DD200002EB81020021D2F8A42108460192099A4F
:10DD300000920B4AFBF7B4FE7AE7064907A88DF874
:10DD400028404BF029FE00287FF478AF01257CE7BE
:10DD5000606200249F9F0A0828BD090884BB090847
:10DD600029960A082DE9F04F0346A1B00846FFF7AF
:10DD7000A5FD054628B1184621B0BDE8F04FFDF7D6
:10DD8000CDBFFF23DFF8C09207464FF0FF388DF874
:10DD90002830D9F8C0300B9093F83820ADF8300017
:10DDA0000D908DF838200F90ADF840001193099137
:10DDB000CDE90500934909A84BF0EEFD044618BBD8
:10DDC00001460AAC904F0B0190481A57002310F9F6
:10DDD000016BB24240F0D2804E1C10463FF0D8FB9F
:10DDE000024631463846FBF76FFE022E4FF0010126
:10DDF000E9D19DF938A09DF92830534540F0C58000
:10DE00008348FBF761FE4DE02378002BD2D0032F2F
:10DE1000D4BF00260126062F00F2A980DFE807F014
:10DE20000447509104475000042F10D079492046F0
:10DE3000FAF708FB58B14FF480600CF057FE002849
:10DE400000F0B58190F90400012306930AE07249BD
:10DE50002046F9F705FA70B9D9F8C03093F93800BF
:10DE6000042F22D0119B119320AB03EB061606F86A
:10DE7000580C01379EE720463FF080FA0028EFDA81
:10DE800001230A2212A92046FAF7F4FA40B2002828
:10DE900003DB129B1B78002BE2D02246711C5F48EB
:10DEA000FBF712FE21B0BDE8F08F0023DBE7204630
:10DEB000FAF790FB20AB03EB061646F8540CD8E7B4
:10DEC00057492046FAF7BEFAB0F1000A55492046F4
:10DED00018BF4FF0010AFAF7B5FA08B14AF0020A82
:10DEE0003301DFF868C1079320AB03EB0616BCE8EB
:10DEF0000F0006F850AC12AE0DF1480A0FC6BCE890
:10DF00000F000FC6BCE80F000FC69CE8030086E8B0
:10DF100003000026B346DAF8001020464BF0CAFE94
:10DF200010B19AF804301E430BF1010B0AF1080AF4
:10DF3000BBF1070FEFD1079B80336B4403F84F6CA5
:10DF400097E739492046F9F78BF9A0B137492046C0
:10DF5000F9F786F900288CD02046FAF73BFB032816
:10DF6000804686D901463248FBF7AEFD9AE7224645
:10DF70000821304894E7012305937AE701330A2BFF
:10DF80007FF425AF01312C488AE70B9B1BB9AAF11E
:10DF900014025542554100235F1CE368002B62D1F7
:10DFA00094F900B058460AF005F8D4F8049018B176
:10DFB0000668002E40F08B80B9F1000F237A14BF61
:10DFC0004E464FF46146666023B91C48FBF77CFD62
:10DFD00003232372627A2AB1394619480792FBF764
:10DFE00073FD079A02925846237ACDE90063002315
:10DFF0001A4619460CF0EFFDE06048BB394611485F
:10E00000B2E700BF9F9F0A0824A90A0883B2090843
:10E0100041A90A08C3A80A08CEA80A08D2A80A0873
:10E02000EDA80A08C6AD0A08689F0A08CEA20A0829
:10E03000F0A80A0808A90A082FA90A085AA90A0874
:10E0400075A90A0890A90A08506E00242CC2090874
:10E0500058493346584A5948B9F1000F18BF0A4683
:10E060003946FCF7D3FE022F04F110044FF00103F0
:10E0700092D1119E0D9F4DB15148FBF775FD33684C
:10E080001B6A1BB13A464F4930469847059B002B07
:10E0900050D04D49474BBAF1140F18BF19464B48A1
:10E0A000FBF712FDBAF1140F09D1059B002B43D0E9
:10E0B0003368DB691BB10022454930469847069B0F
:10E0C000002B43D10022314638463FF06FF9E6601D
:10E0D000B9F1000F2CD04946304601F067FE3D4AA9
:10E0E000B36839463C48FBF7EFFC94F80890B9F167
:10E0F000000F0CD03279914509D04B46394637484C
:10E10000FBF7E2FC3368494630469B699847637ADF
:10E1100023B1727939463248FBF7D6FCF36A002BFB
:10E12000A1D039462F48FBF7CFFC0023F3629AE7D2
:10E13000204AD5E71F49B2E7B8F1000FBFDB3368CB
:10E14000DB69002BBBD042462749B6E7DFF89C903D
:10E150000025DFF89CA04FF0030B07F025F8052001
:10E16000F8F70EF89AF80030AB42ABD919F8014F26
:10E17000C4B1204608F0BAF8804698B12046F5F7B9
:10E180001BFA0446EBB210B180F806B0C37120460A
:10E190000121F4F7ABFD98F806302046DB0703D5E4
:10E1A000F4F7D6FB0135DDE7F4F7CCFBFAE74FF0E7
:10E1B000FF3049E6C9A90A08A8A80A08ACA90A08B4
:10E1C00062AA0A08ADFD0408B6A80A088BAA0A08C4
:10E1D00003790408B1A80A08CAA90A08EFA90A081D
:10E1E00012AA0A0849AA0A088D760408132F0024E7
:10E1F000481C00202DE9F04380468BB008460F46AE
:10E20000FFF75CFB044640B100235E4901201A463B
:10E210000BB0BDE8F043FBF7D7BF0846FAF7DAF9D1
:10E220001D28054600F3A5800A268DF827404643A1
:10E23000781CF9F75AFB10B101238DF82730F9F754
:10E2400054FB514C074668B1FAF7C4F90D2809D8B8
:10E250000A2303FB054383F82C019DF82730013383
:10E260008DF82730DFF81C91711C0DF1270238461C
:10E270004944FAF7B3F9F9F738FB074668B1FAF7FA
:10E28000A9F9232809D89DF827300A22013302FB77
:10E2900005428DF8273082F82F013846F9F725FB23
:10E2A000074668B1FAF796F90D2809D89DF8273086
:10E2B0000A22013302FB05428DF8273082F8300133
:10E2C0009DF82730062B0CD0002309EB06024046B0
:10E2D00049F80630536013810BB0BDE8F043FDF7F9
:10E2E0001DBD0A260023384606FB0546A6F8323136
:10E2F000A6F83431F9F7F9FA074618B1FAF76AF9CE
:10E30000A6F832013846F9F7F0FA30B1FAF762F9B7
:10E310000A2303FB0543A3F834011C4B4FF0FF32E3
:10E320004FF461705A600A2303FB0542B2F834319E
:10E330000693B2F83231059392F83031049392F893
:10E340002F310393192392F82E1113FB010102912F
:10E3500092F82D1113FB010300210193084692F856
:10E360002C310B4A00932B46FBF79AFB0BB0BDE810
:10E37000F0831D232246074940460BB0BDE8F04319
:10E38000FDF7A4BD7C6F0024506E0024C805002456
:10E3900046960A08F1A70A082DE9F14F06460D46F0
:10E3A000DFF890B12846FFF789FA074640B100230D
:10E3B000594901201A4601B0BDE8F04FFBF766BF8E
:10E3C000052256492846FAF719F860B9524B00223F
:10E3D0001A601A611A621A631A641A651A661A6751
:10E3E00001B0BDE8F08F042259462846FAF706F836
:10E3F00004462846002C42D1F9F777FA0746002850
:10E40000EED049F0A9FADFF830A15FFA80F85AF8A7
:10E41000049BB9F1000F07D12A464149304601B0AB
:10E42000BDE8F04FFDF726BC424649463846013468
:10E43000F9F7E4FF84460028E9D1374A0346002172
:10E440001546013342F8101B082BFAD1354B03EB6C
:10E45000C40257682FB949463348344DFBF734FBA3
:10E46000A0E713F834E0F445F5DA07EB0C1305EBFD
:10E470000C140CF1010C0FCB84E80F00F3E7FAF752
:10E48000A9F8072804463DD82846F9F72EFA07468A
:10E4900058B3F8F783FF204B012503EB041383EDFA
:10E4A000000A3846F9F721FA074638B1F8F776FF3F
:10E4B000194B013503EB041383ED010A3846F9F7D4
:10E4C00014FA074638B1F8F769FF134B013503EB2F
:10E4D000041383ED020A3846F9F707FA38B93046D3
:10E4E00001B0BDE8F04FFDF719BC0546D9E7F8F7D4
:10E4F00055FF094B032D03EB041383ED030A3FF48F
:10E5000056AFECE707233A460949304601B0BDE86B
:10E51000F04FFDF7DBBC00BFEC350024689F0A0814
:10E52000739F0A0890B20908849F0A08C9A90A08BB
:10E53000F1A70A086E9F0A0840C109082DE9F341B6
:10E5400005460846FFF7BAF90C46074640B10023D6
:10E55000334901201A4602B0BDE8F041FBF730BF55
:10E5600030492046F8F77CFE70B904222C4B4FF45A
:10E570007A704FF4FA61013A1880598003F104036C
:10E58000F9D102B0BDE8F0812046FAF723F803285C
:10E59000064641D82046F9F7A8F9074698B1FAF798
:10E5A00019F84FF0010804463846F9F79EF920B1F2
:10E5B000FAF710F8B8F1000F09D1284602B0BDE80B
:10E5C000F041FDF7ABBB40F2EE248046ECE7A4F24D
:10E5D000EE2240F2DC539A4203D8A0F2EE229A4295
:10E5E0000AD940F6CA0340F2EE220F49284602B08B
:10E5F000BDE8F041FDF76ABC0C4B00210C4A03EB6F
:10E600008603A3F85842A3F85A023346CDE90040E6
:10E610000846FBF745FAB4E703233A460549E5E720
:10E62000A8700024689F0A08AEAA0A08506E002449
:10E630007D960A08A0A80A08F0B5074689B00846E2
:10E640000E46FFF73BF9054640B100231A49012069
:10E650001A4609B0BDE8F040FBF7F4BE0846F9F7EA
:10E66000B9FF1F2804461DD83046F9F73EF9014688
:10E6700020462FF09DFC78B103AE0F48314600EBE9
:10E6800084003EF035FF23460C4A29462846009672
:10E69000FBF706FA09B0F0BD384609B0BDE8F04016
:10E6A000FDF7FEBA1F232A460549384609B0BDE8E2
:10E6B000F040FDF70BBC00BFB87000248E960A082E
:10E6C000F1A70A08F0B5074685B008460E46FFF7E1
:10E6D000F5F8054640B100231D4901201A4605B052
:10E6E000BDE8F040FBF7F6BE0846F9F773FF0F28C8
:10E6F000044623DC3046F9F7F8F8014620462FF0AF
:10E7000031FDA8B104F12002124B2946284603EB43
:10E71000820393F86B22029293F86A220192B3F873
:10E7200068320D4A00932346FBF7BAF905B0F0BDF5
:10E73000384605B0BDE8F040FDF7B2BA0F232A46CF
:10E740000649384605B0BDE8F040FDF7BFBB00BF45
:10E7500038710024506E002498960A08F1A70A0820
:10E76000F0B5054685B008460B46FFF7A7F8044606
:10E7700040B100231B4901201A4605B0BDE8F04016
:10E78000FBF7EEBE01AE184F6A46174918464BF02C
:10E7900030F988B1032C04D12846FDF7BFFA05B043
:10E7A000F0BDF9F717FF6A4646F8040B394600201A
:10E7B00001344BF01EF9ECE7032CEDD1039FDDE9AA
:10E7C00001463A463146E0B22FF006FD18B9284618
:10E7D000FDF766FAE3E73B46324621460348FBF77E
:10E7E00073F9DCE7B87000249F9F0A08AA960A080C
:10E7F000F0B506468BB008460D46FFF75FF80446B5
:10E8000028B300233E4901201A460BB0BDE8F04072
:10E81000FBF740BF2D2903D0A1F13003092B49D8C4
:10E82000052C05DD30460BB0BDE8F040FDF776BAAB
:10E830002846F9F7CFFE0AAB621C03EB440424F828
:10E840000C0C15F8013F303B092BFAD914462978F6
:10E850000029DFD1062CE5D1BDF81C20BDF91C3004
:10E86000072ADFD8BDF91E50A5F5FA7292B2B2F5AB
:10E87000FA6F18D8BDF92070A7F5FA7292B2B2F506
:10E88000FA6F10D8BDF922C065450CDC67450ADB7C
:10E89000BDF924E00EF1640292B2C82A03D8BDF992
:10E8A0002640112C11DD174930460BB0BDE8F04071
:10E8B000FDF7E0B9202902D101352246C6E73046EE
:10E8C0000BB0BDE8F040FDF7EBB90C200E4A64B286
:10E8D00000FB03220846A2F84050A2F84270A2F8BA
:10E8E00044C082F846E082F84740084A0095CDE9E6
:10E8F00003E4CDE9017CFBF7D3F80BB0F0BD00BF1A
:10E900008C6E0024A79F0A08506E0024BE960A0849
:10E910002DE9F04F074689B008468B46FEF7CEFF3B
:10E92000054640B100234D4901201A4609B0BDE813
:10E93000F04FFBF7D1BF4A4B084693F8E4A693F893
:10E94000E59693F8CE87F9F745FE092804467BDC67
:10E9500006268DF81F50414D46430BF10100F8F794
:10E96000C4FF834638B1F9F735FE0D2803D80123DB
:10E97000A8558DF81F305846F8F7B7FF834660B1A9
:10E98000F9F728FE504508D8062303FB04535870B6
:10E990009DF81F3001338DF81F305846F8F7A5FF5A
:10E9A000824660B1F9F716FE484508D8062303FBF6
:10E9B000045398709DF81F3001338DF81F30504676
:10E9C000F8F793FF814660B1F9F704FE804508D35C
:10E9D000062303FB0453D8709DF81F3001338DF8D4
:10E9E0001F30311D0DF11F0248462944F9F7F6FD8D
:10E9F0009DF81F30062B09D00023AA193846AB51C9
:10EA0000938009B0BDE8F04FFDF788B963434FF438
:10EA100061761921EA18507911FB00600590107990
:10EA200011FB00610491D17803919178029100214A
:10EA3000527808460192EB5C0A4A00932346FBF7A2
:10EA40002FF809B0BDE8F08F09232A460649384659
:10EA500009B0BDE8F04FFDF739BA00BF48370024D0
:10EA6000585D002408970A08F1A70A082DE9F74F16
:10EA700005460846FEF722FF0B46044618B9334AFE
:10EA800092F858732FB9284603B0BDE8F04FFDF750
:10EA900007B92646DFF8C890DFF8C8A001AA2C49BC
:10EAA00018464AF0A6FF10B906F08AFB08E056B9EE
:10EAB000012201462846FDF7F5FF421C04461AD103
:10EAC00003B0BDE8F08FF9F785FD2F28834636D8CF
:10EAD0000FB106F069FBBBF1060F13D01D490123EE
:10EAE0005FFA8BF20978E0B205F0FAFE002759468A
:10EAF0004846FAF7E9FF01AA1549002001364AF015
:10EB000078FFD0E7DAF800301B0114D5FF2C0ED0C7
:10EB1000E1B22846FDF7F0FFE8E701372846FDF7A8
:10EB2000EBFFF9B298F800208A42F6D8DEE700271A
:10EB3000DFF82080F5E70848FBF716F8D6E72F2224
:10EB400006492846FDF796F8D5E700BF506E002429
:10EB50009F9F0A08481C0020DEA20A08CDAA0A08C6
:10EB6000BCAA0A08683500242DE9F7430746084681
:10EB7000FEF7A4FE0B46044628B1384603B0BDE8B4
:10EB8000F043FDF7CBB801AA2E49184626464AF0B5
:10EB900030FFA0460546DFF8AC9065B92A4B3246F7
:10EBA000A1B2D3F8C00041F0D7FF68BB274938466F
:10EBB000FDF760F828E0B8F1000F06D0B8F1010FBA
:10EBC00025D03846FDF7AAF81EE0284648F0C4FED6
:10EBD0001F49064602462846F9F710FC50B3324654
:10EBE0001C492846F9F70AFC30B332461A49284630
:10EBF000F9F704FC10B3324618492846F9F7FEFB32
:10EC0000F0B13846FDF74CF803B0BDE8F083B31E11
:10EC1000294638465A425A41FDF744FF421C0446F1
:10EC2000F2D001AA4946002008F101084AF0E1FEAD
:10EC30000546B2E74646F4E70126F2E70226F0E78A
:10EC40000426EEE79F9F0A08506E0024F9AA0A08DE
:10EC5000EDAA0A08F0AA0A08F3AA0A08F6AA0A08FE
:10EC60002DE9F74380460846FEF728FE0B46054689
:10EC700028B14046FDF752F803B0BDE8F08301AA81
:10EC80002C4918462F464AF0B4FE2E460446DFF8BB
:10EC9000A4907CB9022DECD1A7F57A73B3F57A7FF5
:10ECA00021D94FF4FA634FF47A7223494046FDF7B5
:10ECB0000DF9E1E74DB1012D10D001AA4946002020
:10ECC00001354AF096FE0446E3E70122214640461C
:10ECD000FDF7E8FE431C0646EFD1CDE72046F9F7E5
:10ECE00079FC0746E9E7154BB8B21B685B689847A3
:10ECF000FCEEC07AFF2E17EE902A0BD1104BB6EE29
:10ED0000C00A19780F4BA14210DC11460E48FAF7E1
:10ED1000DBFEB1E70D4B31460D48B6EEC00A03EB02
:10ED2000860383EDD70AFAF7CFFEA5E70134A3ECFB
:10ED3000010AE8E79F9F0A0807AC0A086023002041
:10ED4000481C0020AC71002424AB0A08506E00243B
:10ED500017AB0A08F8B507460846FEF7AFFDD0B175
:10ED6000204BD3F8C86001363046344608F050FFD7
:10ED70000546F0B90134182CA8BF0024204608F03D
:10ED800047FF0546A8B9B442F4D138461649BDE854
:10ED9000F840FCF76FBF0846F9F71CFC044608F082
:10EDA00037FF054628B921461048BDE8F840FAF774
:10EDB0008BBE0C4BC3F8C8400BF0A8FF2A46214677
:10EDC0000B48FAF781FE172C09D80A4B0C2202FBDC
:10EDD000043393F8E006BDE8F8400BF0D3BF002001
:10EDE000F9E700BFC805002433AB0A0847AB0A089F
:10EDF0005DAB0A0884BB090838B50446114D0846C6
:10EE0000FEF75CFD68B1104B93F900104B1C06D166
:10EE10000E4B19780E48BDE83840FAF755BEC9B216
:10EE2000F8E70846F9F7D6FB032804D8C0B2FAF78A
:10EE3000CFFA2946E3E7204603220649BDE83840D9
:10EE4000FCF718BFC9A90A08C805002438350024F2
:10EE500076AB0A0886AB0A080329F0B5054685B0EB
:10EE60000C46164614D80B4F3970FAF715FE0A49AE
:10EE70002846FFF7C1FF2246084901A8F9F7C6F95D
:10EE800001AB324608212846FCF774FEFF233B7095
:10EE900005B0F0BDC8050024C9A90A0876AB0A0868
:10EEA00038B50446114D0846FEF708FD68B1104B11
:10EEB00093F901104B1C06D10E4B59780E48BDE852
:10EEC0003840FAF701BEC9B2F8E70846F9F782FB05
:10EED000032804D8C0B213F0F5FB2946E3E7204627
:10EEE00003220649BDE83840FCF7C4BEC9A90A0898
:10EEF000C80500243835002472AB0A0881AB0A0823
:10EF00000329F0B5054685B00C46164614D80B4FBC
:10EF10007970FAF7C1FD0A492846FFF7C1FF22467A
:10EF200008496846F9F772F96B46324610212846BF
:10EF3000FCF720FEFF237B7005B0F0BDC805002460
:10EF4000C9A90A0872AB0A08444B2DE9F74FDFF84C
:10EF5000289105461A785B78009189F80130404B7A
:10EF600089F800201B780BB905F0BAF900263D4C52
:10EF700039F076FDB0460D233A4A0099734352F8B2
:10EF800003A05046F9F75EFA002841D0B8F1000F0F
:10EF900001DDFAF781FD51463348FBF737FF0022C8
:10EFA00021462846FCF758FEFAF776FD237903F050
:10EFB0001803082B45D0102B48D02046FBF733FF11
:10EFC0000D22284B02FB0633B3F8090039F00EFD81
:10EFD0008346D8B12046F8F723FB0746DBE9022138
:10EFE000024401442046F8F7B3FA78B9514601903B
:10EFF0001E48FBF70BFFDBF80810019A2846134662
:10F00000CA192146FCF7CCFCFAF746FD08F10108C5
:10F01000013640F263230D349E42ACD10020F8F754
:10F02000DEFAFF2389F8003089F80130B8F1000FCB
:10F0300011D1009A28460E4903B0BDE8F04FFCF705
:10F0400019BE0C492846FFF7D7FEB6E709492846FE
:10F05000FFF726FFB1E703B0BDE8F08F3835002495
:10F06000585D00245CCA0908A99E0A08A1AB0A08D9
:10F07000739F0A08C9A90A08C80500242DE9F74F9B
:10F08000804608460F4648F067FC044620B1012838
:10F0900024D13B782A2B21D1A94E00254FF00D0A0F
:10F0A000A84FB14604F00104A748FAF75DFD0AFB3A
:10F0B00005F33846013559F80310FBF7A7FE314632
:10F0C00022464046FCF7C8FD0D36FAF7E5FC40F253
:10F0D00063239D42EBD103B0BDE8F08F3D2138465C
:10F0E0004AF0C1FC002800F0248103469A4613F838
:10F0F000012D202AFAD0AAEB070A0130054610F8A4
:10F10000013B202BFAD05FFA8AFA4FF00009DFF8B2
:10F1100030B20D235246384603FB09F35BF8031067
:10F120000BEB03040091F9F769F9064670BB0099EF
:10F13000084648F011FC824528D1277907F0E00104
:10F14000402900F08A8012D871B366797F4A00277F
:10F1500002EBC606BA463B4696F8F0220092009AA9
:10F16000BA4202D9BAF1000F63D02BB12DE0602969
:10F17000ECD0802900F0A58040467549FCF77AFD67
:10F18000204603B0BDE8F04FFBF74DBE09F1010981
:10F1900040F263239945BCD13A466E49404603B0DC
:10F1A000BDE8F04FFCF766BD07F00703042B1CD148
:10F1B0000B460A222846F9F75DF9D4F805300146D6
:10F1C0008342D9D32046F8F74DFB0D23624803FB59
:10F1D00009F95BF80910FBF719FE002221464046A9
:10F1E00003B0BDE8F04FFCF737BD052B0DD101236F
:10F1F0000A222846F9F73EF9D4F805300146834241
:10F20000BADB5B428342B7DCDCE72846F9F7E2F978
:10F2100017F0050F014607D1B4F80520B4F8073000
:10F220009142A9DB9942EEE7B4F90520B4F9073021
:10F23000F6E7D6F8EC1251F8270060B129460193A1
:10F24000F8F70EF8019B30B94FF0010A3946204615
:10F25000F8F708FB5346013781E707F007076379A2
:10F26000013F0093009BB342AFDDAA4615F8013B76
:10F27000202BFAD02046F8F7E1FA0546042F04D8EF
:10F28000DFE807F0030E0E141D005046F9F7A2F94F
:10F29000A8552C2150464AF0E6FB0136451CE1E713
:10F2A0005046F9F797F925F81600F2E700230A22ED
:10F2B00000215046F9F7DEF845F82600E9E701237A
:10F2C000F5E7284648F048FBE379064694F805A0A0
:10F2D000DB07A7790AD52046F8F7B0FA037801468C
:10F2E00023B1324628464AF097FCE0B9DEB1B74276
:10F2F00019D32046F8F7A2FA3A4600214AF09CFBBF
:10F30000B2453FF662AF3246144928464AF084FCC3
:10F3100000283FF45AAF2046F8F790FA32462946C3
:10F320004AF02CFB51E73A460D494046FCF7A2FC57
:10F3300022E73946404603B0BDE8F04F04E600BF7F
:10F340005CCA0908A99E0A08B1AB0A0884BB09086F
:10F35000FFAB0A08739F0A08F4AB0A0820B00A083A
:10F36000C4AB0A0870B504460E46084648F0F4FAE5
:10F370003146054602462046F9F740F868B9635D14
:10F380001846F9F71FF800B933B901352C44204667
:10F3900001340378202BFAD070BD0020FCE708B5BB
:10F3A00004460948FAF770FBFAF752FB074BD3F80B
:10F3B000C0000BF0F3FB05F093FE012C01D140F0EF
:10F3C000EBFCF4F773FB00BF0DAC0A08506E002491
:10F3D00010B5044608460B46FEF770FA28B903221A
:10F3E00008491846F9F70AF828B90748FAF718FC47
:10F3F0000120FFF7D4FF20460449BDE81040FCF788
:10F4000039BC00BF19AC0A081DAC0A08DCA40A0804
:10F410002DE9F74F4FF0000B064601AA08462D498B
:10F420005D464AF0E6FA01270446DFF8B880DFF8C7
:10F43000B890DFF8A0A014BBBBF1000F27D1264C79
:10F44000002D43D029462548FAF73EFB23780BB917
:10F4500004F046FF39F004FB002384F84D30FAF73E
:10F46000CDFA15B12846F8F7BAF89FB13046FDF746
:10F4700025FD78B1FAF73AF90020FFF790FFBBF1CC
:10F48000000F0AD02046F9F7A5F885B2C5B9304675
:10F49000FCF706FC03B0BDE8F08F41462046F8F7C4
:10F4A000D1FF80B949462046F8F7CCFF0028EED0BE
:10F4B0005F4601AA514600204AF09BFA0446BAE78B
:10F4C0004FF0000BF5E74FF0010BF2E70448FAF7B5
:10F4D000A7FBBFE79F9F0A08585D002448AC0A08B5
:10F4E0006BAC0A083FAC0A0827AD0A0810B50C46F9
:10F4F000FDF7E4FC78B1084B01229A73FAF7F6F8AD
:10F500000648FAF78DFB06492046F7F7A9FE10B129
:10F510000020FFF744FF10BD3835002481AC0A08F5
:10F52000C4950A082DE9F04F0E4693B0A04917463E
:10F5300002903046FFF716FF0546002840F0218173
:10F540009C493046FFF70EFF0546002840F01B811E
:10F5500099493046FFF706FF0546002840F015811F
:10F5600096493046FFF7FEFE0546002840F00F8121
:10F5700093493046FFF7F6FE002805460ABF0124EE
:10F58000082435467F428F49284607F010073C4340
:10F59000FFF7E8FE002800F0FC8044F020048A4BCE
:10F5A0001B780BB904F09CFE39F05AFA14F0090FDD
:10F5B00000F04C838548FAF733FB0020FCF710F885
:10F5C00014F48073059340F0EE808148FAF728FB2D
:10F5D0008048FAF7C9FA04F01803182B05D17E48C1
:10F5E000FAF71EFB7D48FAF7BFFA01230493FAF7F6
:10F5F00053FA7B497B48FAF767FA7B497B48FAF76D
:10F6000063FA04F48473082B07D179490298FAF756
:10F610006AFA77490298FDF73FF814F080030793E0
:10F620000ED1744B204693F87C2303F55F73002AB8
:10F63000714A06BF012113460021704AFAF730FAD9
:10F640006F492046FBF75EFB6E492046FAF708FC3F
:10F650006D492046FAF7FDFA6C4B14F01006D3F80A
:10F6600000A06B4B1D6840F0A0806A48FAF7D8FAFA
:10F670000396694B4FF00008994606936AEA050322
:10F68000099359F804BBBBF1000F21D00127099B56
:10F69000039A204607FA08F73B400CBF01210021DE
:10F6A0000893FAF7C9FA65EA0A035C4A0390204610
:10F6B0003B425B4614BF01210021FAF771FC089917
:10F6C0005B46564A0039204618BF0121FAF7E8F98F
:10F6D00008F10108B8F11D0FD3D165EA0A034FF014
:10F6E0000008DFF850910893069B53F804BB06937B
:10F6F000BBF1000F24D0012707FA08F73D420AD0DA
:10F700006AEA05034A4620463B425B4614BF012194
:10F710000021FAF745FC1AEA070F11D0089B204692
:10F72000039A1F400CBF01210021FAF785FA391E08
:10F7300003905B464A4618BF01212046FAF7B0F90C
:10F7400008F10108B8F11D0FCED12A4D2046344BE7
:10F75000344A05F57971FAF7B3FC079B002B6BD09F
:10F76000134B224618210298FCF704FA049B002B45
:10F7700000F0D1812C48FAF753FA2C48FAF7F4F943
:10F78000C9E10124FEE60224FCE60424FAE6812411
:10F79000F8E627492846FFF7E5FD00283FF4FFAECD
:10F7A00044F48074FBE6002320E71A4B039360E7E0
:10F7B000A7AC0A08AEAC0A08B6AC0A08BCAC0A088A
:10F7C000D1A70A0862AC0A08585D0024CAAC0A082E
:10F7D000D2AC0A08EAAC0A08F6AC0A081EAD0A0860
:10F7E000339C0A08DEA10A08419C0A08FCA10A0809
:10F7F000C9A90A08506E002420B00A082EAD0A08D4
:10F800003BAD0A0845AD0A0823990A08383D002493
:10F81000603B002488AC0A08B0C109084BAD0A0857
:10F8200062AD0A086062002426AE0A083CAE0A08EF
:10F83000C5AC0A0857AD0A08DFF8B8A32046DFF8C0
:10F84000B8B39AF800209BF80030BA4F9A42BA4AEF
:10F8500013BF012100214FF001094FF00009FAF711
:10F86000EBF99BF800308046B44A07EB8303494626
:10F870002046D3F8B835FAF793FB9AF8003049469A
:10F88000AE4A07EB83072046D7F8B835AC4FFAF7F6
:10F8900007F9AC4A2046D7ED007AF5EE407AF1EE52
:10F8A00010FA0CBF01210021FAF7FAF843463A4654
:10F8B000A5492046FAF7EAFCA44B05F13C0205F500
:10F8C0008C612046FAF7E6FE26B115F9323C002B92
:10F8D00000F027819E48FAF7A3F99E48FAF744F909
:10F8E00000239D4A20469D4F02F2F4419C4DFAF7B9
:10F8F00077FF9C4B9C4A2046019300923A68296806
:10F90000FBF7AAF940F20222984B2046009201939D
:10F91000BA68A968FBF7A0F9002E40F0048194486A
:10F92000FAF77EF93246934F012593480021DFF81C
:10F93000CCC217F8013B10F8018B03F1480EEE44DE
:10F940000EF8208C1CF801EB0EF14809E94409F887
:10F95000108C002D00F0E980A3EB0E056B426B418B
:10F9600001311D460829E4D1002783F0010120461A
:10F970008DF83070FAF760F90EAB804A29462046C0
:10F980008DF84070FAF70CFB0AAB7C4A29462046FA
:10F99000FAF786F87A4A7B4B204602F53F71FAF770
:10F9A00051FD794A794B204602F53F71FAF792FDF5
:10F9B000734A774B204602F53F71FAF7D1FD754B3C
:10F9C000754A20467549FAF703FB754A754B204680
:10F9D00002F5B461FAF7F8FB734A744B204602F55E
:10F9E000B461FAF7EDFC724B724A20467249FAF79D
:10F9F000D1FF724B724A20467249FAF76DFF002E12
:10FA000040F09580B3467048FAF70AF96F4D00262A
:10FA1000DFF8EC81A5F61C073946022228464AF099
:10FA20005FF9002895F800A05A4614BF0121002173
:10FA300020460CBF4FF001094FF00009FAF7FCF81F
:10FA4000BAF1020F834640F0DD807B784FF0190A4F
:10FA500040F2EE22494620461AFB03235C4A0193FA
:10FA60003B7818F8033000933346FAF799FA6B782D
:10FA700040F2EE22494620461AFB0323544A0193E2
:10FA80002B7818F8033000933346FAF709F801365B
:10FA900002350237122EBFD100214E4B224602986A
:10FAA000FCF768F8210740F1C5800025E9B201356F
:10FAB00022460298FFF7D0F9042DF7D1464F474D63
:10FAC0003B782B70059B33B94548FAF7A9F84549AF
:10FAD0000298FFF791F9FF2300262B70F1B201364F
:10FAE00022460298FFF70CFA042EF7D17B786B7050
:10FAF000059B002B40F09B803B48FAF791F8394971
:10FB00000298FFF7CDF93948FAF78AF83848F9F73B
:10FB1000BBFFFF236B70002013B0BDE8F04FF7F779
:10FB20005EBD0B4BDDE6124AFDE62B4618E7DFF81B
:10FB300098B06BE784BB090896AC0A0869AD0A085F
:10FB4000EC35002472AD0A08683B0024A19F0A0826
:10FB500090AC0A0881AD0A081C6E0024C43600244B
:10FB60004C3D00248EAD0A08FFFF7F0095AD0A08CA
:10FB70009CAC0A088073002440330A08489F0A0896
:10FB8000B87000249AA20A0838710024A1AD0A08AE
:10FB90009CAD0A08A7AD0A08A0630024A474002441
:10FBA0007C6F0024ABAD0A08A8700024B4AD0A082D
:10FBB000BCAD0A083C64002458760024C5AD0A0890
:10FBC00048370024443C0024A0AC0A087477002481
:10FBD00083A80A08A7AC0A08083C0024C80500242A
:10FBE000C9AD0A08C9A90A08ECAD0A0813AE0A088B
:10FBF00029AD0A08403D0024E43500242C6200248D
:10FC000050350A083B7849461A4A204618F803300E
:10FC100000933346FAF7C4F92B78164A494618F888
:10FC20000330204600933346F9F73AFF2FE7FF23CE
:10FC30006B709BE5104D224602982978FFF70CF96E
:10FC4000224669780298FFF75BF98FE5A20706D58F
:10FC5000094B224602981978FFF7FEF85BE7630725
:10FC60007FF559AF044B224602985978FFF748F9BF
:10FC700051E700BF93A80A08083C0024224BB0F5C6
:10FC8000FA6F1A680346A8BF4FF4FA63B3F57A7F98
:10FC9000B8BF4FF47A73D20416D540F2DC529042CA
:10FCA00015D040F2DB5207EE903A9042F8EE677AB8
:10FCB0001FD8DFED166A9FED167A77EEE67A9FED94
:10FCC000150AA7EE870A7047B0F57A7F02D89FED34
:10FCD000120A704707EE903ADFED106A9FED107A36
:10FCE000F8EE677A9FED0F0A77EEE67AA7EE870ABD
:10FCF0007047DFED0D6A9FED0D7A77EEE67A9FEDA6
:10FD00000C0AA7EE870A70476835002400007A4481
:10FD1000D62000C000E082440000000000407A4489
:10FD2000661000400000404200A0BB44D6200040C6
:10FD300000008344704700BF704700BF0020704739
:10FD400001207047704700BF704700BF704700BF79
:10FD5000704700BF9FED010A704700BF0000000020
:10FD600000207047064B1B78834206D900EB400009
:10FD7000044B03EBC003586970470020704700BF75
:10FD8000000600203C05002000EB4000024B03EB86
:10FD9000C003587C704700BF3C050020024B187818
:10FDA000003818BF012070470006002003681B6957
:10FDB00003B11847704700BF70B5094C236873B191
:10FDC0000546002606E099681A681E732160904770
:10FDD000236823B15A681846AA1A002AF3DA70BDBC
:10FDE000F07D00240022FFF79DBB0122FFF79ABBA4
:10FDF0002DE9F84F002607460C461D4DB046DFF8AA
:10FE00007890DFF878A02046FDF758FDD5F800B0CF
:10FE100048B921465846F8F715FB20B921466868CD
:10FE2000F8F710FB80B15846F9F72EFE696811B15A
:10FE30005046FAF7EBFFA96811B14846FAF7E6FF1A
:10FE40004FF00108F9F728FE013610353A2EDAD1C5
:10FE50002046FDF733FD48B9B8F1000F06D1224620
:10FE600038460449BDE8F84FFBF704BFBDE8F88FFA
:10FE700064E9090880AE0A087AAE0A0874AE0A0876
:10FE8000F8B5354C2368002B53D00A2801D00D2833
:10FE90004DD1324D2B790BB1F9F7FEFD304E2321B8
:10FEA000304649F0E0FD08B1801B20602368002245
:10FEB0006BB902B12360F9F7BBFD2B79EBB129488F
:10FEC000BDE8F840F9F7E0BD01220B46F0E7591E06
:10FED000705C2028F8D08AB90022234C204FF254BD
:10FEE0003B26013E0CD13146204B9C4211D2E368A7
:10FEF000206898476B79002BDDD1F8BD2360EBE7D4
:10FF000021683846FFF72EFA01460028ECD110345C
:10FF1000E7E72B7923B116491648FBF727FDCAE717
:10FF20001548F9F7B1FD0E48F9F71EFEC3E7FF2BA0
:10FF3000E3D8A0F120025E2ADFD80BB92028DCD05C
:10FF40005A1C2260064AD054044B1B79002BD4D093
:10FF5000BDE8F840FAF71AB868660024F07D00247E
:10FF600066650024BF950A0864E9090804ED0908DC
:10FF700094AE0A08B0AE0A08B6AE0A0808B5294B16
:10FF80001B68DB041ED5B5EE400AF1EE10FA26D050
:10FF9000DFED257AB4EEE70AF1EE10FA1FD49FEDFB
:10FFA000237AB4EEC70AF1EE10FA2AD870EE677A17
:10FFB0009FED1F7A9FED1F0AA7EE870A49F006F80A
:10FFC00080B208BDDFED187AB4EEE70AF1EE10FA60
:10FFD0000BDA9FED190A48F0F9FF80B208BD9FEDDA
:10FFE000170A48F0F3FF80B208BD70EE677A9FED04
:10FFF000147A9FED140AA7EE870A48F0E7FF80B253
:020000040805ED
:1000000008BDDFED117ADFED116A70EE677A9FEDC2
:10001000107AA7EEA67AB0EE470A48F0D7FF80B272
:1000200008BD00BF683500240000404200E0824463
:1000300066BEFFBE0060BB4400007A440080BB4443
:1000400038DFFF3E00407A440000834466BEFF3E36
:1000500000A0BB44F8B5CB4B1B6813F004052DED95
:10006000048B40F0D8809FEDC88AC84C13F0200361
:1000700004D094F8D43013F0020344D194F815213D
:10008000DFEDC38A12F0010294F8141150D1A9BB1C
:10009000D4ED467A9FEDBF6ADFEDBF6A67EE867AE0
:1000A00094ED487A38EE477AE8EE267A84ED477A7E
:1000B000C4ED467A63B1012194F82821D4F8D830F0
:1000C0008A4284F81611C4F8243118BFC4F81C31D0
:1000D000B24B1E780D2E0BD1D4ED367A9FEDB07A4F
:1000E000B04B67EE877AFDEEE77A17EE902A9A809A
:1000F000B0EE489A00259FEDA47A37E084F81621E7
:1001000084F81421C4E7D4ED397AB4F8E830F8EE75
:10011000E77AC4ED367A002B40F0EF80DFED9C8A61
:1001200094F81521012394F8141112F00102AED0B5
:10013000002900F0CB80D4ED489A984A38EE699AAD
:1001400094F816711678002B6AD0012F02D0002D7A
:1001500040F0EB80002F40F003810D2E00F0058170
:10016000002D40F0BB8094ED4C7A0125D4ED4E7A01
:10017000D4ED4F6A37EE677A94ED4D8AE6EE877AD2
:1001800037EEC87AC4ED4E7AA6EE878A84ED4D8AA2
:1001900084ED4C8A0DB184ED478AD4ED527A94ED0A
:1001A000507AB0EE676ADFED805A38EE477AD4EDC8
:1001B000536A94ED510A84ED508A97EE256AE6EE73
:1001C000867A37EEC07AC4ED527AA6EE870A84EDBD
:1001D000510A84ED540A48F0F9FE02B282EAE27351
:1001E000A3EBE2739BB2092B6ED9002AACBF0A388D
:1001F0000A3005B20D2EA4F8545150D0242E41D00F
:10020000382E05D1B0EE480A48F0E0FE654B9880E4
:10021000BDEC048BF8BD5D4C012594ED328A25E7D9
:100220000D2E77D0DFED588A002F99D094F8283121
:10023000002B5CD194ED4C7A002D96D077EE487A65
:1002400094F829319FED596A06EE903A77EEA97A33
:10025000F8EEE66AF0EEE77A67EEA67AF4EEC67A92
:10026000F1EE10FA03DD28EE866AC6EE278AF7EE75
:10027000007A77EEE87A67EE897AE8EE877AB0EE70
:10028000677A73E7DFED4A7A94ED470A20EE270A92
:1002900048F09CFE434BBDEC048B5880F8BDDFED6D
:1002A000427A9FED430A68EEA77A3E4C29EE000A97
:1002B000FDEEE77A17EE903A238048F087FEE5805E
:1002C0006080BDEC048BF8BD002593E7D4ED469A21
:1002D0000122C4ED489A84F814212EE794F82831BD
:1002E000012B94BFB0EE497A94ED4C7A3EE7022B95
:1002F0003FF439AF002DF1D135E707EE903ADFED4D
:100300002A6A9FED2C7AF8EEE77AC6EEA78AC8FE35
:10031000C78A05E7DFED267A94ED4C0A20EE270A1E
:1003200048F054FE1F4B98807CE794ED360A012379
:1003300070EE487A84F8163177EEA97AC4ED497ADE
:1003400030EE670A0D2E84ED4C0A7FF46FAFDFEDBF
:10035000187A20EE270A48F039FE124B988065E79C
:1003600094ED360AD4ED497AEAE7DFED117A94ED9F
:100370004C0A20EE270A48F029FE0A4B9880002DEF
:10038000ACD1F0E67C66002400000000F07D002483
:100390009A99993ECDCC4C3FCDCC4C3E00300024B8
:1003A0000AD7233C043000240000C84200401C4609
:1003B000CDCCCC3D6666663F70B5254C2378012BCD
:1003C00000D070BD234B1B68002BFAD0224D2B6848
:1003D00028465B6898470028F3D0204B204E1A68C7
:1003E000338892889A421FD31E4900222846096802
:1003F0004968EA622A6803FB01F1D36898472B68D1
:100400009B6813B128469847F8B13388164A0133E0
:1004100052683380002AD4D0116893884A69134205
:1004200018BF1B048B6170BD0F4A00210F4B52682F
:100430001B782170002AC4D0C3F34003918812684E
:100440001B0101FA03F3936170BD3FF0ADFCDCE7E3
:1004500056300024E0220024E422002450300024FE
:10046000543000244C300024202300242C2300246A
:100470002DE9F84FB24C8046B24B2DED028B94F82B
:10048000152194F85651D2071F885DD5AE4E012D27
:1004900094ED5A8A00F09080022D49D0ADB9B4F89D
:1004A0005C319F42A94B00F2B5801A68F37DD4F805
:1004B0006C1103EB8303521A03EB8303B2EB830F3C
:1004C000C0F22381012584F85651F37B33B1B389FF
:1004D00023B19F4B1B78002B40F0908094F857215C
:1004E000AA4238BF2A46337A632B07D8022D94F8E4
:1004F000601100F0DA80002940F0EB80954B9FED11
:10050000967A1A70B17BD4E95E30C4F87C311B1A3C
:1005100007FB03F307EE903AF8EEE77AA7EE878A37
:1005200084ED5A8A00293BD1BDEC028BBDE8F88FDF
:10053000B4F85A31BB42C8D2844B01251B6884F8F9
:100540005651C4F86C31C0E7EA1E012A44D9188913
:100550007D4EC0F30B0049F01FFC092897DDB6F86B
:100560000690B94502D83388BB4290D2B7EB490F09
:100570008DDC0323DFED797A754A84F85631B0EECD
:10058000678A84F857310023C4ED5A7A1370A4F8AF
:100590005831A4F85A31A4F85C31A4F85E312BE04C
:1005A000012A00F0A080022ABED10720BDEC028BF8
:1005B000BDE8F84F0AF0E6BBB4F85E31BB422ED27C
:1005C000B4F85831BB4202D2002584F856515F4B33
:1005D0001B68C4F86C3178E75B4EB6F80690B945F5
:1005E00002D83288BA422CD2B7EB490F29DC032D4E
:1005F00040F0988094ED5A8A032566E712F010F8CF
:10060000002877D102232A469D4284F8573138BF0B
:100610001A4668E71B680025C4F86C3155E74B4B58
:10062000D4F86C111A68337E521A03EB830303EB80
:100630008303B2EB830FFFF648AF022584F85651CF
:1006400043E71889C0F30B0049F0A6FB09285EDDDB
:100650000022317D84F8562184F85721002900F0CA
:1006600083803B4B1970B388728813FB01F312FB34
:1006700001F2717C9BB292B28B42A4F85831A4F87B
:100680005A215AD95B1A9BB28A42A4F85C3152D9DA
:10069000521A92B2A4F85E21642294ED5A8A84F828
:1006A00061210022C4F86421FBE691B90120C4F85D
:1006B000648184F86001C3F1640301FB03F0284BFB
:1006C00083FB0013C017A0EBA350643084F86101D2
:1006D00014E7D4F864112348A8EB01018142EADB56
:1006E00084F861310AE7BDEC028B0820BDE8F84FC1
:1006F0000AF048BB337C83420FD301232A469D4234
:1007000084F8573138BF1A46EDE60025DDE6032DA3
:100710003FF470AF94ED5A8AD7E600232A4684F856
:100720005731E0E61889C0F30B0049F035FB092882
:100730003FF717AFEEE70022ACE70023A4E700BFC6
:10074000F07D0024F46D002430630024182300247D
:10075000046E0024056E0024ACC52737000000009D
:100760006BCA5F6B809698003588B7FBF5F501354D
:10077000082D39DCE9B2204ADFF88890126889F840
:10078000001092F97620AA423FF46DAF002A3FF4A0
:100790006AAF1A4A92F800E00EF1010202F0030279
:1007A00096453FF460AF4FF0FF30DFF85CB04FF09C
:1007B000EA0A0AE0002803DABCF1000F08BF10467D
:1007C000013202F00302964511D00AFB02BC9CF9EB
:1007D00076C0AC45EED11046C0B2F8F7F9FD084B33
:1007E00099F800101F883EE708252946C3E700282E
:1007F000FFF639AFF0E700BFBC36002438350024DF
:10080000F46D0024046E0024805E00242DE9F8437A
:10081000A84C2DED048BA36820469847002800F0D3
:10082000BB80B4F90E30A17D06EE903AB4F91030D9
:10083000092907EE103AB4F91230F8EEE66A07EE2D
:10084000903AB8EEC77AF8EEE77AC4ED126A84ED12
:10085000137AC4ED147A00F0A380974E04F1480097
:1008600021F0C0FAB28DB36A002A40F0A580934A05
:10087000934D1268520700F1E880B3F90020D4EDDF
:10088000147A06EE102AB3F90220B3F9043006EE0A
:10089000902AB8EEC66A07EE103A8A4BF8EEE66A7E
:1008A00094ED128AB8EEC77A93F86E75864B38EEDF
:1008B000468AD4ED138A93F8008037EEC79AB4F8CD
:1008C000443078EEE68A84ED128A07EE903A338857
:1008D000C4ED138AF8EEE79A84ED149A002B40F0E9
:1008E000FF80B8F1040F00F0D881D5ED6B7AD5ED1B
:1008F0006C6A95ED6D7A78EEE66A85ED6B8A39EE75
:10090000477AC5ED6C8A38EE678A85ED6D9A66EE9A
:10091000A96A27EE297A28EE298AC4ED166A84EDA1
:10092000177A84ED158A94ED137AB8F1040FD4ED9B
:10093000167A27EE077AD4ED124A67EEA77A94ED7D
:10094000155AD4ED145AA4EEA47A94ED176AE5EE84
:10095000057AD4ED006AA5EEA57AE6EE067AB1EE48
:10096000C70AB1EEE77A26EE800A84ED180A26EE71
:10097000878A84ED198A0CD1DFED548A544D20EE1C
:10098000280A48F023FB28EE280AA88048F01EFB1E
:100990002881012384F86830BDEC048BBDE8F8831E
:1009A000454E04F1200104F1480021F0B3F9B28D65
:1009B000B36A002A3FF45BAFB2F5C87F00F0518103
:1009C0003F4D4FF0000E94ED127A4FF0000CD5ED34
:1009D000606A012AD4ED137AF8EEE66A94ED146A9F
:1009E000C4F848E0A3F800C076EE876A95ED617A16
:1009F000C4F84CE0B8EEC77AA3F802C0FDEEE66A90
:100A0000C4F850E0A3F804C037EE277AD5ED627A37
:100A100016EE907AC5ED606AF8EEE77ABDEEC77A19
:100A200077EE867A17EE100A85ED617AFDEEE77AA9
:100A300017EE901AC5ED627A00F01682013AB2857F
:100A40001E4A126852077FF518AFB5F88C71322F25
:100A500000F0C180002F40F0828195F8AA21002A81
:100A60003FF40BAF05F5CE70DFF86CC0B4F80CE0C6
:100A7000002707C88CFB0298D21785F8AA71C2EB31
:100A80002812A2EB0E029A808CFB00E2C017C0EB8A
:100A900022108CFB012CC91701221880C1EB2C11EC
:100AA00059800C4BDF81C3F80A20F8F755FEB36A72
:100AB000E3E600BF04350020302300206835002421
:100AC000F07D0024A01D00200030002400007A44A6
:100AD00004300024846300241F85EB510AD7233C93
:100AE000002F00F0B380D6ED027AD6ED036A38EE1F
:100AF000678A96ED010A95ED6B7AE8EE267A37EE75
:100B0000C06AC6ED027AA6EE260A30EE478A86ED66
:100B1000010A84ED120A85ED6B0A28EE298A84ED1C
:100B2000158A002F7FD0012F00F07981D6ED057A4C
:100B3000012F96ED067A78EEE78A96ED040A95ED98
:100B40006C8AE8EE877A77EEC06AC6ED057AA6EE83
:100B5000870A30EE488A86ED040A84ED130A85ED93
:100B60006C0A28EE298A84ED168A00F03A81022F59
:100B700000F04A8196ED087A022FD6ED096A79EEE7
:100B8000477A96ED070A95ED6D8AA6EEA77A77EE7D
:100B9000407A86ED087AA6EEA70A30EE488A86EDFE
:100BA000070A84ED140A85ED6D0A28EE298A84ED82
:100BB000178A7FF4B8AEB8F1040F7FF4B4AE48F0F2
:100BC00005FA1FED3A0ABB4D28EE000A688048F08E
:100BD000FDF9E880A7E6B84A0021D4ED126AD26890
:100BE00094ED137AFDEEE66AC5F898211A68BDEE19
:100BF000C77AD4ED147AC5F890219A88FDEEE77A89
:100C0000A164A5F894210022C5ED676A1A8085EDDC
:100C1000687AE164C5ED697A5A8021659A80013F5E
:100C2000A5F88C7119E7B8F1040F7FF47FAF48F095
:100C3000CDF99FEDA20ADFF87C9228EE000AA9F810
:100C4000020048F0C3F9A9F806006FE7B8F1040FF5
:100C50007FF449AFB0EE480A48F0B8F9954B1880D8
:100C600041E7D4ED126A002094ED137A0021D4ED0F
:100C7000147AFDEEE66ABDEEC77A914DFDEEE77A95
:100C8000A064C5ED606A198085ED617AE064C5ED08
:100C9000627A598020659980D0E697B3D5ED6B7A5A
:100CA000012F85ED6B8A38EE678A28EE298A84ED5C
:100CB000158A00F0BF80D5ED6C7A022FC5ED6C8AE5
:100CC00078EEE77A67EEA97AC4ED167A3CD1B0EEF9
:100CD000490A784E48F07AF9D5ED6D7A9FED770A9A
:100CE00000B279EE677A85ED6D9A3080708067EE9C
:100CF000A97A27EE800AC4ED177A48F067F9F080E8
:100D000011E6B0EE480A6B4E48F060F9D5ED6B7A0B
:100D10009FED6A0A00B278EE677A85ED6B8A3080C3
:100D2000708067EEA97A27EE800AC4ED157A48F044
:100D30004DF9D5ED6C7AF08078EEE77AC5ED6C8AE6
:100D400067EEA97AC4ED167AD5ED6D7A85ED6D9AC8
:100D500079EE677A67EEA97AC4ED177AE3E5D5ED07
:100D6000676A002194ED127A0022F8EEE66AD4ED6B
:100D7000137A94ED146A012FA16476EE876A95EDDB
:100D8000687A1A80B8EEC77AE164FDEEE66A5A80A6
:100D9000216537EE277AD5ED697AC5ED676AF8EEF9
:100DA000E77A9A80BDEEC77A77EE867A85ED687A23
:100DB000FDEEE77AC5ED697A7FF431AF0B2085F857
:100DC000A82185F8A97109F0DDFFB36AD5F8902153
:100DD000D5F898111A60B5F894219A80364AD160F6
:100DE0001DE7B8F1040F7FF4C5AE48F0EFF89FEDB2
:100DF000330ADFF8C09028EE000AA9F8020048F094
:100E0000E5F8A9F80600B5E6B8F1040F7FF4B2AE34
:100E1000B0EE490A48F0DAF8264B1880AAE6B8F195
:100E2000040F7FF483AEB0EE680A48F0CFF8214B90
:100E300018807BE6B0EE680A1E4E48F0C7F8D5ED84
:100E40006C7A9FED1E0A00B278EEE77AC5ED6C8AE7
:100E50003080708067EEA97A27EE800AC4ED167A9A
:100E600048F0B4F8F0806FE7DFF858E0C831C837D1
:100E7000C8304FEAE1788EFB0191C8EBE111B4F87C
:100E80000C80A1EB080199808EFB0781FF17C7EB4F
:100E9000E1178EFB001EC0171F80C0EBEE105880BC
:100EA000054BC3F80A20A3F80EC0F8F755FCB28D25
:100EB000B36AC3E504300024846300240AD7233CCA
:100EC000F07D00241F85EB514B4B1B68190700D4A4
:100ED00070472DE9F047494F0546494C2DED108BE1
:100EE0003978D4F8C8315829D4F8B821C4F8B801F1
:100EF000187800F0F881012800F0A6824149D4F862
:100F0000C031A1F58070984797F8008080F001000B
:100F1000B8F1580FC0B265D0002840F0B682B4F9DD
:100F2000BC3294F8881206EE903AB4F9BE32092920
:100F300007EE103AB4F9C032F8EEE66A07EE903ADE
:100F4000B8EEC77A4FF00103F8EEE77AC4EDB26A63
:100F500084EDB37A84F8C432C4EDB47A45D02A481B
:100F600020F040FF94F8D492B9F1000F58D1DFF887
:100F7000ACA0264EB6F90830B8F1570F94EDB29AEE
:100F800007EE903AB6F90A3094EDB38AF8EEE77AB4
:100F900007EE103AB6F90C30B8EEC77AD4EDB48A41
:100FA00039EE679A07EE903AF8EEE77A38EE478A1C
:100FB00084EDB29A78EEE78A84EDB38AC4EDB48A00
:100FC00000F09A81B8F1580F00F01F82104B0122F7
:100FD0001B688AF80020002B40F05D82BDEC108B6E
:100FE000BDE8F0870B4B588196E70B4901F13C00B7
:100FF00020F090FEB6E700BF7C660024003000249D
:10100000F07D0024AC800024B88000244C630024D0
:1010100094060024043000247C800024383600200C
:10102000D4F8D83294F8D5225B1B002B40F3C08152
:10103000DFF878A39FEDD46ADAED027ADAED016A7F
:1010400067EEA77A9AED037AE6EEA67AE7EE077ADC
:10105000F4EE467AF1EE10FA40F34081012A00F0F6
:101060003D810D20C94E09F08DFE0023B360B38190
:10107000012384F8D532F4F7FFFAC54B97F80080C6
:101080000344C4F8D832C34B1A6852B1C24B91889A
:101090001B781268DB4303F001031B0101FA03F321
:1010A000936194EDB30AD4EDB23A60EE006AD4EDE8
:1010B000B40A94EDC08A94EDB85AE3EEA36AD4ED75
:1010C000D07AB0EE45AA94EDC5FA94EDC12A23EE8C
:1010D0008F7AD4EDCAFAD4EDC61A60EE2F5A94ED89
:1010E000C24AE0EEA06AD4EDCBDA94EDC7DAE3EEC3
:1010F000A15A94EDCF3A94EDD2EA20EE833A94EDE2
:10110000C3CAD4EDBE8A26EE886AD4EDD3EAA6EE31
:10111000827A94EDBD9AE6EE845AD4EDBC9A66EEDE
:10112000272AA6EE22AA65EE8E4AF0EE64BA87EE72
:101130008A6AF0EE4AAA60EE2D7AE3EE8D7A73EEBB
:10114000277A84EDD06A94EDD16AE6EE8C7A27EEA8
:10115000061A87EE0A6AE7EE01AAB0EE427AA6EE18
:10116000627AB0EE626AA2EE016AB0EE412A84EDC4
:10117000C17A27EE017AA1EEA42AA8EE227A85EEA2
:10118000AA8AF0EE6A2AE5EEA42AF0EE445AC7EEE7
:10119000A2CAE8EE465AE8EE411A20EE288AA4EEEA
:1011A000246AB0EE454AA3EE898AA5EEA47AC4ED7E
:1011B000C25A67EEAE5AC4EDC61AB0EE62BAA3EEDA
:1011C000254AB7EE003AA7EEA5BAE5EEADBA73EE42
:1011D000487A94EDBF8AE0EEC87AF0EE6D0AECEE44
:1011E000E40AE6EEE97AC4EDCB0A65EEA00A67EE02
:1011F000ABBAEFEEA40AA0EE204AB0EE4C0AF0EE35
:101200004D0AACEEC60AECEEC20AA5EE8C6AA5EE5B
:101210008D2AA5EE807A84EDC30AC4EDC70A65EE77
:10122000A00A27EE866A27EE822AEFEE010A67EE11
:10123000A57AA6EE874A83EE0B7AE1EEA40A25EEA4
:101240000BBAA3EEA04AE7EE069A82EE8B6A65EE31
:10125000222AC5EE046A2AEE855ACAEEA24AA7EEF1
:10126000278AA7EE029AEBEE878A8AEE057A83EE4A
:10127000294A24EE8E5AD4EDD14A26EE2E6AFEEE8D
:10128000007A84EDD25A66EEA66A84EDD36A69EEDE
:10129000275A27EE247A28EEA76A68EE277A84ED8B
:1012A000D17A94EDB77A65EE845AC4EDBC9A33EEE8
:1012B000473A84EDBD9A26EE046AC4EDBE8A67EE15
:1012C000847A84EDBF8AA3EE267AC4EDB95A84ED00
:1012D000BA6AC4EDBB7A84EDB87A4BE62B4E002A8D
:1012E0003FF448AECFE6AA1A2C4E0128B28100F096
:1012F000D6800023338101E6284EB0EE490A47F03C
:1013000065FE94EDB90A308047F060FEB0EE480A01
:10131000308147F05BFE94EDBA0A708047F056FECC
:10132000B0EE680A708147F051FE94EDBB0AB080C0
:1013300047F04CFE28EE080AB081A9EE090AA8EE93
:10134000A80AB1EEC00A47F041FEF080B9F1000FE3
:1013500013D094F8D53283B1D4EDB76A9FED107AEB
:101360009FED106A37EE667AD4EDB87A77EEE67ABA
:1013700086EE070A20EE270A01E09FED0B0A47F0F0
:1013800025FEF08122E600BFFF41EF474C630024B9
:1013900080C3C901202300242C230024043000240E
:1013A0000800803F0000FA440000000038360020AA
:1013B000002A65D094EDB90A4FF00108414E47F07C
:1013C00005FE94EDBA0A308147F000FE94EDBB0AA9
:1013D000708147F0FBFDB081012009F0D3FC3A4B4E
:1013E00083F80080394B83F80E80F8F77FF9F7F720
:1013F000EFFE404609F070FD4FF0000997F80080BD
:10140000DFF8D8A084F8D492B4E5D4F85063C4F8D7
:101410005053F4F731F93B78582B7FF4D7ADAE1B1E
:10142000DFED2B6A2B4B282207EE906A401B1A80B7
:10143000B8EEE77A9E80D880C6EE877AFCEEE77A2F
:1014400017EE902A5A80C1E593F904206421224BBB
:1014500001FB023393F85920202A04D19B699B6930
:101460001B047FF54BAD1D4A01214FF4FA73117037
:101470001B4A1268BDEC108B12681361BDE8F0873F
:101480000C20104E09F07EFCB6E7144A01214FF4FF
:101490007A731170ECE70A2BB8BF0A23E8E793F9D7
:1014A000042064210C4B01FB023393F85920202ABD
:1014B00002D001233381D6E79B699B691A04F8D4D3
:1014C00017E700BF4C6300240035002038350024A6
:1014D00000247449043000242424002438360020D9
:1014E000343600202DE9F04FDFF850B393B09BF86D
:1014F00054330390022B019329D114F04FFE12F0C4
:10150000ADFB9BF8155115F0010500F00F8300238A
:10151000BE4A1C4602928BF85433029B1B784BB395
:10152000BB4B1B78472B08D10199BA4A0BEB8103BF
:10153000D3F8AC359B1122F811300BEB8404D4F8AE
:10154000AC359B11CBF8B83513B0BDE8F08F012452
:10155000B14B1C70019BA3422AD013F0F3F8002872
:10156000D5D0AA4A234602928BF85433029B1B78AB
:10157000002BD5D1F4F780F8039B019AC3F1010346
:101580001844A64B1B68DD690BEB82039200D3F86D
:10159000AC35E9099E11B6EBD51F01D08B0199112D
:1015A00088425A4440F3D9848001C2F8AC05B7E7B9
:1015B00015F03CFD9BF859339FED997A054607EEEF
:1015C000903A9BF81531F8EEE77A13F0010F954B3E
:1015D00067EE877A0493FCEEE77A17EE904A40F0C4
:1015E0001A87039B1C44CBF86043DBF86C23550738
:1015F00000F183849BF87033002B00F0BD84DFF88A
:101600004082824B0293049BD3F8009019F0040FA0
:1016100040F0048600230DF12C0A0D930B930C93DC
:10162000CDE90E3304231093DBF8D433002B45DDD2
:101630007D4E7E4D3344CDF81480009306E0BEF11C
:101640002F0F40F2B280009BB34233D016F8014B0B
:1016500004EB44004FEA4409034615F810E005EB9B
:1016600040004FEA430C0EF01F0201234FEA5E17C1
:10167000804603FA02F212ABB90003EB870353F87A
:101680000C3C1340DBD00BEB0103D3F86833134061
:1016900000F0D8800DAB0DA953F8273023EA0203E0
:1016A00041F827305AF8273013434AF82730009B77
:1016B000B342CBD1DDE90438D3F80090DBF8F46312
:1016C000002E2BDD5A4C0127584D264414F8010BEF
:1016D00052460DA900EB400305EB430393F805C008
:1016E000184612AB4FEA5C1E0CF01F0C03EB8E0E7B
:1016F00007FA0CFC5EF81C3C1CEA030F5EF8143C75
:101700000CEA030C14BF01230023BCF1000F18BF27
:1017100083F0010315F0C2FCA642D7D10B9B09F45C
:1017200080090D9A53400E9A0B9303F4000359EA73
:1017300003090C9B83EA02030C933E4B9AE80300D7
:1017400083E8030014BF012300238BF85B339BF86D
:10175000D033002B40F093859BF80530002B00F030
:1017600096859BF8157107F00105DBF868339C0737
:1017700040F19B80D8F80020900740F19B80BBF897
:101780005C43E10700F1B48044F00106A642ABF8E7
:101790005C6308D0284B41F202420E201A80FF22DF
:1017A0009A7009F0EFFA3446A2E00CF1020C41788D
:1017B00005EB0C0015F80C20407882421FD20BEB91
:1017C000810140F28334192740F6330CD1EDE17AE0
:1017D00017FB0241FDEEE77A17EE902A6245A8BF9B
:1017E0006246B2F5617FB8BF4FF461728A4206DD8E
:1017F00017FB00403B468242CCBF002301234046FA
:1018000052460DA915F04AFC1DE700BF0035002027
:101810000030002404300024383600203436002004
:101820000024744968350024C8810024A063002482
:10183000E88100245881002444780024F07D0024AD
:101840007C6600240CF1020C407805EB0C0715F8BF
:101850000CC097F801E0F44519D20BEB8000192772
:10186000D0EDE17A40F28330FDEEE77A17FB0C0C05
:1018700040F6330717EE900AB842A8BF3846B0F5D5
:10188000617FB8BF4FF46170604500F36B831F4602
:101890005944D1F8EC331A4200F017813B464046D8
:1018A00052460DA915F0FAFBCDE6944AD278002AEB
:1018B0007FF460AFBBF85C6326F00104F207A4B2CA
:1018C000ABF85C4302D45B0712D50CE08C4B41F2C1
:1018D00002420E201A80FF229A7009F053FADBF8B8
:1018E0006833590704D5D8F80030980700F1E1872C
:1018F00024F00206A307B6B2ABF85C630FD4F5B1CF
:10190000DBF868335C0515D5300540F1CC803446F2
:101910001FE044F00206B442ABF85C63EFD0784BB2
:1019200041F202420E201A80FF229A7009F02AFA30
:101930002DB1E5E7714AD278002A40F05A8626F4A4
:1019400000643105A4B2ABF85C4300F1B480DBF86D
:1019500068336C4A14F02B0F6B491278496802F017
